:020000040800F2
:1000000000060020E1010008E3010008E301000808
:10001000E3010008E3010008E3010008E301000830
:10002000E3010008E3010008E30100089D2F000838
:10003000E3010008E3010008E3010008E301000810
:10004000E3010008E3010008E3010008E301000800
:10005000E3010008E3010008453200086D320008A2
:1000600095320008BD320008E5320008E3010008BF
:10007000E3010008E3010008E3010008E3010008D0
:10008000E3010008E3010008E3010008E3010008C0
:10009000E3010008E3010008E30100080D33000854
:1000A000E3010008E3010008E3010008E3010008A0
:1000B000E1330008E3010008E3010008E301000860
:1000C000E3010008E3010008E3010008E301000880
:1000D000E3010008E3010008E3010008E301000870
:1000E00071330008E3010008E3010008E3010008A0
:1000F000E3010008E3010008E3010008E301000850
:10010000E3010008E3010008E3010008E30100083F
:10011000E3010008E3010008E3010008E30100082F
:10012000E3010008E3010008E3010008E30100081F
:10013000E3010008E3010008E3010008E30100080F
:10014000E3010008E3010008E3010008512700086B
:10015000E3010008E3010008E3010008E3010008EF
:10016000E3010008E3010008E3010008E3010008DF
:10017000E3010008E3010008E3010008E3010008CF
:10018000E3010008E3010008E3010008E3010008BF
:10019000E3010008E3010008E3010008E3010008AF
:1001A000E3010008E3010008E3010008E30100089F
:1001B000E3010008E3010008E3010008E30100088F
:1001C000E3010008E3010008E3010008E30100087F
:1001D000E3010008E3010008E3010008E30100086F
:1001E00002E000F000F8FEE772B6374880F30888B6
:1001F000364880F3098836483649086040F20000E6
:10020000CCF200004EF63471CEF200010860BFF36C
:100210004F8FBFF36F8F40F20000C0F2F0004EF638
:100220008851CEF200010860BFF34F8FBFF36F8F8C
:100230004FF00000E1EE100A4EF63C71CEF20001E4
:100240000860062080F31488BFF36F8F01F048FF29
:1002500002F042FE4FF055301F491B4A91423CBF0D
:1002600041F8040BFAE71D49184A91423CBF41F896
:10027000040BFAE71A491B4A1B4B9A423EBF51F83E
:10028000040B42F8040BF8E700201849184A914281
:100290003CBF41F8040BFAE701F026FF02F070FEC4
:1002A000144C154DAC4203DA54F8041B8847F9E7A7
:1002B00000F042F8114C124DAC4203DA54F8041B22
:1002C0008847F9E701F00EBF000600200022002059
:1002D0000000000808ED00E00000002000060020FB
:1002E000A8370008002200204022002040220020E1
:1002F000602E0020E0010008E0010008E001000895
:10030000E00100082DE9F04F2DED108AC1F80CD066
:10031000C3689D46BDEC108ABDE8F08F002383F3CF
:1003200011882846A047002001F08AFAFEE701F074
:1003300019FA00DFFEE7000038B500F0BFFB01F05E
:100340009FFE054601F0C2FE0446C8B90E4B9D4211
:1003500018D001339D4218BF044641F2883504BFCE
:1003600001240025002001F095FE0CB100F074F886
:1003700000F018FD284600F0C3F800F06DF8F9E72A
:100380000025EFE70546EDE7010007B008B500F0EE
:1003900067FBA0F120035842584108BD07B541F260
:1003A0001203022101A8ADF8043000F077FB03B07E
:1003B0005DF804FB38B5302383F3118817480368D0
:1003C0000BB101F009FB164A144800234FF47A716F
:1003D00001F0F8FA002383F31188124C236813B15B
:1003E0002368013B2360636813B16368013B63606A
:1003F0000D4D2B7833B963687BB9022000F034FCD3
:10040000322363602B78032B07D163682BB902205A
:1004100000F02AFC4FF47A73636038BD402200205C
:10042000B50300086023002058220020084B1870F4
:1004300003280CD8DFE800F008050208022000F0CD
:1004400003BC022000F0F0BB024B00225A60704750
:100450005822002060230020244B254A10B51C465A
:100460001968013140D004339342F9D16268214BBD
:100470009A4239D9204B9B6803F1006303F580331E
:100480009A4231D2002000F033FB0220FFF7CEFF6A
:100490001A4B1A6C00221A64196E1A66196E596C7E
:1004A0005A64596E5A665A6E5A6942F080025A610D
:1004B0005A6922F080025A615A691A6942F0005260
:1004C0001A611A6922F000521A611B6972B64FF064
:1004D000E0233021C3F8084DD4E9003281F31188BC
:1004E0009D4683F30888104710BD00BF0000010837
:1004F00020000108FFFF0008002200200038024011
:100500002DE9F04F93B0AA4B00902022FF210AA8BA
:100510009D6800F0F1FBA74A1378A3B9A648012112
:1005200003601170302383F3118803680BB101F06D
:1005300053FAA24AA04800234FF47A7101F042FA1C
:10054000002383F31188009B13B19D4B009A1A601E
:100550009C4A009C1378032B1EBF00231370984AFB
:100560004FF0000A18BF5360D3465646D1460120CB
:1005700000F06AFB24B1924B1B68002B00F0118243
:10058000002000F06DFA0390039B002BF2DB0120AA
:1005900000F04AFB039B213B162BE8D801A252F83E
:1005A00023F000BF0106000829060008BD06000868
:1005B0006F0500086F0500086F0500084707000871
:1005C000170900083108000893080008BB08000854
:1005D000E10800086F050008F30800086F0500082F
:1005E00065090008A10600086F050008A9090008B0
:1005F0000D060008A10600086F0500089308000812
:100600000220FFF7C3FE002840F0F581009B022185
:10061000BAF1000F08BF1C4605A841F21233ADF82D
:10062000143000F03BFAA2E74FF47A7000F018FAA9
:10063000071EEBDB0220FFF7A9FE0028E6D0013FF2
:10064000052F00F2DA81DFE807F0030A0D101336F8
:1006500005230593042105A800F020FA17E054486B
:100660000421F9E758480421F6E758480421F3E744
:100670004FF01C08404600F03DFA08F104080590D0
:10068000042105A800F00AFAB8F12C0FF2D10120DC
:1006900000FA07F747EA0B0B5FFA8BFB4FF00009F4
:1006A00000F076FB26B10BF00B030B2B08BF0024E8
:1006B000FFF774FE5BE746480421CDE7002EA5D086
:1006C0000BF00B030B2BA1D10220FFF75FFE0746B7
:1006D00000289BD0012000F00BFA0220FFF7A6FEB5
:1006E00000261FFA86F8404600F012FA044690B140
:1006F0000021404600F01CFA01360028F1D1BA462C
:10070000044641F21213022105A8ADF814303E460A
:1007100000F0C4F92BE70120FFF788FE2546244BA3
:100720009B68AB4207D9284600F0E4F9013040F05D
:1007300067810435F3E7234B00251D70204BBA4633
:100740005D603E46ACE7002E3FF460AF0BF00B035C
:100750000B2B7FF45BAF0220FFF768FE322000F026
:100760007FF9B0F10008FFF651AF18F003077FF4EE
:100770004DAF0F4A926808EB050393423FF646AF30
:10078000B8F5807F3FF742AF124B0193B84523DDA8
:100790004FF47A7000F064F90390039A002AFFF690
:1007A00035AF019B039A03F8012B0137EDE700BF3A
:1007B000002200205C23002040220020B503000816
:1007C000602300205822002004220020082200205C
:1007D0000C2200205C220020C820FFF7D7FD07462E
:1007E00000283FF413AF1F2D11D8C5F12002424558
:1007F0000AAB25F0030028BF424683490192184402
:1008000000F054FA019A8048FF2100F075FA4FEA8F
:10081000A8037D490193C8F38702284600F074FAC3
:10082000064600283FF46DAF019B05EB830537E7D3
:100830000220FFF7ABFD00283FF4E8AE00F0A4F97A
:1008400000283FF4E3AE0027B846704B9B68BB42DC
:1008500018D91F2F11D80A9B01330ED027F003039C
:1008600012AA134453F8203C05934046042205A9DC
:1008700000F0C2FA04378046E7E7384600F03AF95C
:100880000590F2E7CDF81480042105A800F006F9E0
:1008900006E70023642104A8049300F0F5F800287B
:1008A0007FF4B4AE0220FFF771FD00283FF4AEAE36
:1008B000049800F051F90590E6E70023642104A8AC
:1008C000049300F0E1F800287FF4A0AE0220FFF7C7
:1008D0005DFD00283FF49AAE049800F04DF9EAE778
:1008E0000220FFF753FD00283FF490AE00F05CF9C2
:1008F000E1E70220FFF74AFD00283FF487AE05A993
:10090000142000F057F904210746049004A800F0D1
:10091000C5F83946B9E7322000F0A2F8071EFFF605
:1009200075AEBB077FF472AE384A926807EB0903D5
:1009300093423FF66BAE0220FFF728FD00283FF4FC
:1009400065AE27F003074F44B9453FF4A9AE4846CA
:1009500000F0D0F80421059005A800F09FF809F1F7
:100960000409F1E74FF47A70FFF710FD00283FF417
:100970004DAE00F009F9002844D00A9B01330BD09A
:1009800008220AA9002000F0BFF900283AD020224E
:10099000FF210AA800F0B0F9FFF700FD1C4800F0A5
:1009A00055FF13B0BDE8F08F002E3FF42FAE0BF0D3
:1009B0000B030B2B7FF42AAE0023642105A80593BB
:1009C00000F062F8074600287FF420AE0220FFF70F
:1009D000DDFC804600283FF419AEFFF7DFFC41F252
:1009E000883000F033FF059800F004FA464600F026
:1009F000CFF93C46BBE5064652E64FF0000905E656
:100A0000BA467EE637467CE65C22002000220020C3
:100A1000A086010070B50F4B1B780133DBB2012BB0
:100A20000C4611D80C4D29684FF47A730E6AA2FB5C
:100A30000332014622462846B047844204D1074B80
:100A400000221A70012070BD4FF4FA7000F0FEFE13
:100A50000020F8E710220020082600209423002020
:100A600007B50023024601210DF107008DF807307C
:100A7000FFF7D0FF20B19DF8070003B05DF804FB3D
:100A80004FF0FF30F9E700000A4608B50421FFF7F0
:100A9000C1FF80F00100C0B2404208BD30B4054C37
:100AA0002368DD69044B0A46AC460146204630BC4B
:100AB000604700BF08260020A086010070B501F045
:100AC000E5F9094E094D30800024286833888342B7
:100AD00008D901F0D5F92B6804440133B4F5803FFF
:100AE0002B60F2D370BD00BF962300206823002046
:100AF00001F07ABA00F1006000F5803000687047BC
:100B000000F10060920000F5803001F005BA0000AD
:100B1000054B1A68054B1B889B1A834202D9104467
:100B200001F0AEB900207047682300209623002012
:100B300038B5084D044629B128682044BDE838403E
:100B400001F0BEB92868204401F0A2F90028F3D0D2
:100B500038BD00BF6823002010F003030AD1B0F5B0
:100B6000047F05D200F10050A0F51040D0F8003805
:100B7000184670470023FBE700F10050A0F5104035
:100B8000D0F8100A70470000064991F8243033B1BC
:100B90000023086A81F824300822FFF7B1BF012042
:100BA000704700BF6C230020014B1868704700BFDE
:100BB000002004E070B5194B1D68194B0138C5F3CE
:100BC0000B0408442D0C04221E88A6420BD15C683D
:100BD0000A46013C824213460FD214F9016F4EB10E
:100BE00002F8016BF6E7013A03F10803ECD1814208
:100BF0000B4602D22C2203F8012B0A4A0524168840
:100C0000AE4204D1984284BF967803F8016B013C50
:100C100002F10402F3D1581A70BD00BF002004E0B5
:100C2000C4340008B0340008022804D1054B4FF04A
:100C300080429A6170470128FCD1024B4FF000526C
:100C4000F7E700BF00000240022804D1054B4FF433
:100C500080429A6170470128FCD1024B4FF4005248
:100C6000F7E700BF00000240022805D1064A536999
:100C700083F48043536170470128FCD1024A5369D1
:100C800083F40053F6E700BF0000024070B504464D
:100C90004FF47A764CB1412C254628BF412506FBFE
:100CA00005F000F0D3FD641BF4E770BD10B5002320
:100CB000934203D0CC5CC4540133F9E710BD00006B
:100CC00010B5013810F9013F3BB191F900409C4249
:100CD00003D11AB10131013AF4E71AB191F90020B8
:100CE000981A10BD1046FCE703460246D01A12F9C6
:100CF000011B0029FAD1704702440346934202D0F7
:100D000003F8011BFAE770472DE9F8431F4D14461D
:100D100095F824200746884652BBDFF870909CB3B4
:100D200095F824302BB92022FF2148462F62FFF787
:100D3000E3FF95F82400C0F10802A24228BF224632
:100D4000D6B24146920005EB8000FFF7AFFF95F861
:100D50002430A41B1E44F6B2082E17449044E4B27B
:100D600085F82460DBD1FFF70FFF0028D7D108E01A
:100D70002B6A03EB82038342CFD0FFF705FF0028E5
:100D8000CBD10020BDE8F8830120FBE76C230020D5
:100D9000024B1A78024B1A70704700BF9423002050
:100DA0001022002010B5104C104800F0B5F8214674
:100DB0000E4800F0DDF82468626DD2F8043843F084
:100DC0000203C2F804384FF47A70FFF75FFF084956
:100DD000204600F0D3F9626DD2F8043823F0020304
:100DE000C2F8043810BD00BF903500080826002066
:100DF000983500087047000030B5094D0A4491420B
:100E00000DD011F8013B5840082340F30004013B8A
:100E10002C4013F0FF0384EA5000F6D1EFE730BD19
:100E20002083B8ED026843681143016003B118479D
:100E30007047000013B5446BD4F894341A681178E5
:100E4000042915D1217C022912D119791289012393
:100E50008B4013420CD101A904F14C0001F0F8FEC3
:100E6000D4F89444019B21790246206800F0D0F91F
:100E700002B010BD143001F07BBE00004FF0FF3314
:100E8000143001F075BE00004C3001F04DBF000081
:100E90004FF0FF334C3001F047BF0000143001F039
:100EA00049BE00004FF0FF31143001F043BE000096
:100EB0004C3001F019BF00004FF0FF324C3001F010
:100EC00013BF00000020704710B5D0F894341A68A2
:100ED00011780429044617D1017C022914D15979CB
:100EE000528901238B4013420ED1143001F0DCFDF6
:100EF000024648B1D4F894444FF480736179206875
:100F0000BDE8104000F072B910BD0000406BFFF763
:100F1000DBBF0000704700007FB5124B0360002369
:100F20004360C0E90233012502260F4B05740446D5
:100F30000290019300F18402294600964FF48073D9
:100F4000143001F08DFD094B0294CDE9006304F5E6
:100F500023724FF48073294604F14C0001F054FED3
:100F600004B070BDE43400080D0F0008350E000811
:100F70000B68302282F311880A7903EB82029061B8
:100F80004A79093243F822008A7912B103EB8203CD
:100F900098610223C0F894140374002080F3118830
:100FA0007047000038B5037F044613B190F8543001
:100FB000ABB9201D01250221FFF734FF04F1140015
:100FC00025776FF0010100F069FC84F8545004F1BA
:100FD0004C006FF00101BDE8384000F05FBC38BD47
:100FE00010B5012104460430FFF71CFF00232377CE
:100FF00084F8543010BD000038B504460025143084
:1010000001F046FD04F14C00257701F015FE201D8E
:1010100084F854500121FFF705FF2046BDE8384011
:10102000FFF752BF90F8443003F06003202B07D144
:1010300090F84520212A4FF0000303D81F2A06D834
:1010400000207047222AFBD1C0E90E3303E0034A97
:1010500082630722C26303640120704711220020CB
:1010600037B5D0F894341A681178042904461AD197
:10107000017C022917D11979128901238B4013426F
:1010800011D100F14C05284601F096FE58B101A996
:10109000284601F0DDFDD4F89444019B21790246F5
:1010A000206800F0B5F803B030BD0000F0B500EBEB
:1010B000810385B09E6904460D46FEB1302383F35B
:1010C000118804EB8507301D0821FFF7ABFEFB6894
:1010D0005B691B6806F14C001BB1019001F0C6FD75
:1010E000019803A901F0B4FD024648B1039B2946CB
:1010F000204600F08DF8002383F3118805B0F0BD81
:10110000FB685A691268002AF5D01B8A013B13401C
:10111000F1D104F14402EAE7093138B550F8214031
:10112000DCB1302383F31188D4F894241368527906
:1011300003EB8203DB689B695D6845B1042160189D
:10114000FFF770FE294604F1140001F0B7FC2046B9
:10115000FFF7BAFE002383F3118838BD7047000003
:1011600001F016B8012303700023C0E90133C36105
:1011700083620362C36243620363704738B5044607
:10118000302383F311880025C0E90355C0E90555D4
:10119000416001F00DF80223237085F31188284681
:1011A00038BD000070B500EB810305465069DA6078
:1011B0000E46144618B110220021FFF79DFDA069CC
:1011C00018B110220021FFF797FD31462846BDE8EF
:1011D000704001F0B7B80000826802F0011282602E
:1011E0000022C0E90422826101F038B9F0B400EBBA
:1011F00081044789E4680125A4698D403D43458108
:1012000023600023A2606360F0BC01F053B90000CA
:10121000F0B400EB81040789E468012564698D401E
:101220003D43058123600023A2606360F0BC01F0B0
:10123000CDB9000070B50223002504460370C0E953
:101240000255C0E90455C564856180F8345001F049
:1012500015F863681B6823B129462046BDE8704035
:10126000184770BD0378052B10B504460AD080F8E6
:1012700050300523037043681B680BB10421984765
:101280000023A36010BD00000178052906D190F865
:101290005020436802701B6803B118477047000074
:1012A00070B590F83430044613B1002380F8343020
:1012B00004F14402204601F0F3F863689B68B3B977
:1012C00094F8443013F0600535D00021204601F039
:1012D00093FB0021204601F085FB63681B6813B176
:1012E000062120469847062384F8343070BD2046F6
:1012F00098470028E4D0B4F84A30E26B9A4288BF9D
:10130000E36394F94430E56B002B4FF0300380F237
:101310000381002D00F0F280092284F8342083F349
:1013200011880021D4E90E232046FFF771FF002326
:1013300083F31188DAE794F8452003F07F0343EA4A
:10134000022340F20232934200F0C58021D8B3F567
:10135000807F48D00DD8012B3FD0022B00F0938026
:10136000002BB2D104F14C02A2630222E263236497
:10137000C1E7B3F5817F00F09B80B3F5407FA4D136
:1013800094F84630012BA0D1B4F84C3043F002035E
:1013900032E0B3F5006F4DD017D8B3F5A06F31D060
:1013A000A3F5C063012B90D8636894F846205E686B
:1013B00094F84710B4F848302046B047002884D04D
:1013C0004368A3630368E3631AE0B3F5106F36D094
:1013D00040F6024293427FF478AF5C4BA363022352
:1013E000E3630023C3E794F84630012B7FF46DAF2D
:1013F000B4F84C3023F00203C4E90E55A4F84C3085
:10140000256478E7B4F84430B3F5A06F0ED194F8B2
:10141000463084F84E30204600F088FF63681B6831
:1014200013B1012120469847032323700023C4E908
:101430000E339CE704F14F03A3630123C3E7237832
:10144000042B10D1302383F311882046FFF7C4FE0C
:1014500085F311880321636884F84F5021701B685D
:101460000BB12046984794F84630002BDED084F824
:101470004F300423237063681B68002BD6D00221F1
:1014800020469847D2E794F848301D0603F00F0134
:1014900020460AD500F0F6FF012804D002287FF488
:1014A00014AF2B4B9AE72B4B98E700F0DDFFF3E7E7
:1014B00094F84630002B7FF408AF94F8483013F0CE
:1014C0000F01B3D01A06204602D501F0A9FAADE704
:1014D00001F09CFAAAE794F84630002B7FF4F5AEB1
:1014E00094F8483013F00F01A0D01B06204602D517
:1014F00001F082FA9AE701F075FA97E7142284F86E
:10150000342083F311882B462A4629462046FFF7CC
:101510006DFE85F31188E9E65DB1152284F834206B
:1015200083F311880021D4E90E232046FFF75EFEE5
:10153000FDE60B2284F8342083F311882B462A46DB
:1015400029462046FFF764FEE3E700BF1435000894
:101550000C3500081035000838B590F834300446D2
:10156000002B3ED0063BDAB20F2A34D80F2B32D8EC
:10157000DFE803F037313108223231313131313196
:1015800031313737C56BB0F84A309D4214D2C36849
:101590001B8AB5FBF3F203FB12556DB9302383F3BD
:1015A00011882B462A462946FFF732FE85F311881B
:1015B0000A2384F834300EE0142384F834303023C6
:1015C00083F3118800231A4619462046FFF70EFEC2
:1015D000002383F3118838BD036C03B198470023BF
:1015E000E7E70021204601F007FA0021204601F03C
:1015F000F9F963681B6813B1062120469847062352
:10160000D7E7000010B590F83430142B044629D0E9
:1016100017D8062B05D001D81BB110BD093B022BF2
:10162000FBD80021204601F0E7F90021204601F017
:10163000D9F963681B6813B1062120469847062331
:1016400019E0152BE9D10B2380F83430302383F3D4
:10165000118800231A461946FFF7DAFD002383F3A9
:101660001188DAE7C3689B695B68002BD5D1036CEE
:1016700003B19847002384F83430CEE70023037584
:10168000826803691B6899689142FBD25A680360BB
:1016900042601060586070470023037582680369D8
:1016A0001B6899689142FBD85A68036042601060D9
:1016B0005860704708B50846302383F311880B7DC6
:1016C000032B05D0042B0DD02BB983F3118808BD53
:1016D0008B6900221A604FF0FF338361FFF7CEFF62
:1016E0000023F2E7D1E9003213605A60F3E700000B
:1016F000FFF7C4BF054BD9680875186802681A60FF
:10170000536001220275D860FEF7FCBD98230020CB
:1017100030B50C4BDD684B1C87B004460FD02B4610
:10172000094A684600F04EF92046FFF7E3FF009BA8
:1017300013B1684600F050F9A86907B030BDFFF753
:10174000D9FFF9E798230020B5160008044B1A6862
:10175000DB6890689B68984294BF00200120704726
:1017600098230020084B10B51C68D86822681A60BE
:10177000536001222275DC60FFF78EFF0146204690
:10178000BDE81040FEF7BEBD9823002038B5074CD9
:1017900007490848012300252370656001F044FBD8
:1017A0000223237085F3118838BD00BF0026002076
:1017B0001C3500089823002000F044B9034A516802
:1017C00053685B1A9842FBD8704700BF001000E0D6
:1017D0008B60022308618B82084670478368A3F1FF
:1017E000840243F8142C026943F8442C426943F8FC
:1017F000402C094A43F8242CC26843F8182C0222D2
:1018000003F80C2C002203F80B2C044A43F8102C8C
:10181000A3F12000704700BF1D030008982300209B
:1018200008B5FFF7DBFFBDE80840FFF761BF000028
:10183000024BDB6898610F20FFF75CBF9823002004
:10184000302383F31188FFF7F3BF000008B501468A
:10185000302383F311880820FFF75AFF002383F316
:10186000118808BD064BDB6839B1426818605A60C0
:10187000136043600420FFF74BBF4FF0FF30704709
:10188000982300200368984206D01A6802605060CE
:1018900099611846FFF72CBF7047000038B5044621
:1018A0000D462068844200D138BD036823605C6027
:1018B0008561FFF71DFFF4E710B503689C68A2423D
:1018C0000CD85C688A600B604C6021605960996834
:1018D0008A1A9A604FF0FF33836010BD1B68121B99
:1018E000ECE700000A2938BF0A2170B504460D460E
:1018F0000A26601901F092FA01F07EFA041BA54253
:1019000003D8751C2E460446F3E70A2E04D9BDE819
:101910007040012001F0C8BA70BD0000F8B5144B4A
:101920000D46D96103F1100141600A2A19698260EC
:1019300038BF0A22016048601861A818144601F0F7
:101940005FFA0A2701F058FA431BA342064606D362
:101950007C1C281901F062FA27463546F2E70A2F67
:1019600004D9BDE8F840012001F09EBAF8BD00BFDF
:1019700098230020F8B506460D4601F03DFA0F4ABF
:10198000134653F8107F9F4206D12A46014630463F
:10199000BDE8F840FFF7C2BFD169BB68441A2C19F3
:1019A00028BF2C46A34202D92946FFF79BFF2246B7
:1019B00031460348BDE8F840FFF77EBF982300207A
:1019C000A823002010B4C0E9032300235DF8044BD2
:1019D0004361FFF7CFBF000010B5194C236998424F
:1019E0000DD0D0E90032816813605A609A680A44C9
:1019F0009A60002303604FF0FF33A36110BD2346BC
:101A0000026843F8102F53600022026022699A4254
:101A100003D1BDE8104001F0FBB9936881680B4425
:101A2000936001F0E9F92269E1699268441AA242DF
:101A3000E4D91144BDE81040091AFFF753BF00BFB5
:101A4000982300202DE9F047DFF8BC8008F110074B
:101A50002C4ED8F8105001F0CFF9D8F81C40AA68E5
:101A6000031B9A423ED81444D5E900324FF00009D6
:101A7000C8F81C4013605A60C5F80090D8F81030C0
:101A8000B34201D101F0C4F989F31188D5E90331DA
:101A900028469847302383F311886B69002BD8D0F0
:101AA00001F0AAF96A69A0EB04094A4582460DD201
:101AB000022001F0F9F90022D8F81030B34208D121
:101AC00051462846BDE8F047FFF728BF121A2244C6
:101AD000F2E712EB090938BF4A4629463846FFF7B4
:101AE000EBFEB5E7D8F81030B34208D01444211A01
:101AF000C8F81C00A960BDE8F047FFF7F3BEBDE8D9
:101B0000F08700BFA8230020982300200020704702
:101B1000FEE70000704700004FF0FF307047000004
:101B200002290CD0032904D00129074818BF00203E
:101B30007047032A05D8054800EBC20070470448E7
:101B400070470020704700BFF435000820220020B5
:101B5000A835000870B59AB00546084601A9144694
:101B600000F0C2F801A8FFF7BFF8431C5B00C5E90D
:101B700000340022237003236370C6B201AB023429
:101B80001046D1B28E4204F1020401D81AB070BDE1
:101B900013F8011B04F8021C04F8010C0132F0E7F1
:101BA00008B5302383F311880348FFF759FA00235F
:101BB00083F3118808BD00BF0826002090F8443048
:101BC00003F01F02012A07D190F845200B2A03D108
:101BD0000023C0E90E3315E003F06003202B08D189
:101BE000B0F848302BB990F84520212A03D81F2A95
:101BF00004D8FFF717BA222AEBD0FAE7034A826328
:101C00000722C26303640120704700BF182200202E
:101C100007B5052917D8DFE801F0191603191920AF
:101C2000302383F31188104A01900121FFF7BAFA9B
:101C300001980E4A0221FFF7B5FA0D48FFF7DCF9CB
:101C4000002383F3118803B05DF804FB302383F392
:101C500011880748FFF7A6F9F2E7302383F31188CC
:101C60000348FFF7BDF9EBE7483500086C3500087D
:101C70000826002038B50C4D0C4C0D492A4604F1BD
:101C80000800FFF767FF05F1CA0204F110000949D7
:101C9000FFF760FF05F5CA7204F118000649BDE8B8
:101CA0003840FFF757BF00BFD02A00202022002075
:101CB00028350008323500083D35000870B5044667
:101CC00008460D46FFF710F8C6B2204601340378E7
:101CD0000BB9184670BD32462946FEF7F1FF0028C1
:101CE000F3D10120F6E700002DE9F04705460C4648
:101CF000FEF7FAFF2B49C6B22846FFF7DFFF08B10F
:101D00000736F6B228492846FFF7D8FF08B1103643
:101D1000F6B2632E0BD8DFF88C80DFF88C90234F5F
:101D2000DFF894A02E7846B92670BDE8F0872946E2
:101D30002046BDE8F04701F09DBB252E2ED107229D
:101D400041462846FEF7BCFF70B9194B224603F105
:101D50000C0153F8040B42F8040B8B42F9D11B8899
:101D6000138007350E34DDE7082249462846FEF782
:101D7000A7FF98B90F4BA21C197809090232C95D57
:101D800002F8041C13F8011B01F00F015345C95D53
:101D900002F8031CF0D118340835C3E704F8016BCE
:101DA0000135BFE7143600083D3500082B36000822
:101DB0001C360008107AFF1F1C7AFF1FBFF34F8FDD
:101DC000024AD368DB03FCD4704700BF003C0240EA
:101DD00008B5094B1B7873B9FFF7F0FF074B1A6979
:101DE000002ABFBF064A5A6002F188325A601A6858
:101DF00022F480621A6008BD2E2D0020003C0240B3
:101E00002301674508B50B4B1B7893B9FFF7D6FF45
:101E1000094B1A6942F000421A611A6842F4805272
:101E20001A601A6822F480521A601A6842F48062BA
:101E30001A6008BD2E2D0020003C02400B28F0B592
:101E400016D80C4C0C4923787BB90C4D0E460C234C
:101E50004FF0006255F8047B46F8042B013B13F069
:101E6000FF033A44F6D10123237051F82000F0BD5E
:101E70000020FCE7602D0020302D00203C360008BB
:101E8000014B53F8200070473C3600080C20704787
:101E90000B2810B5044601D9002010BDFFF7CEFF76
:101EA000064B53F824301844C21A0BB90120F4E74A
:101EB00012680132F0D1043BF6E700BF3C3600085F
:101EC0000B2810B5044621D8FFF778FFFFF780FFF5
:101ED0000F4AF323D360C300DBB243F4007343F033
:101EE00002031361136943F480331361FFF766FF44
:101EF000FFF7A4FF074B53F8241000F0D9F8FFF7C1
:101F000081FF2046BDE81040FFF7C2BF002010BD92
:101F1000003C02403C360008F8B512F001031446BC
:101F200042D18218B2F1016F57D82D4B1B6813F0C4
:101F3000010352D02B4DFFF74BFFF323EB60FFF76C
:101F40003DFF40F20127032C15D824F00104661848
:101F5000244C401A40F20117B142236900EB0105FD
:101F600024D123F001032361FFF74CFF0120F8BDCA
:101F7000043C0430E7E78307E7D12B6923F440737F
:101F80002B612B693B432B6151F8046B0660BFF357
:101F90004F8FFFF713FF03689E42E9D02B6923F0B0
:101FA00001032B61FFF72EFF0020E0E723F44073CD
:101FB000236123693B4323610B882B80BFF34F8F41
:101FC000FFF7FCFE2D8831F8023BADB2AB42C3D027
:101FD000236923F001032361E4E71846C7E700BF44
:101FE00000380240003C0240084908B50B7828B18F
:101FF0001BB9FFF7EDFE01230B7008BD002BFCD0D1
:10200000BDE808400870FFF7FDBE00BF2E2D002080
:1020100010B50244064BD2B2904200D110BD441C10
:1020200000B253F8200041F8040BE0B2F4E700BF1F
:10203000502800400F4B30B51C6F240407D41C6F90
:1020400044F400741C671C6F44F400441C670A4C81
:10205000236843F4807323600244084BD2B2904259
:1020600000D130BD441C00B251F8045B43F820504D
:10207000E0B2F4E700380240007000405028004011
:1020800007B5012201A90020FFF7C2FF019803B0A4
:102090005DF804FB13B50446FFF7F2FFA04205D03C
:1020A000012201A900200194FFF7C4FF02B010BD76
:1020B00070470000034B1A681AB9034AD2F8742813
:1020C0001A607047642D00200030024008B5FFF709
:1020D000F1FF024B1868C0F3407008BD642D00206A
:1020E00070470000FEE700000A4B0B480B4A904285
:1020F0000BD30B4BDA1C121AC11E22F003028B42C7
:1021000038BF00220021FEF7F7BD53F8041B40F84A
:10211000041BECE7E8370008602E0020602E00204A
:10212000602E002070B5D0E915439E6800224FF064
:10213000FF3504EB42135101D3F800090028BEBF5C
:10214000D3F8000940F08040C3F80009D3F8000B31
:102150000028BEBFD3F8000B40F08040C3F8000B4E
:10216000013263189642C3F80859C3F8085BE0D2FD
:102170004FF00113C4F81C3870BD0000890141F014
:102180002001016103699B06FCD41220FFF716BBF6
:1021900010B5054C2046FEF7E5FF4FF0A043636500
:1021A000024BA36510BD00BF682D002090360008CB
:1021B00070B50378012B054650D12A4B446D9842E7
:1021C0001BD1294B5A6B42F080025A635A6D42F080
:1021D00080025A655A6D5A6942F080025A615A6902
:1021E00022F080025A610E2143205B6900F022FC3C
:1021F0001E4BE3601E4BC4F800380023C4F8003EB9
:10220000C02323606E6D4FF40413A3633369002B66
:10221000FCDA012333610C20FFF7D0FA3369DB07C6
:10222000FCD41220FFF7CAFA3369002BFCDA00262F
:10223000A6602846FFF776FF6B68C4F81068DB6875
:10224000C4F81468C4F81C684BB90A4BA3614FF07A
:10225000FF336361A36843F00103A36070BD064BC5
:10226000F4E700BF682D0020003802404014004011
:1022700003002002003C30C0083C30C0F8B5446D7B
:10228000054600212046FFF779FFA96D00234FF096
:1022900001128F68C4F834384FF00066C4F81C2867
:1022A0004FF0FF3004EB431201339F42C2F8006944
:1022B000C2F8006BC2F80809C2F8080BF2D20B682A
:1022C0006A6DEB65636210231361166916F01006E0
:1022D000FBD11220FFF772FAD4F8003823F4FE6322
:1022E000C4F80038A36943F4402343F01003A3610A
:1022F0000923C4F81038C4F814380A4BEB604FF0C7
:10230000C043C4F8103B084BC4F8003BC4F8106944
:10231000C4F80039EB6D03F1100243F48013EA6551
:10232000A362F8BD6C36000840800010426D90F842
:102330004E10D2F8003823F4FE6343EA0113C2F8CA
:10234000003870472DE9F84300EB8103456DDA68EA
:10235000166806F00306731E022B05EB41130C46AC
:1023600080460FFA81F94FEA41104FF00001C3F89F
:10237000101B4FF0010104F1100398BFB60401FADD
:1023800003F391698EBF334E06F1805606F5004681
:1023900000293AD0578A04F15801490137436F5058
:1023A000D5F81C180B43C5F81C382B180021C3F8AE
:1023B000101953690127611EA7409BB3138A928BA2
:1023C0009B08012A88BF5343D8F85C20981842EA3A
:1023D000034301F1400205EB8202C8F85C0021468C
:1023E00053602846FFF7CAFE08EB8900C3681B8AC2
:1023F00043EA8453483464011E432E51D5F81C38F7
:102400001F43C5F81C78BDE8F88305EB4917D7F8DA
:10241000001B21F40041C7F8001BD5F81C1821EA65
:102420000303C0E704F13F0305EB83030A4A5A6044
:1024300028462146FFF7A2FE05EB4910D0F80039E7
:1024400023F40043C0F80039D5F81C3823EA070705
:10245000D7E700BF0080001000040002826D126800
:10246000C265FFF75FBE00005831436D49015B58FC
:1024700013F4004004D013F4001F0CBF022001200D
:10248000704700004831436D49015B5813F4004028
:1024900004D013F4001F0CBF02200120704700007D
:1024A00000EB8101CB68196A0B6813604B685360BD
:1024B0007047000000EB810330B5DD68AA6913683E
:1024C000D36019B9402B84BF402313606B8A146812
:1024D000426D1C44013CB4FBF3F46343033323F02B
:1024E000030302EB411043EAC44343F0C043C0F886
:1024F000103B2B6803F00303012B09B20ED1D2F875
:10250000083802EB411013F4807FD0F8003B14BF71
:1025100043F0805343F00053C0F8003B02EB4112FC
:10252000D2F8003B43F00443C2F8003B30BD00004A
:102530002DE9F041244D6E6D06EB40130446D3F8AF
:10254000087BC3F8087B38070AD5D6F81438190772
:1025500006D505EB84032146DB6828465B6898476F
:10256000FA071FD5D6F81438DB071BD505EB840313
:10257000D968CCB98B69488A5A68B2FBF0F600FB7F
:1025800016228AB91868DA6890420DD2121AC3E985
:102590000024302383F311880B482146FFF78AFF7C
:1025A00084F31188BDE8F081012303FA04F26B89FA
:1025B00023EA02036B81CB68002BF3D0214602484B
:1025C000BDE8F041184700BF682D002000EB8103F3
:1025D00070B5DD68436D6C692668E6604A0156BBDC
:1025E0001A444FF40020C2F810092A6802F00302CE
:1025F000012A0AB20ED1D3F8080803EB421410F4F2
:10260000807FD4F8000914BF40F0805040F00050A3
:10261000C4F8000903EB4212D2F8000940F004406C
:10262000C2F80009D3F83408012202FA01F101438B
:10263000C3F8341870BD19B9402E84BF4020206003
:1026400020682E8A8419013CB4FBF6F440EAC440A9
:1026500040F000501A44C6E72DE9F8433B4D6E6D3B
:1026600006EB40130446D3F80889C3F8088918F02C
:10267000010F4FEA40171AD0D6F81038DB0716D5ED
:1026800005EB8003D9684B691868DA68904230D24C
:10269000121A4FF000091A60C3F80490302383F334
:1026A000118821462846FFF791FF89F3118818F019
:1026B000800F1CD0D6F834380126A640334216D0FD
:1026C00005EB84036D6DD3F80CC0DCF814200134E5
:1026D000E4B2D2F800E005EB04342F4451687145B0
:1026E00015D3D5F8343823EA0606C5F83468BDE8B2
:1026F000F883012303FA04F22B8923EA02032B81D6
:102700008B68002BD3D0214628469847CFE7BCF8EA
:102710001000AEEB0103834228BF0346D7F8180927
:1027200080B2B3EB800FE2D89068A0F1040959F8A9
:10273000048FC4F80080A0EB09089844B8F1040F96
:10274000F5D818440B4490605360C7E7682D00200B
:102750002DE9F74FA24C656D6E69AB691E4016F40A
:1027600080586E6107D02046FEF764FD03B0BDE8D7
:10277000F04F00F047BC002E12DAD5F8003E984822
:102780009B071EBFD5F8003E23F00303C5F8003EAB
:10279000D5F8043823F00103C5F80438FEF774FDBA
:1027A000370505D58E48FFF7BDFC8D48FEF75AFD6D
:1027B000B0040CD5D5F8083813F0060FEB6823F4F5
:1027C00070530CBF43F4105343F4A053EB60310734
:1027D0001BD56368DB681BB9AB6923F00803AB61E9
:1027E0002378052B0CD1D5F8003E7D489A071EBFF3
:1027F000D5F8003E23F00303C5F8003EFEF744FD84
:102800006368DB680BB176489847F30274D4B7026B
:1028100027D5D4F85490DFF8C8B100274FF0010A4B
:1028200009EB4712D2F8003B03F44023B3F5802FA5
:1028300011D1D2F8003B002B0DDA62890AFA07F3B6
:1028400022EA0303638104EB8703DB68DB6813B1CF
:10285000394658469847A36D01379B68FFB29F429F
:10286000DED9F00617D5676D3A6AC2F30A1002F096
:102870000F0302F4F012B2F5802F00F08580B2F55C
:10288000402F08D104EB83030022DB681B6A07F5A5
:10289000805790426AD13003D5F8184813D5E10328
:1028A00002D50020FFF744FEA20302D50120FFF766
:1028B0003FFE630302D50220FFF73AFE270302D54D
:1028C0000320FFF735FE75037FF550AFE00702D513
:1028D0000020FFF7C1FEA10702D50120FFF7BCFED3
:1028E000620702D50220FFF7B7FE23077FF53EAF50
:1028F0000320FFF7B1FE39E7636DDFF8E4A0019331
:1029000000274FF00109A36D9B685FFA87FB9B4589
:102910003FF67DAF019B03EB4B13D3F8001901F495
:102920004021B1F5802F1FD1D3F8001900291BDAFF
:10293000D3F8001941F09041C3F80019D3F80019F9
:102940000029FBDB5946606DFFF718FC218909FA65
:102950000BF321EA0303238104EB8B03DB689B6801
:1029600013B15946504698470137CCE7910708BF45
:10297000D7F80080072A98BF03F8018B02F1010203
:1029800098BF4FEA182884E7023304EB830207F567
:1029900080575268D2F818C0DCF80820DCE9001C27
:1029A000A1EB0C0C002188420AD104EB830463687C
:1029B0009B699A6802449A605A6802445A606AE7BE
:1029C00011F0030F08BFD7F800808C4588BF02F8CC
:1029D000018B01F1010188BF4FEA1828E3E700BF2E
:1029E000682D0020436D03EB4111D1F8003B43F407
:1029F0000013C1F8003B7047436D03EB4111D1F860
:102A0000003943F40013C1F800397047436D03EBFC
:102A10004111D1F8003B23F40013C1F8003B70478B
:102A2000436D03EB4111D1F8003923F40013C1F8D1
:102A30000039704700F1604303F561430901C9B2F1
:102A400083F80013012200F01F039A4043099B0002
:102A500003F1604303F56143C3F880211A607047B6
:102A600030B5039C0172043304FB0325C0E906530F
:102A7000049B03630021059BC160C0E90000C0E91D
:102A80000422C0E90842C0E90A11436330BD0000D6
:102A9000416A0022C0E90411C0E90A22C2606FF055
:102AA0000101FEF7FBBE0000D0E90432934201D1E0
:102AB000C2680AB9181D7047002070470369196081
:102AC000C2680132C260C2691344826903619342E1
:102AD00024BF436A03610021FEF7D4BE38B5044623
:102AE0000D46E3683BB16269131D1268A36213448B
:102AF000E362002007E0237A33B929462046FEF737
:102B0000B1FE0028EDDA38BD6FF00100FBE70000F0
:102B1000C368C269013BC36043691344826943616E
:102B2000934224BF436A436100238362036B03B172
:102B30001847704770B53023044683F31188866ABE
:102B40003EB9FFF7CBFF054618B186F3118828463A
:102B500070BDA36AE26A13F8015BA362934202D3D9
:102B60002046FFF7D5FF002383F31188EFE700002D
:102B70002DE9F84F04460E46174698464FF03009A7
:102B800089F311880025AA46D4F828B0BBF1000FBC
:102B900009D141462046FFF7A1FF20B18BF31188F0
:102BA0002846BDE8F88FD4E90A12A7EB050B521AA4
:102BB000934528BF9346BBF1400F1BD9334601F123
:102BC000400251F8040B43F8040B9142F9D1A36A77
:102BD00040334036A3624035D4E90A239A4202D3F7
:102BE0002046FFF795FF8AF31188BD42D8D289F3BA
:102BF0001188C9E730465A46FEF758F8A36A5B4485
:102C00005E44A3625D44E7E710B5029C01720433A1
:102C100003FB0421C0E906130023C0E90A33039B28
:102C20000363049BC460C0E90000C0E90422C0E95A
:102C30000842436310BD0000026AC260426AC0E9F4
:102C400004220022C0E90A226FF00101FEF726BE2D
:102C5000D0E904239A4201D1C26822B9184650F83B
:102C6000043B0B60704700231846FAE7C368C2694B
:102C70000133C3604369134482694361934224BFB3
:102C8000436A43610021FEF7FDBD000038B50446EC
:102C90000D46E3683BB123691A1DA262E269134441
:102CA000E362002007E0237A33B929462046FEF785
:102CB000D9FD0028EDDA38BD6FF00100FBE7000018
:102CC00003691960C268013AC260C269134482692B
:102CD0000361934224BF436A036100238362036B51
:102CE00003B118477047000070B530230D46044605
:102CF000114683F31188866A2EB9FFF7C7FF10B11A
:102D000086F3118870BDA36A1D70A36AE26A01335D
:102D10009342A36204D3E16920460439FFF7D0FF50
:102D2000002080F31188EDE72DE9F84F04460D46A9
:102D3000904699464FF0300A8AF311880026B34630
:102D4000A76A4FB949462046FFF7A0FF20B187F395
:102D500011883046BDE8F88FD4E90A073A1AA8EB83
:102D60000607974228BF1746402F1BD905F140039D
:102D700055F8042B40F8042B9D42F9D1A36A403347
:102D8000A3624036D4E90A239A4204D3E16920467B
:102D90000439FFF795FF8BF311884645D9D28AF3A2
:102DA0001188CDE729463A46FDF780FFA36A3B44E8
:102DB0003D44A3623E44E5E7D0E904239A4217D19B
:102DC000C3689BB1836A8BB1043B9B1A0ED013601E
:102DD000C368013BC360C3691A44836902619A42B4
:102DE00024BF436A036100238362012318467047AE
:102DF0000023FBE700F030B94FF08043586A70477A
:102E00004FF08043002258631A610222DA60704753
:102E10004FF080430022DA60704700004FF080439B
:102E200058637047FEE7000070B51B4B0163002537
:102E3000044686B0586085620E4600F0BFF804F183
:102E40001003C4E904334FF0FF33C4E90635C4E985
:102E50000044A560E562FFF7CFFF2B460246C4E9B8
:102E6000082304F134010D4A256580232046FEF72E
:102E7000AFFC0123E0600A4A037500927268019278
:102E8000B268CDE90223074B6846CDE90435FEF769
:102E9000C7FC06B070BD00BF002600209C360008AD
:102EA000A1360008252E0008024AD36A1843D062D2
:102EB000704700BF982300204B6843608B68836095
:102EC000CB68C3600B6943614B6903628B694362E2
:102ED0000B6803607047000008B5264B26481A6946
:102EE00040F2FF110A431A611A6922F4FF7222F0BC
:102EF00001021A611A691A6B0A431A631A6D0A43AE
:102F00001A651E4A1B6D1146FFF7D6FF02F11C0120
:102F100000F58060FFF7D0FF02F1380100F5806016
:102F2000FFF7CAFF02F1540100F58060FFF7C4FF0C
:102F300002F1700100F58060FFF7BEFF02F18C0125
:102F400000F58060FFF7B8FF02F1A80100F580608E
:102F5000FFF7B2FF02F1C40100F58060FFF7ACFF9C
:102F600002F1E00100F58060FFF7A6FFBDE8084030
:102F700000F0EEB80038024000000240A836000819
:102F800008B500F059FAFEF701FCFFF793F8BDE829
:102F90000840FEF76FBE000070470000EFF30983A2
:102FA00005494A6B22F001024A63683383F30988BA
:102FB000002383F31188704700EF00E0302080F396
:102FC000118862B60C4B0D4AD96821F4E0610904FE
:102FD000090C0A43DA60D3F8FC20094942F08072F8
:102FE000C3F8FC200A6842F001020A602022DA7766
:102FF00083F82200704700BF00ED00E00003FA05EF
:10300000001000E010B5302383F311880E4B5B688D
:1030100013F4006314D0F1EE103AEFF30984683C26
:103020004FF08073E361094BDB6B236684F30988FF
:10303000FEF78CFB10B1064BA36110BD054BFBE7FF
:1030400083F31188F9E700BF00ED00E000EF00E036
:103050002F030008320300080F4B1A6C42F00102E4
:103060001A641A6E42F001021A660C4A1B6E9368CB
:1030700043F0010393604FF0804353229A624FF074
:10308000FF32DA6200229A615A63DA605A600122E2
:103090005A611A60704700BF00380240002004E007
:1030A0004FF0804208B51169D3680B40D9B2C943CB
:1030B0009B07116107D5302383F31188FEF77CFB52
:1030C000002383F3118808BD1F4B1A696FEAC252AF
:1030D0006FEAD2521A611A69C2F308021A614FF0FC
:1030E000FF301A695A69586100215A6959615A6951
:1030F0001A6A62F080521A621A6A02F080521A62E8
:103100001A6A5A6A58625A6A59625A6A1A6C42F0C2
:1031100080521A641A6E42F080521A661A6E0B4A76
:10312000106840F480701060186F00F44070B0F5C3
:10313000007F1EBF4FF4803018671967536823F46F
:103140000073536000F054B9003802400070004032
:10315000334B4FF080521A64324A4FF440411160B1
:103160001A6842F001021A601A689107FCD59A6841
:1031700022F003029A602A4B9A6812F00C02FBD1EB
:10318000196801F0F90119609A601A6842F48032F6
:103190001A601A689203FCD55A6F42F001025A670E
:1031A0001F4B5A6F9007FCD51F4A5A601A6842F0AD
:1031B00080721A601B4A53685904FCD5184B1A6870
:1031C0009201FCD5194A9A60194B1A68194B9A4218
:1031D000194B21D1194A1168194A91421CD140F268
:1031E00005121A60144A136803F00F03052BFAD175
:1031F0000B4B9A6842F002029A609A6802F00C0245
:10320000082AFAD15A6C42F480425A645A6E42F447
:1032100080425A665B6E704740F20572E1E700BF7C
:10322000003802400070004008544007009488387D
:10323000002004E011640020003C024000ED00E0AA
:1032400041C20F41074A08B5536903F001035361B6
:1032500023B1054A13680BB150689847BDE8084090
:10326000FFF7D0BE003C0140E02D0020074A08B522
:10327000536903F00203536123B1054A93680BB10C
:10328000D0689847BDE80840FFF7BCBE003C01404D
:10329000E02D0020074A08B5536903F00403536189
:1032A00023B1054A13690BB150699847BDE808403E
:1032B000FFF7A8BE003C0140E02D0020074A08B5FA
:1032C000536903F00803536123B1054A93690BB1B5
:1032D000D0699847BDE80840FFF794BE003C014024
:1032E000E02D0020074A08B5536903F0100353612D
:1032F00023B1054A136A0BB1506A9847BDE80840EC
:10330000FFF780BE003C0140E02D0020164B10B5B9
:103310005C6904F478725A61A30604D5134A936A6F
:103320000BB1D06A9847600604D5104A136B0BB1F5
:10333000506B9847210604D50C4A936B0BB1D06BA8
:103340009847E20504D5094A136C0BB1506C9847B5
:10335000A30504D5054A936C0BB1D06C9847BDE822
:103360001040FFF74FBE00BF003C0140E02D0020A1
:10337000194B10B55C6904F47C425A61620504D5AE
:10338000164A136D0BB1506D9847230504D5134AA7
:10339000936D0BB1D06D9847E00404D50F4A136EBE
:1033A0000BB1506E9847A10404D50C4A936E0BB133
:1033B000D06E9847620404D5084A136F0BB1506F62
:1033C0009847230404D5054A936F0BB1D06F9847F3
:1033D000BDE81040FFF716BE003C0140E02D002084
:1033E00008B5FFF75DFEBDE80840FFF70BBE000023
:1033F000062108B50846FFF71DFB06210720FFF749
:1034000019FB06210820FFF715FB06210920FFF70D
:1034100011FB06210A20FFF70DFB06211720FFF7FD
:1034200009FB06212820FFF705FBBDE8084007211E
:103430001C20FFF7FFBA000008B5FFF745FE00F0BB
:103440000BF8FDF78DFEFDF765FDFFF7A5FDBDE867
:103450000840FFF7CFBC00000023054A194601339E
:10346000102BC2E9001102F10802F8D1704700BF29
:10347000E02D0020034611F8012B03F8012B002A50
:10348000F9D1704753544D3332463F3F3F005354B8
:103490004D3332463430780053544D333246343253
:1034A000780053544D3332463434365858000000B7
:1034B000012033000010410001105A000310590090
:1034C00007103100000000008434000813040000DD
:1034D0008E3400081904000098340008210400000C
:1034E000A234000800000000910E00087D0E0008C4
:1034F000B90E0008A50E0008B10E00089D0E0008C8
:10350000890E0008750E0008C50E000800000000B6
:1035100001000000000000006330000018350008C2
:10352000F0230020002600204172647550696C6F02
:10353000740025424F415244252D424C00255345ED
:103540005249414C2500000002000000000000002C
:10355000AD1000081911000840004000A02A00200A
:10356000B02A00200200000000000000030000005C
:10357000000000005D1100080000000010000000C5
:10358000C02A002000000000010000000000000030
:10359000682D002001010200111C0008211B0008F9
:1035A000BD1B0008A11B000843000000B035000847
:1035B00009024300020100C03209040000010202B6
:1035C0000100052400100105240100010424020269
:1035D0000524060001070582030800FF0904010015
:1035E000020A0000000705010240000007058102F1
:1035F0004000000012000000FC350008120110011C
:1036000002000040091241570002010203010000BC
:103610000403090425424F41524425004D6174655D
:103620006B463430352D57696E6700303132333494
:1036300035363738394142434445460000400000A2
:1036400000400000004000000040000000000100B9
:103650000000020000000200000002000000020062
:103660000000020000000200000002000000000054
:10367000A112000859150008051600084000400076
:10368000C82D0020C82D002001000000D82D0020EA
:103690008000000040010000030000006D61696EC1
:1036A0000069646C650000000A01A81600000000B3
:1036B000AAAAAAAA05011400FF9F00008800000022
:1036C00070A70A000000000100000000AAAAAAAA30
:1036D00000000001FFFF00000000000000000000EB
:1036E00000A0A01200000000AAAAAAAA005050112F
:1036F000FFFF0000000000880077080020000000A5
:1037000000000000AAAAAAAA10000000FFFF000003
:1037100000080000000000000000000000000000A1
:10372000AAAAAAAA00000000FFFF000000000000F3
:10373000000000000000000000000000AAAAAAAAE1
:1037400000000000FFFF000000000000000000007B
:103750000000000000000000AAAAAAAA00000000C1
:10376000FFFF00000000000000000000000000005B
:10377000000000000A00000000000000030000003C
:103780000000000000000000000000000000000039
:103790000000000000000000000000000000000029
:1037A00000000000000000007F000000000000009A
:1037B00000000F0000000000FF009600000000085D
:1037C0000096000000000800040000001036000809
:1037D00000000000000000000000000000000000E9
:1037E0000000000000000000FFFFFFFFFFFFFFFFE1
:1037F000FFFFFFFFFFFFFFFFFFFFFFFFFFFFFFFFD9
:10380000FFFFFFFFFFFFFFFFFFFFFFFFFFFFFFFFC8
:10381000FFFFFFFFFFFFFFFFFFFFFFFFFFFFFFFFB8
:10382000FFFFFFFFFFFFFFFFFFFFFFFFFFFFFFFFA8
:020000040801F1
:100000000006002099120108F17B09084D7B0908C0
:10001000B97B09084D7B0908857B09089B120108FB
:100020009B1201089B1201089B120108EDF50B08B9
:100030009B1201089B1201089B1201089B120108E8
:100040009B1201089B1201089B1201089B120108D8
:100050009B1201089B12010885010C08AD010C08D8
:10006000D5010C08FD010C0825020C086DA40B0835
:1000700095A40B08C1A40B08EDA40B0819A50B0847
:1000800041A50B086DA50B08F1A30B089B120108F5
:100090009B1201089B1201089B1201084D020C08DB
:1000A00099030C08AD030C08C1030C08C5030C0828
:1000B000C9030C08DD030C08F1030C08C5AD0B08DF
:1000C000D9AD0B08FDAD0B0811AE0B089B12010852
:1000D0009B12010821030C0835030C0849030C0886
:1000E000B1020C089B1201089B12010815040C08B0
:1000F00019040C082D040C0831040C0899A50B08F0
:100100009B1201089B12010805040C089B120108B0
:100110005D030C0871030C089B1201089B12010877
:10012000C5A50B08EDA50B0819A60B0845A60B08DD
:1001300071A60B089B1201089B1201089B12010873
:100140009B1201089B1201089B12010819FD0B0864
:1001500099A60B08C5A60B08F1A60B0885030C0889
:100160009B1201089B1201089B1201089B120108B7
:100170009B1201089B1201089B1201089B120108A7
:100180009B1201089B1201089B1201089B12010897
:100190009B1201089B1201089B1201089B12010887
:1001A0009B1201089B1201089B1201089B12010877
:1001B0009B1201089B1201089B1201089B12010867
:1001C0009B1201089B1201089B1201089B12010857
:1001D0009B1201089B1201089B1201089B12010847
:1001E0004D580108957E02085DF70308C9B9050856
:1001F000EDBF050829330608E9970608AD9F0608F4
:10020000E5A2060861080708912E0708D1EE070845
:10021000554A0808AD5708088D6D0908717209081C
:10022000CD850A0861E10A08C5070B0831130B08E0
:10023000BD420B08E9480B08000000000000000068
:1002400081F0004102E000BF83F0004330B54FEA87
:1002500041044FEA430594EA050F08BF90EA020FF4
:100260001FBF54EA000C55EA020C7FEA645C7FEA87
:10027000655C00F0E2804FEA5454D4EB5555B8BFAA
:100280006D420CDD2C4480EA020281EA030382EA1B
:10029000000083EA010180EA020281EA0303362DAD
:1002A00088BF30BD11F0004F4FEA01314FF4801C80
:1002B0004CEA113102D0404261EB410113F0004F92
:1002C0004FEA03334CEA133302D0524263EB430349
:1002D00094EA050F00F0A780A4F10104D5F1200EE7
:1002E0000DDB02FA0EFC22FA05F2801841F1000142
:1002F00003FA0EF2801843FA05F359410EE0A5F116
:1003000020050EF1200E012A03FA0EFC28BF4CF046
:10031000020C43FA05F3C01851EBE37101F00045FC
:1003200007D54FF0000EDCF1000C7EEB00006EEB09
:100330000101B1F5801F1BD3B1F5001F0CD3490893
:100340005FEA30004FEA3C0C04F101044FEA4452EA
:1003500012F5800F80F09A80BCF1004F08BF5FEA71
:10036000500C50F1000041EB045141EA050130BD51
:100370005FEA4C0C404141EB0101013C28BFB1F563
:10038000801FE9D291F0000F04BF01460020B1FAAE
:1003900081F308BF2033A3F10B03B3F120020CDA81
:1003A0000C3208DD02F1140CC2F10C0201FA0CF05F
:1003B00021FA02F10CE002F11402D8BFC2F1200CC4
:1003C00001FA02F120FA0CFCDCBF41EA0C0190407A
:1003D000E41AA2BF01EB0451294330BD6FEA0404C3
:1003E0001F3C1CDA0C340EDC04F11404C4F12002AE
:1003F00020FA04F001FA02F340EA030021FA04F3C0
:1004000045EA030130BDC4F10C04C4F1200220FA16
:1004100002F001FA04F340EA0300294630BD21FA54
:1004200004F0294630BD94F0000F83F4801306BF1A
:1004300081F480110134013D4EE77FEA645C18BF0E
:100440007FEA655C29D094EA050F08BF90EA020FA5
:1004500005D054EA000C04BF1946104630BD91EA9D
:10046000030F1EBF0021002030BD5FEA545C05D1A0
:100470004000494128BF41F0004130BD14F58004DF
:100480003CBF01F5801130BD01F0004545F0FE4153
:1004900041F470014FF0000030BD7FEA645C1ABF88
:1004A000194610467FEA655C1CBF0B46024650EABF
:1004B000013406BF52EA033591EA030F41F40021EB
:1004C00030BD00BF90F0000F04BF0021704730B571
:1004D0004FF4806404F132044FF000054FF0000146
:1004E00050E700BF90F0000F04BF0021704730B507
:1004F0004FF4806404F1320410F0004548BF4042DC
:100500004FF000013EE700BF42004FEAE2014FEA30
:1005100031014FEA02701FBF12F07F4393F07F4F0B
:1005200081F06051704732F07F4208BF704793F00E
:100530007F4F04BF41F40021704730B54FF4607421
:1005400001F0004521F000411CE700BF50EA010224
:1005500008BF704730B54FF000050AE050EA0102CD
:1005600008BF704730B511F0004502D5404261EB3D
:1005700041014FF4806404F132045FEA915C3FF47E
:10058000D8AE4FF003025FEADC0C18BF03325FEA1B
:10059000DC0C18BF033202EBDC02C2F1200300FACC
:1005A00003FC20FA02F001FA03FE40EA0E0021FAF1
:1005B00002F11444BDE600BF70B54FF0FF0C4CF4DF
:1005C000E06C1CEA11541DBF1CEA135594EA0C0F91
:1005D00095EA0C0F00F0DEF82C4481EA030621EACC
:1005E0004C5123EA4C5350EA013518BF52EA033507
:1005F00041F4801143F4801338D0A0FB02CE4FF0B9
:100600000005E1FB02E506F00042E0FB03E54FF0E8
:100610000006E1FB03569CF0000F18BF4EF0010EE0
:10062000A4F1FF04B6F5007F64F5407404D25FEADC
:100630004E0E6D4146EB060642EAC62141EA55518F
:100640004FEAC52040EA5E504FEACE2EB4F1FD0CD1
:1006500088BFBCF5E06F1ED8BEF1004F08BF5FEA4F
:10066000500E50F1000041EB045170BD06F0004601
:1006700046EA010140EA020081EA0301B4EB5C04AE
:10068000C2BFD4EB0C0541EA045170BD41F48011A6
:100690004FF0000E013C00F3AB8014F1360FDEBFCB
:1006A000002001F0004170BDC4F10004203C35DAA7
:1006B0000C341BDC04F11404C4F1200500FA05F32A
:1006C00020FA04F001FA05F240EA020001F00042CB
:1006D00021F0004110EBD37021FA04F642EB060141
:1006E0005EEA430E08BF20EAD37070BDC4F10C046B
:1006F000C4F1200500FA04F320FA05F001FA04F22F
:1007000040EA020001F0004110EBD37041F100011A
:100710005EEA430E08BF20EAD37070BDC4F1200525
:1007200000FA05F24EEA020E20FA04F301FA05F28D
:1007300043EA020321FA04F001F0004121FA04F235
:1007400020EA020000EBD3705EEA430E08BF20EA05
:10075000D37070BD94F0000F0FD101F0004640003F
:1007600041EB010111F4801F08BF013CF7D041EAC1
:10077000060195F0000F18BF704703F000465200C5
:1007800043EB030313F4801F08BF013DF7D043EA96
:100790000603704794EA0C0F0CEA135518BF95EA4C
:1007A0000C0F0CD050EA410618BF52EA4306D1D1D3
:1007B00081EA030101F000414FF0000070BD50EAF2
:1007C000410606BF1046194652EA430619D094EA7C
:1007D0000C0F02D150EA013613D195EA0C0F05D166
:1007E00052EA03361CBF104619460AD181EA0301BA
:1007F00001F0004141F0FE4141F470014FF0000072
:1008000070BD41F0FE4141F4780170BD70B54FF00C
:10081000FF0C4CF4E06C1CEA11541DBF1CEA13558C
:1008200094EA0C0F95EA0C0F00F0A7F8A4EB05046E
:1008300081EA030E52EA03354FEA013100F0888065
:100840004FEA03334FF0805545EA131343EA12632E
:100850004FEA022245EA111545EA10654FEA0026E3
:100860000EF000419D4208BF964244F1FD0404F59C
:10087000407402D25B084FEA3202B61A65EB0305F8
:100880005B084FEA32024FF480104FF4002CB6EBB5
:10089000020E75EB030E22BFB61A754640EA0C0035
:1008A0005B084FEA3202B6EB020E75EB030E22BF75
:1008B000B61A754640EA5C005B084FEA3202B6EBB6
:1008C000020E75EB030E22BFB61A754640EA9C0075
:1008D0005B084FEA3202B6EB020E75EB030E22BF45
:1008E000B61A754640EADC0055EA060E18D04FEA03
:1008F000051545EA16754FEA06164FEAC30343EAA3
:1009000052734FEAC2025FEA1C1CC0D111F4801F6F
:100910000BD141EA00014FF000004FF0004CB6E768
:1009200011F4801F04BF01430020B4F1FD0C88BF07
:10093000BCF5E06F3FF6AFAEB5EB030C04BFB6EB12
:10094000020C5FEA500C50F1000041EB045170BD05
:100950000EF0004E4EEA113114EB5C04C2BFD4EB32
:100960000C0541EA045170BD41F480114FF0000EB6
:10097000013C90E645EA060E8DE60CEA135594EA32
:100980000C0F08BF95EA0C0F3FF43BAF94EA0C0F35
:100990000AD150EA01347FF434AF95EA0C0F7FF4AA
:1009A00025AF104619462CE795EA0C0F06D152EAFE
:1009B00003353FF4FDAE1046194622E750EA4106E2
:1009C00018BF52EA43067FF4C5AE50EA41047FF4F3
:1009D0000DAF52EA43057FF4EBAE12E74FF0FF3C58
:1009E00006E000BF4FF0010C02E000BF4FF0010C29
:1009F0004DF804CD4FEA410C7FEA6C5C4FEA430CA2
:100A000018BF7FEA6C5C1BD001B050EA410C0CBFF0
:100A100052EA430C91EA030F02BF90EA020F002052
:100A2000704710F1000F91EA030F58BF994208BFB9
:100A300090422CBFD8176FEAE37040F00100704776
:100A40004FEA410C7FEA6C5C02D150EA013C07D1CD
:100A50004FEA430C7FEA6C5CD6D152EA033CD3D018
:100A60005DF8040B704700BF8446104662468C4612
:100A70001946634600E000BF01B5FFF7B7FF002845
:100A800048BF10F1000F01BD4DF808EDFFF7F4FF6E
:100A90000CBF012000205DF808FB00BF4DF808EDF9
:100AA000FFF7EAFF34BF012000205DF808FB00BF1C
:100AB0004DF808EDFFF7E0FF94BF012000205DF83E
:100AC00008FB00BF4DF808EDFFF7CEFF94BF0120F3
:100AD00000205DF808FB00BF4DF808EDFFF7C4FFEC
:100AE00034BF012000205DF808FB00BF4FEA410C35
:100AF0007FEA6C5C02D150EA013C0AD14FEA430C18
:100B00007FEA6C5C02D152EA033C02D14FF0000054
:100B100070474FF0010070474FEA410212F5001292
:100B200015D211D56FF47873B3EB625212D94FEA34
:100B3000C12343F0004343EA505311F0004F23FA1E
:100B400002F018BF404270474FF00000704750EA73
:100B5000013005D111F0004008BF6FF00040704730
:100B60004FF00000704700BF4A0011D212F500128A
:100B700011D20DD56FF47873B3EB62520ED44FEAF5
:100B8000C12343F0004343EA505323FA02F0704775
:100B90004FF00000704750EA013002D14FF0FF30B3
:100BA00070474FF0000070474FEA4102B2F1E04356
:100BB00024BFB3F5001CDCF1FE5C0DD901F0004C44
:100BC0004FEAC0024CEA5070B2F1004F40EB830094
:100BD00008BF20F00100704711F0804F21D113F1C0
:100BE0003872BCBF01F00040704741F480114FEAF9
:100BF0005252C2F11802C2F1200C10FA0CF320FA82
:100C000002F018BF40F001004FEAC1234FEAD3239E
:100C100003FA0CFC40EA0C0023FA02F34FEA430308
:100C2000CCE77FEA625307D150EA01331EBF4FF091
:100C3000FE4040F44000704701F0004040F0FE40AC
:100C400040F40000704700BF80F0004002E000BFA9
:100C500081F0004142001FBF5FEA410392EA030FA7
:100C60007FEA226C7FEA236C6AD04FEA1262D2EBF1
:100C70001363C1BFD218414048404140B8BF5B42F6
:100C8000192B88BF704710F0004F40F4000020F08F
:100C90007F4018BF404211F0004F41F4000121F0A5
:100CA0007F4118BF494292EA030F3FD0A2F10102EF
:100CB00041FA03FC10EB0C00C3F1200301FA03F12D
:100CC00000F0004302D5494260EB4000B0F5000F50
:100CD00013D3B0F1807F06D340084FEA310102F10F
:100CE0000102FE2A51D2B1F1004F40EBC25008BFC1
:100CF00020F0010040EA03007047490040EB00008B
:100D0000013A28BFB0F5000FEDD2B0FA80FCACF18B
:100D1000080CB2EB0C0200FA0CF0AABF00EBC250B8
:100D200052421843BCBFD0401843704792F0000FA6
:100D300081F4000106BF80F400000132013BB5E7F9
:100D40004FEA41037FEA226C18BF7FEA236C21D06F
:100D500092EA030F04D092F0000F08BF08467047D4
:100D600090EA010F1CBF0020704712F07F4F04D1A2
:100D7000400028BF40F00040704712F100723CBFB5
:100D800000F50000704700F0004343F0FE4040F4DF
:100D9000000070477FEA226216BF08467FEA23639D
:100DA0000146420206BF5FEA412390EA010F40F488
:100DB000800070474FF0000304E000BF10F00043D4
:100DC00048BF40425FEA000C08BF704743F09643BB
:100DD00001464FF000001CE050EA010208BF7047D6
:100DE0004FF000030AE000BF50EA010208BF70475D
:100DF00011F0004302D5404261EB41015FEA010C72
:100E000002BF84460146002043F0B64308BFA3F169
:100E10008053A3F50003BCFA8CF2083AA3EBC2534B
:100E200010DB01FA02FC634400FA02FCC2F120026A
:100E3000BCF1004F20FA02F243EB020008BF20F0A1
:100E40000100704702F1200201FA02FCC2F1200207
:100E500050EA4C0021FA02F243EB020008BF20EAFC
:100E6000DC7070477BB972B90029BEBF00204FF01B
:100E7000004106E008BF00281CBF6FF000414FF0A2
:100E8000FF3000F007BAADF1080C6DE904CE00297F
:100E900009DB002B1ADB00F095F8DDF804E0DDE952
:100EA000022304B07047404261EB4101002B1BDB81
:100EB00000F088F8DDF804E0DDE9022304B04042E8
:100EC00061EB4101524263EB43037047524263EBD3
:100ED000430300F077F8DDF804E0DDE9022304B015
:100EE000404261EB41017047524263EB430300F023
:100EF00069F8DDF804E0DDE9022304B0524263EB57
:100F00004303704753B94AB9002908BF00281CBFE2
:100F10004FF0FF314FF0FF3000F0BCB9ADF1080CDD
:100F20006DE904CE00F04EF8DDF804E0DDE90223BF
:100F300004B07047430803F05533C01A830803F028
:100F4000333300F03330184400EB101000F00F3052
:100F500000EB002000EB0040000E704707EE900A07
:100F6000F5EEC07AF1EE10FA01D400F00BB8F1EE14
:100F7000677A08B517EE900A00F004F8404261EB7A
:100F8000410108BDD0B5FFF7BFFA0C4B0022064661
:100F90000F46FFF711FBFFF7E7FD0446FFF792FA54
:100FA000074B0022FFF708FB02460B463046394646
:100FB000FFF74AF9FFF7D8FD2146D0BD0000F03D0C
:100FC0000000F0412DE9F047089D04468E46002BB5
:100FD0004DD18A42944669D9B2FA82F252B101FAED
:100FE00002F3C2F1200120FA01F10CFA02FC41EAFD
:100FF000030E94404FEA1C48210CBEFBF8F61FFA82
:101000008CF708FB16E341EA034306FB07F199421C
:101010000AD91CEB030306F1FF3080F01F819942CF
:1010200040F21C81023E63445B1AA4B2B3FBF8F0A9
:1010300008FB103344EA034400FB07F7A7420AD930
:101040001CEB040400F1FF3380F00A81A74240F258
:1010500007816444023840EA0640E41B00261DB1C3
:10106000D4400023C5E900433146BDE8F0878B42F8
:1010700009D9002D00F0EF800026C5E900013046B7
:101080003146BDE8F087B3FA83F6002E4AD18B4291
:1010900002D3824200F2F980841A61EB030301203B
:1010A0009E46002DE0D0C5E9004EDDE702B9FFDE27
:1010B000B2FA82F2002A40F09280A1EB0C014FEAD2
:1010C0001C471FFA8CFE0126200CB1FBF7F307FB2F
:1010D000131140EA01410EFB03F0884208D91CEBD2
:1010E000010103F1FF3802D2884200F2CB8043466F
:1010F000091AA4B2B1FBF7F007FB101144EA01444E
:101100000EFB00FEA64508D91CEB040400F1FF31DC
:1011100002D2A64500F2BB800846A4EB0E0440EACA
:1011200003409CE7C6F12007B34022FA07FC4CEAD3
:10113000030C20FA07F401FA06F31C43F9404FEAC6
:101140001C4900FA06F3B1FBF9F8200C1FFA8CFEDB
:1011500009FB181140EA014108FB0EF0884202FA2F
:1011600006F20BD91CEB010108F1FF3A80F08880F0
:10117000884240F28580A8F102086144091AA4B2AD
:10118000B1FBF9F009FB101144EA014100FB0EFE2E
:101190008E4508D91CEB010100F1FF346CD28E455D
:1011A0006AD90238614440EA0840A0FB0294A1EBEE
:1011B0000E01A142C846A64656D353D05DB1B3EB4B
:1011C000080261EB0E0101FA07F722FA06F3F1407B
:1011D0001F43C5E9007100263146BDE8F087C2F122
:1011E0002003D8400CFA02FC21FA03F3914001439A
:1011F0004FEA1C471FFA8CFEB3FBF7F007FB1036D3
:101200000B0C43EA064300FB0EF69E4204FA02F47E
:1012100008D91CEB030300F1FF382FD29E422DD9D1
:10122000023863449B1B89B2B3FBF7F607FB163306
:1012300041EA034106FB0EF38B4208D91CEB010186
:1012400006F1FF3816D28B4214D9023E6144C91A06
:1012500046EA004638E72E46284605E70646E3E616
:101260001846F8E64B45A9D2B9EB020864EB0C0E20
:101270000138A3E74646EAE7204694E74046D1E72F
:10128000D0467BE7023B614432E7304609E76444DD
:10129000023842E7704700BF02E000F000F8FEE7C6
:1012A00072B6374880F30888364880F30988364894
:1012B0003649086040F20000CCF200004EF634716E
:1012C000CEF200010860BFF34F8FBFF36F8F40F283
:1012D0000000C0F2F0004EF68851CEF20001086026
:1012E000BFF34F8FBFF36F8F4FF00000E1EE100A96
:1012F0004EF63C71CEF200010860062080F314889F
:10130000BFF36F8FAEF0D0F9ADF038FA4FF0553033
:101310001F491B4A91423CBF41F8040BFAE71D49A3
:10132000184A91423CBF41F8040BFAE71A491B4A9C
:101330001B4B9A423EBF51F8040B42F8040BF8E7EE
:1013400000201849184A91423CBF41F8040BFAE7C3
:10135000AEF0AEF9ADF066FA144C154DAC4203DABE
:1013600054F8041B8847F9E701F002F9114C124DBB
:10137000AC4203DA54F8041B8847F9E7AEF096B99B
:1013800000060020002200200000010808ED00E017
:101390000000002000060020C8960E080022002051
:1013A000002C0020002C0020B85D0120E001010885
:1013B0003802010838020108380201082DE9F04F0F
:1013C0002DED108AC1F80CD0C3689D46BDEC108A83
:1013D000BDE8F08F002383F311882846A047002042
:1013E000ACF052FFFEE7ACF0AFFD00DFFEE700001F
:1013F00001F0FF01102A2BDB10F0070F08D010F8C6
:10140000013B013A8B422DD010F0070F42B3F6D1C9
:10141000F0B441EA012141EA014122F007047FF0E2
:1014200000070023F0E80256083C85EA010586EA39
:10143000010685FA47F5A3FA87F586FA47F6A5FA75
:1014400087F68EB9EED1F0BC01F0FF0102F0070281
:1014500032B110F8013B013A83EA010313B1F8D12C
:101460000020704701387047002D06BF354603380D
:10147000073815F0010F07D1013015F4807F02BF46
:10148000013015F4C03F0130F0BC0138704700BF97
:1014900010F8012B11F8013B012A28BF9A42F7D01E
:1014A000D01A7047034613F8012B002AFBD1181AF3
:1014B0000138704738B50022002304460D46FFF777
:1014C000EDFA28B920462946BDE8384000F00AB8B0
:1014D000204605F1004100F005F8404261EB410172
:1014E00038BD00BFD0B50C4B002206460F46FFF7B3
:1014F00063F8FFF739FB0446FEF7E4FF074B0022D1
:10150000FFF75AF802460B4630463946FEF79CFE76
:10151000FFF72AFB2146D0BD0000F03D0000F0415E
:10152000036800221B68184710B503685B6804460F
:10153000984708B194F84D0010BD000038B5044636
:101540007CF002FD0E4B1D680146E86A02681268D5
:10155000904753F08FFEEB6A93F89C1052F076FEA2
:1015600094F837305BB186F079FBEB6AD3F8A030A2
:10157000C01AB0F5FA6F24BF002384F8373038BDA5
:101580000C2C002070B50E4605465FF089FB5FF01D
:101590004BFB10B90124204670BD0A4B93F9D2349D
:1015A000012BF7D15FF07CFB437A002BF2D15FF087
:1015B00077FB847A002CEDD1034A314628467CF033
:1015C000EFFEE8E7104C00202C7A0C08034BD3F810
:1015D0003C350BB97CF06EBC01207047104C0020EC
:1015E0002DE9F0432DED028BC47F91B006460F46E6
:1015F0008CB990F90430002B00F00681834B1D68F4
:10160000A86A03685B6B9847044650B9804A39461C
:1016100030467CF0C5FE204611B0BDEC028BBDE823
:10162000F083B3684BB933685B6B3946304611B011
:10163000BDEC028BBDE8F0431847E86AFFF774FF82
:1016400004460028E7D1394630467DF069FDDFF8D1
:10165000F4810546394630467CF0CAFE08F2E44281
:1016600008F59C6392ED007AD3ED007AB4EEE77A48
:101670002840F1EE10FAC5B209D598F9DC34032BF5
:1016800005D0644A394630467CF08AFE254608F289
:101690008443D3ED007AB0EE088AF4EEC87AF1EE16
:1016A00010FA0BD517EE900AFEF72EFF5A4ACDE935
:1016B0000001394630467CF073FE002508F5916341
:1016C000D3ED007AF4EEC87AF1EE10FA0BD517EEEE
:1016D000900AFEF719FF514ACDE90001394630461C
:1016E0007CF05EFE002508F28C43D3ED007AB8EE64
:1016F000087AF4EEC77AF1EE10FA0BDD17EE900AD5
:10170000FEF702FF464ACDE90001394630467CF03B
:1017100047FE0025B8F97034042B07DC052200923F
:101720003946404A30467CF03BFE0025D8F8280F69
:101730005FF012FB80B198F9D2346BB1D8F8283F32
:10174000B8F9D424B3F90E309A4205DA364A39464C
:1017500030467CF025FE0025DFF8EC903946304617
:10176000FFF710FF99F86D30002B46D100EA050411
:101770002E484FF4806100F0DFFE78B1D8F8283FA2
:10178000B3F90C30A3F2E24292B2B2F5FA7F05D976
:10179000274A394630467CF003FE002499F8083782
:1017A00053B124482DF05AF8054628B9224A394643
:1017B00030467CF0F5FD2C4600212E2204A80DF1C8
:1017C0000C080391B1F0CAFED9F858004246322104
:1017D00008F092F9054600287FF41DAFD9F85800AB
:1017E00003689B689847154ACDF800800346394640
:1017F00030467CF0D5FD2C460DE7114A394630467F
:101800007CF0CEFD0024B3E7012404E70C2C00207B
:101810003C7A0C08537A0C08767A0C08967A0C08F5
:10182000B87A0C08DA7A0C08F97A0C08102C002027
:10183000347B0C08108300205C7B0C08942D0D0871
:101840001F7B0C08104C0020107C002070B5054652
:101850000E46FFF797FE3146044628467DF00CFB06
:101860002040C0B270BD0000F0B591B005460E46F4
:101870007CF074FE0446D8B1102128467CF080FB31
:10188000B0B100212E2204A803AF0391B1F066FE8F
:1018900010F014FD32233A4601210FF0FBFF0446FD
:1018A00030B9054B00973246102128467CF070FB7A
:1018B000204611B0F0BD00BF707B0C0870B5054626
:1018C0000E46B1B990F910408CB116480BF0A8FA49
:1018D000DFED157AB0EEC00AB4EEE70AF1EE10FAC9
:1018E00007D4124A012128467CF05AFD344620468E
:1018F00070BDAB689BB10E4B1B68D86AFFF714FE36
:10190000044630B15DF0D8FC0A4A042156F0FCFDD3
:10191000EDE731462846BDE870407DF0EBB8012484
:10192000E5E700BF102C0020000000347C7B0C0891
:101930000C2C00208E7B0C0838B504467DF0AAFCE8
:101940000546A8B10B4805F081FB38B10A490B48A0
:1019500010F0E0F810B1074800F0C2FD2046FFF794
:10196000EDFD0123064984F8373020467DF0A8FBC1
:10197000284638BD102C0020EC8D0020504000205F
:10198000B07B0C08F8B505460E461746C2B12329B0
:1019900001D0012914D81C4807F018FC044668B18E
:1019A00000242046F8BD95F91030022B08D05DF0D8
:1019B00083FC164A062156F0A7FDF2E7002EF2D06E
:1019C0003A46314628467DF01BFD04460028E7D004
:1019D0000F4EB26DA6F1DC039A4203D006F5E0602B
:1019E0002DF072FBB06D03689B6B984786F8D406A8
:1019F0002846FFF7A3FD4FF0FF330649C6F88830AD
:101A000028467DF05DFBCCE7102C0020C07B0C0845
:101A1000107C0020D87B0C08F8B505460E467CF0FB
:101A20005BFB0446104890F9A774D7B9BD2100F5B7
:101A30005C502DF0DFFA38B10C4B32464FF4804148
:101A400028467CF0A5FA3C460948BC212DF0D2FA84
:101A500038B1084B32464FF4804128467CF098FA62
:101A600000242046F8BD00BF104C0020EC7B0C0881
:101A700010830020187C0C0800207047014800F0FB
:101A8000DDBC00BF102C002003685B681847000015
:101A90000DF06EBB65F0EAB95FF050B825F0CEBA34
:101AA00052F056BD07F0C2BC50F010BE0AF0BABCEE
:101AB0000CF0D0BB02F014BE4FF0A4B914F0C8BCB7
:101AC00062F0CABA61F048BF0CF026BC46F0E6BD31
:101AD0000BF024BA14F01AB866F07CBF5EF050BD6B
:101AE0005CF058BE06F0E2BE04F064BA09F0EABF4A
:101AF0000AF006BC0CF0F8B90CF0C4BC0BF04CB802
:101B00000CF016BB01F020B900F2845016F060BE54
:101B100007F000BA90F8F432B02202FB030390F809
:101B2000382393F8D13012B1012B28BF0123184676
:101B300070470000034808602E21117008221A60C7
:101B4000704700BF7C7F0C0870B5044600F5C540A7
:101B50006C3004F5A255FFF7F1FC0021284610F087
:101B600033FB802120460CF0F3FE18B127F0EAF891
:101B700024F07EFE04F5005303F28C4292ED007ACD
:101B8000DFED216A03F28442D2ED007A67EEA67A95
:101B9000D5ED936AFDEEE77A03F63C73F8EEE77A4B
:101BA00004F5BB5167EEA67A1831FDEEE77A05F52C
:101BB000457017EE902A43F8042CD5ED927AF0EE9A
:101BC000E77A67EE877A04F5AC46C3ED007A2AF02F
:101BD00039F994ED467AD6ED147AE7EE007AC6ED3F
:101BE000147AB0EE670A27F01BFE4FF4001186ED61
:101BF000140A20460CF0ACFE20B12846BDE8704027
:101C00000EF0E6BD70BD00BF0000C842FFF79CBFEC
:101C100038B500F5A0450446A86D03689B6B98474E
:101C200095F88F363BB930B104F53F501030BDE820
:101C3000384081F09BBD38BDFFF7EABF38B54FF49F
:101C4000801104460CF084FE054620B9012120468F
:101C50000CF07EFE0546022120460CF079FE40B1D4
:101C600015B9204602F0E0FC04F5A2500EF0AEFCDF
:101C700001E0002DF8D14FF4805120460CF068FEB1
:101C800030B104F5C4406830BDE8384062F00ABBAA
:101C900038BD0000FFF7D2BF38B54FF480110446BD
:101CA0000CF056FE0121054620460CF051FE18B1FD
:101CB00015B9204602F0B8FC102120460CF048FE71
:101CC00060B1204602F024FD4FF4800120460CF064
:101CD0003FFE18B927F036F824F0C6FE2021204632
:101CE0000CF036FE28B1204602F086FD204602F0B8
:101CF0009FFE4FF4005120460CF02AFE10B1204602
:101D000002F07EFE802120460CF022FE28B127F052
:101D100019F8BDE8384024F0CFBD38BDFFF7BCBF8F
:101D200000F5A04300F5C240D96F40307EF060BF9F
:101D3000FFF7F6BF10B5044616F03AFE90F92130D1
:101D40008BB190F8403373B194F9A8355BB1064B71
:101D50001B68DB6A93F89C302BB904F28450BDE811
:101D6000104016F04DBB10BD0C2C0020FFF7E2BF59
:101D70002DE9F843434B1B68DB6A93F89C3004461B
:101D8000002B7CD000F5805898F84937002B76D08E
:101D900007F01CFA002872D004F5005504F5055729
:101DA00095F88E1238460DF0B5FF002867D004F57F
:101DB00090763046FFF7AEFE022860D994F81424DE
:101DC0004FF0B00909FB024292ED837AF1EE007AFE
:101DD000B4EEE77AF1EE10FA51D495F88E12384647
:101DE0000EF048FAB5F9703407EE903AB8EEE77A9B
:101DF000B4EEC07AF1EE10FA0CDD94F8143409FB5D
:101E00000343F8EE677A93ED837AF4EEC77AF1EE46
:101E100010FA34DCD8F83836D5F8382F002BB8BF94
:101E20005B4293422BDC08F23C63D3ED007A9FEDDA
:101E3000166A05F59163D3ED006AF8EEE77A66EE6F
:101E4000866AF4EEE67AF1EE10FA18DC05F63C73D9
:101E500093ED007A27EE067AF4EEC77AF1EE10FAE7
:101E60000DD494F81414B5F97224B02303FB016166
:101E7000384601F58271BDE8F8430DF061BDBDE85B
:101E8000F88300BF0C2C00200000C842FFF770BF91
:101E90002DE9F04190F814342D4D00EB03132F6819
:101EA000D3F8C48100F5907604463046FFF732FE41
:101EB000474514D0022814D904F5A047C5F800807E
:101EC00097F88030012B15D817D104F5C045D5F807
:101ED000E431E3B9D5F8E831CBB905230BE00228AA
:101EE00010D804F5A04393F880205AB1052283F856
:101EF000802007E0013B87F8803004F5C3501C3098
:101F000011F05CFB2046BDE8F04109F09BBF114B8E
:101F10001B68D86A03685B68984780460028ECD144
:101F200094F81414B02303FB0161DC31204605F062
:101F3000FDF8D5F8C8310FCB05F5E67605F5F67551
:101F400086E80F0085E80F0087F88080D5E700BF9E
:101F5000002C00200C2C0020FFF79ABF10B500F5D4
:101F6000A04300F5805493F88F261AB1002384F81B
:101F700049370AE0D3F8DC36042B07D100F5C1401D
:101F8000343081F091FE84F8490710BD0123EEE75B
:101F900010B500F5A04400F59E43A26D24339A428B
:101FA00008D000F59E4368339A421CBF4FF0FF33C0
:101FB000C4F8483604F5C763064A1A6004F23C6365
:101FC000054A1A60FFF7CAFFA06D0368BDE810401C
:101FD0001B6918470000C8420000C8C2FFF7D8BFFD
:101FE000F7B500F5A0460446D6F8DC368B420D4620
:101FF0003FD00B1F00F5C147594207F13407594143
:102000003846019181F040FD0199384681F03CFD50
:10201000042D02D118486DF01DFBD6F8DC36012BDB
:1020200018D1032D16D104F5C5406C307BF096FF16
:1020300040B1204607F0CAF820B104F53B500C30FF
:102040006DF002FB2046C6F8DC5603B0BDE8F04058
:1020500002F03CBC072DF5D104F55B50D6F85826AC
:102060006423052192FBF3F32030044A56F04CFA26
:10207000E8E703B0F0BD00BFDC5A0020BC7C0C08D0
:1020800038B500F5A0450446A86D03689B6B9847DA
:10209000002840D095F8D436002B3CD1AA6D04F529
:1020A0009E4324339A4238D195F888362BB90121C2
:1020B0002046BDE83840FFF793BFB5F83E37152BF3
:1020C00029D104F5C04393F8B81011F0010120D1D3
:1020D000D5F8DC26072A1CD093F92E310BB9042140
:1020E000E6E720460AF09CFEDFED0F7AB4EEE70A41
:1020F000F1EE10FAF3DB04F5C140343081F014FD49
:102100000028ECD004F55B50084A0621203056F038
:10211000FBF90721CCE70321CAE704F59E436833A6
:102120009A42F8D138BD00BF0000B442E07C0C08F0
:1021300010B5204CA26DA4F1DC039A422DED028B68
:10214000B0EE408A03D00020BDEC028B10BDD4F865
:10215000DC36042B25D194F8813033B11649A1F631
:10216000DC202DF029FA0028EED19FED147AF0EE54
:10217000C87AF4EEC77AF1EE10FA09D49FED100A8E
:1021800028EE008ABDEEC88A18EE103AC4F8583618
:102190000C4881F0C9FC0028D5D0002384F88B3688
:1021A000D2E7B4F83E17A4F5A04006F0E1F9002804
:1021B000D1D1C8E7107C0020EC8D00200000003455
:1021C0000000C842C48C002010B52DED028B00F534
:1021D000A0430446D3F8DC36042B0BD104F094F969
:1021E0002046B0EE408A04F05DFA38EE400ABDECBD
:1021F000028B10BD00F5C04494ED860AF7E700009D
:102200002DE9F0412DED028B00F58C658AB0044676
:10221000284612F0D7FB002307A904F5A250079324
:10222000089309930FF05CFE002800F085809DED77
:10223000090ADFED587A04F5A04505F5CD6393ED65
:10224000007A20EE270ADFED547AA7EE270A04F57C
:10225000AF40783083ED000A66F0D0FD2046FFF7EE
:102260000FFFA86D03689B6B984795F88F36002B7E
:102270005DD100285BD095F8D436002B57D1D5F826
:10228000DC36042B6FD09FED458A204604F02CFAF3
:1022900004F5C04204F59E43C2F8A403A96D3C3383
:1022A000994204F500561AD192F86032BBB9B6F9DA
:1022B000043F002B04DC3A49D1F8C41EC9060ED5F0
:1022C000D2F8C871D2F8D0117F680A33C91B6427CD
:1022D0007B438142ACBF5B181B18C2F8A433D5F80E
:1022E000DC36D2F8A413D5F8842005912046049258
:1022F00003930CF0AFFDB5F9928007462046FFF737
:1023000063FFCDE9007806F20C5605F5DF6504F5AC
:102310003F50F0EE400ADDE90332D6ED001A95EDAC
:10232000001A0599B0EE480A103080F0C3FE0AB0DA
:10233000BDEC028BBDE8F08104F59070FFF7EAFB7D
:1023400002280AD994F81434B02202FB034393F80C
:10235000402212B193ED8B0A6BE7284612F0CCF9BC
:10236000B1EE400A65E704F5C34604F5C3475C36A1
:102370006C3704F5C3413A464C31304615F05CFCED
:10238000002880D03946304615F0EAFCB0EE408A8D
:102390007BE700BFCDCC4C3ECDCC4C3F00000000D5
:1023A000104C0020FFF72CBF00F5A04300F59E4025
:1023B0009A6D603082421FBF03F5CE6301201B6817
:1023C0000B6008BF0020704710B500F5A04200F573
:1023D0009E43926D60339A420C4612D000F54050F5
:1023E000D0F8080903681B69984707EE900A9FED2B
:1023F000067AF8EEE77A012067EE877AC4ED007A74
:1024000010BD0020FCE700BF0AD7233C10B500F543
:10241000A04200F59E43926D60339A420C460AD06A
:1024200000F54050D0F8080903685B69984701201F
:1024300084ED000A10BD0020FCE7000030B5054621
:102440000FC985B06C4684E80F0040F2793221460E
:10245000284604F0FDFC0B4BA3F1B4029B6D9342A4
:102460000ED19DF8001011F0040102D1204615F0A4
:10247000DFF90548214604F0A7FD012005B030BD75
:102480000020FBE7107C0020102C002000F5A0406D
:10249000806D03689B6C184700F5A040806D036851
:1024A000DB6C184710B500F5A25300F50050D3F8C7
:1024B00008421460D3F804320B60D0F8C43E9B0588
:1024C0000BD400F20C50D0ED006AD2ED007A9FEDF3
:1024D000037AE6EEC77AC2ED007A10BD35FA8E3C7B
:1024E00038B50C4D044629460B480FF025FC04F581
:1024F000A04305F13C0183F8810004F5A25004F5E6
:10250000C0440FF0B1FAD4ED867AF1EE677AC4EDEB
:10251000867A38BDEC8D00205040002010B504466E
:1025200000F590701EF06AFF2046BDE81040FFF7EE
:10253000D7BF0000FFF7F2BF00F50050D0F8C43E4F
:10254000194214BF012000207047000010B500F5AB
:10255000A0430446986D03689B6D9847014604F5B7
:102560009F401830BDE8104083F054BFFFF7EEBF26
:1025700038B5054B1C6823680A461D68034B0146A5
:102580002046A847002038BD0C2C0020102C00202D
:1025900070B52DED028B0446036804F500559B6D64
:1025A0009847D5F8C43E1B0617D5B5F97034B5F970
:1025B0007214CA1A0B4402EBD27203EBD37352109B
:1025C0005B1000EE902A00EE103AF8EEE00AB8EE4A
:1025D000C00A04F5A2500FF005F85A4BB5F8A22432
:1025E0001A7004F5C54560F04DFC6C3560F09CF840
:1025F00000212846FEF7F4FF534E0123B071284610
:10260000F3717BF0A1FC28B928467CF06DFDB0FA8F
:1026100080F040093071042120460CF099F920B176
:1026200004F5B040183050F003F928467BF08CFCDC
:10263000E0B994F8143404F5C04504EB031341F2F7
:102640008832D3F8C461D5F86432F31A93420DD9B5
:1026500004F59070FFF75EFA022807D9C5F86462A6
:10266000204604F0F3FC0023C5F8B430B4F9A430DC
:102670001BB9B4F8A230A4F8A430B4F8A430DFED4C
:10268000338A07EE903AF8EEE77AB7EE008A88EEE2
:10269000270AD4ED2B7AF0EEE77AF4EEE87AF1EE41
:1026A00010FA09D5B4F9A23007EE903AF8EEE77ABD
:1026B00088EE277A84ED2B7AD4ED2B0A26F0B2FF30
:1026C00020BB50F0C5FF40F27D124FF4801150F056
:1026D00077FF4EF04DFC4EF0B5F804F54A500C3043
:1026E000B0EE408A74F082FD04F54F50B0EE480A17
:1026F000283074F07BFDB0EE480ABDEC028B04F587
:1027000054501C30BDE8704074F070BDD4ED2B7A8D
:1027100094ED460AF0EEE77AF4EEE87AF1EE10FA7C
:1027200009D5B4F9A23007EE903AF8EEE77A88EED0
:10273000277A84ED2B7AD4ED2B0A26F073FF00283C
:10274000BFD0C6E75C2300205D900020000000346D
:10275000FFF71EBF70B500F5C046044696F92C3150
:10276000002B2ADD06F032FD38BB04F5C5456C357B
:1027700028467CF0B9FC00B328467BF0E5FBE0B1CD
:1027800085F06CFA04F5A0434FF47A72D3F87836EA
:10279000C01A96F92C31534398420ED301221C21C2
:1027A0002846FFF7EFF840B104F55B50034ABDE857
:1027B00070400621203055F0A7BE70BD007D0C088A
:1027C00030B52DED028B83B0044601A900F5A2506F
:1027D0000FF058FB002874D004F5AC4595ED187A3D
:1027E000DDED017AB4EEE77AF1EE10FA05F160055D
:1027F00007D504F5C5406C307BF0B0FB08B1019BF8
:102800002B6004F500541820B4F97034052BB8BFC0
:10281000052307EE903A04F2C443D3ED006AB4F9FD
:10282000723407EE103AB8EEC77AF8EEE77A37EE70
:10283000077AC6EE870AB6EE007AF4EE470AF1EEA2
:1028400010FAC8BFF0EE470A9FED2D7A67EE877A3F
:102850009FED2C7A86EEA71AF0EE007AB4EE671A96
:10286000F1EE10FA48BFB0EE671ADDED017AF4EE32
:10287000C77AF1EE10FACCBF86EEA70AB0EE410A95
:1028800026F0E2FFB0EE408A1F480EF0E3FA90B95E
:102890001E484021FFF750FE68B11D4BD3F8DC36CF
:1028A000012B08D1F7EE007AB4EEE78AF1EE10FAC8
:1028B00058BFB0EE678AB0EE480A03B0BDEC028B99
:1028C00030BD04F5C5406C307BF048FBB7EE008AA4
:1028D0000028D9D046205FF077FDB4EEC80ADFEDBE
:1028E0000D7AF1EE10FAD8BFB0EE480A87EE800AF2
:1028F000AEF084FD2F209FED081ADFED080ABFE738
:102900003333333F17B7D13850400020102C00200C
:10291000107C0020000034428FC2D53F9A99193FA5
:10292000F8B504465EF0BCF90368DB6898470546D5
:1029300010B900252846F8BD204606F0D9FA04F55E
:10294000A0460746B06D03689B6B984778B10E4B65
:10295000986D03685B6B984748B104F5005494F98F
:102960001935002BE5D0032BE3D03D46E2E796F87E
:102970006C30002BDED004F5005494F9DC54023D99
:1029800018BF0125D6E700BF107C002073B500F505
:10299000A04300F59D42996D93ED280A4032914283
:1029A00029D100F50052D2F8202FB2F90840003C9E
:1029B00018BF012400F5495500F58050D3F8F066A2
:1029C000D0F8382693F8EC361435B61A5BB10B48BC
:1029D0008DED010A4FF40061FFF7AEFD9DED010A98
:1029E00080F00100C3B222463146284602B0BDE85D
:1029F00070407DF021BA0024DCE700BF102C0020DD
:102A000010B5044605F0B2FE98B104F5A042D2F824
:102A1000F03603F58C415031C2F8F01604F58051C0
:102A2000D1F838160029BEBFA3F58C43503BC2F83D
:102A3000F0362046FFF7AAFFBDE8104004205FF003
:102A4000AFBC00002DE9F0412DED048B00F50056E0
:102A500006F20C5393ED008ADFED358A28EE288AC2
:102A600000F5A048BDEEC88AD8F8F43698ED289A4B
:102A700018EE102A1A4408EE102A054646205FF088
:102A8000A3FC06F2B443D3ED007AD8F85800B8EEB0
:102A9000C88A05F59D43A0EE278A40339842FDEE93
:102AA000C87A17EE904A41D1D6F8243FB3F90860AE
:102AB000003E18BF012603685B699847C0B9D8F883
:102AC000580003689B6B984790B905F5C047D7F845
:102AD0009C33022B0CD1284609F0F6FF40B1D7ED0C
:102AE000437A67EEA87AFDEEE77A17EE903A1CB2C9
:102AF00005F54E5705F580552C37D5F83C36E41AC8
:102B000098F8EC363BB10B484FF40061FFF714FD29
:102B100080F00100C3B2B0EE490ABDEC048B32462E
:102B200021463846BDE8F0417CF0C2BE0026C2E72F
:102B30000000C842102C002010B504460CF0D6FA54
:102B400068B100B200EB4000C0EB001300EE103A99
:102B5000B8EEC00ABDE8104013205FF021BC20464B
:102B6000FFF770FFF6E7000010B50E48FFF7D8FE3C
:102B7000B0B10D4C04205FF027FCD4F8200F5EF0BC
:102B8000FFFA04205FF00CFC13205FF01DFCD4F86A
:102B9000240F5EF0F5FABDE8104013205FF000BC92
:102BA00010BD00BF102C0020104C002070B52DED82
:102BB000028B0446FFF7B4FE00287BD004F5A04545
:102BC00004F59D42AB6D5032934273D004F59D42A3
:102BD000783293426ED004F59E421C32934269D003
:102BE00004F59E42934265D00832934262D004F5C8
:102BF0009D42483293425DD004F50056F6EE008ABD
:102C0000D6F8200F5EF07CF9B4EEE80AF1EE10FA87
:102C10003DDDB0EE087AFFEE007AE0EE077AB0EE26
:102C2000670AD6F8382FD5F8F03607EE902AB8EEB6
:102C3000E77A07EE903AF8EEE77A5142E7EE007A4B
:102C4000FDEEE77A17EE900AC5F8F00626F09CFE36
:102C5000AA6DC5F8F00604F59E4344339A4222D08B
:102C6000D6F8240F5EF04CF9B4EEE80AF1EE10FA53
:102C7000B0EE408A21DCFEEE007AB4EEE70AF1EE17
:102C800010FA22D5B0EE087AF7EE007A19E0FEEEDF
:102C9000007AB4EEE70AF1EE10FAC2D5B0EE087A87
:102CA000F7EE007AB9E726484FF48051FFF744FC6D
:102CB0000028D5D0BDEC028B70BDB0EE087AFFEED7
:102CC000007AE8EE077AB0EE678A204605F04EFDFE
:102CD00008B1B1EE488A06F59163D3ED006AD5F8E4
:102CE000F4369FED186A06F63C7696ED007AB5EE5E
:102CF000C08A07EE903AF1EE10FACCBF28EE268A91
:102D000027EE488AF8EEE77A66EE866AE8EE067AFB
:102D100027EE067AFDEEE77AFDEEE66A17EE903AC8
:102D2000BDEEC77A16EE902A17EE101A17EE900A2B
:102D3000C5F8F43626F028FEC5F8F406BAE700BF59
:102D4000102C00200000C84270B5044604F5A045D0
:102D500084F084FFAB6EC31AB3F5FA6F064602D94E
:102D6000A86D06F0E3FE2D4BAE66986D0268136801
:102D70009847002120460AF053F8DFED297AB0EE9B
:102D8000C00AB4EEE70AF1EE10FA45D504F5C043E7
:102D9000D3ED867AB1EE047AF0EEE77AF4EEC77AF4
:102DA000F1EE10FA38D504F58C6011F0A5FCF6EEC2
:102DB000007AB0EEC00AB4EEE70AF1EE10FA2BD5B5
:102DC00004F5C25595ED017AF0EE087AB4EEE77A93
:102DD000F1EE10FA05F104051ED504F54950143042
:102DE0007DF09AF804F54E502C307CF011FE04F57D
:102DF000545004307DF03EFD95ED007AF7EE007AF8
:102E0000B4EEE77AF1EE10FA06D504F559503830F1
:102E1000BDE870407DF084BA70BD00BF107C00201A
:102E20000000003400F5005090F96734012BC3BF57
:102E300000F57D6090ED290ADFED047A9FED040A2C
:102E4000C8BF20EE270A46205FF0AABA0000C84299
:102E5000000000002DE9F0412DED028B00F5A048A7
:102E60000546D8ED288A09F04FFC0746D8F85800E7
:102E700003681B6A984705F55456043698B14E4CC2
:102E8000D4F8B436002B0EDD84F0E8FED4F8B43666
:102E9000C01A40F6B733984205D8B4F9A846304670
:102EA0007DF0F4FC7AE005F5C04305F5005493F895
:102EB000913343B1B4F9F834002B04DD05F54053E8
:102EC00093F91A3513BBD8F8583005F59D454035B0
:102ED000AB426DD00021B0EE680A30467DF06EFA4C
:102EE000054604205FF070FA2AB207EE902A04F239
:102EF000AC43F8EEE77A93ED007AE0EE077AFDEE68
:102F0000E77A17EE904A3C4424B2C8E701212846EC
:102F100009F0D0FD9FED297AB4F9F834C0EE077AB4
:102F200008EE103AD8F8F0369FED250AB8EEC88AB8
:102F300028EE278A07EE903AF8EEE77A67EE807A75
:102F40009FED200A27EE800AAEF07CF8B4F97034C9
:102F5000DFED1D7A20EE270A07EE903A08F2FC63B7
:102F600093ED007AF8EEE77A0021B4EEE77AF1EE1D
:102F700010FA58BFF0EE477A80EE277A3046DFED40
:102F8000137AB0EE480AA7EE270AF0EE680A7DF041
:102F900071FBBDEEC00A10EE103A1CB2BDEC028B04
:102FA00020460B49BDE8F04141F2941226F0FCBCEA
:102FB000391E18BF01218EE7107C002000A08C452F
:102FC0000AD7233C35FA8E3C0AE81C41E02E6542C4
:102FD0006CEEFFFF38B500F540530546D3F80809FD
:102FE0000368DB689847014605F5595038307DF095
:102FF00079F904B22846FFF793FC70B107EE904AC6
:1030000005F50055B8EEE70AD5F82C0F5EF0B8F8D4
:10301000BDEEC00A10EE103A1CB220460349BDE8CE
:10302000384041F2941226F0BFBC00BF6CEEFFFFA7
:1030300038B590F81434B02202FB030393ED837A81
:10304000F7EE007AB4EEE77AF1EE10FA054600F5F5
:10305000A0441DD5002109F0E3FEDFED427AB0EE79
:10306000C00AB4EEE70AF1EE10FA11D5D4F8DC3656
:10307000012B0DD0072B0BD0002384F84C3604F520
:10308000CA64002323602846BDE8384009F03CBBF1
:1030900084F0E4FDD4F85436C4F85406C31AB3F5EA
:1030A0007A7F84BF002384F84C36284609F02CFB35
:1030B000D4F8DC36012B07EE100A2DD0072B2BD0CD
:1030C000B8EEC77ADFED286AC7EE267A05F500521A
:1030D000B2F9BC2400EE102AB8EEC00A27EE800A2E
:1030E000DFED207AB0EEC07AB4EEE77AF1EE10FAB6
:1030F00014D4002384F84C3694F84C3605F5595016
:103100003830DBB97CF0D6FFBDE83840174900B253
:1031100041F2941226F048BC9FED150A94F84C2613
:10312000002AE9D10122934284F84C26E4D0072BEF
:103130001EBF04F5CA6300221A60DDE704F5CA6405
:1031400094ED007ADFED0B7A67EEC77A9FED0A7A8D
:1031500067EE877AFDEEE77A17EE901A7DF0C2F8F7
:10316000D2E700BF0000003400A08C456CEEFFFFEA
:1031700000000000E02E65420000C84270B52DED51
:10318000028B00F5C146343682B00546304680F0E9
:10319000FBFB0446E8B905F50053D3F8202FB2F93C
:1031A000082082B905F5C042D2ED867A03F597630F
:1031B00093ED007AF0EEE77AF4EEC77AF1EE10FACA
:1031C0004CBF01240024304680F0F2FB002808BFE9
:1031D0000024304680F0D8FB28BB05F5A043D3F887
:1031E0004836013319D0F4B99FED1A8A2846FFF703
:1031F00031FE07EE900AB8EEE70A8DED010AD4B968
:1032000015205FF0CDF89DED010A1A2002B0BDEC4B
:10321000028BBDE870405FF0C3B8002CE4D02846B4
:10322000FFF706FF02E02846FFF7D4FE07EE900AFC
:10323000B8EEE78ADAE71A205FF054FB9DED010A49
:1032400008B9B0EE480A15205FF0AAF8B0EE480AB7
:10325000DBE700BF0000000010B500F5005303F5E8
:103260009162D2ED006ADFED137A9FED136A03F6E7
:103270003C7292ED007A03F57D6366EEA76A27EE55
:10328000277AD3ED2A7A67EE867AFDEEE66ABDEEFE
:10329000C77AFDEEE77A044616EE902A17EE101A6A
:1032A00017EE900A26F070FB04F5A044C4F8F4066B
:1032B00010BD00BF0000C842A00CB34510B50446C5
:1032C0000BF04AFB031E2CDB04F5005292F9672435
:1032D0009A4226DD04F5A041D1F8DC06022820D070
:1032E00004F51354D4ED007ADFED0E6AD31A66EEBE
:1032F000E76A07EE102A07EE903AB8EEC77AF8EEC2
:10330000E77AD1F8F43687EE876A07EE903AF8EE5E
:10331000E77AE6EE867AFDEEE77A17EE903AC1F8A4
:10332000F43610BD0000C842F8B52DED028B00F553
:10333000A0459FED440AD5F8F0369FED437A07EE9D
:10334000903AF8EEE77A044667EE807A9FED3F0AFE
:10335000F0EEE76AF4EE476AF1EE10FAC8BFF0EE5D
:10336000477A27EE800AADF0DDFC26F08FF9B7EE44
:10337000008AC8EE007A05F5DF6704F50056C7ED50
:10338000007A96F9983453B3204605F0EFF930BB34
:10339000B6F97034012BB8BF012307EE903A05F25D
:1033A000FC62F8EEE77AD2ED006A86EEA77AB4EE18
:1033B000C87AF1EE10FA15D840F6C4122449D5F8AF
:1033C000F00626F0E1FAC5F8F006D6F8382F40F6F8
:1033D000C4139A42D4BFC6F8382FC6F8383FBDECA4
:1033E000028BF8BDD7ED007AB4EEE77AF1EE10FA71
:1033F000F5D588EE070A20EE000AADF04DFEDFEDB0
:10340000157AD5F8F00620EE270ADFED137A20EEC4
:10341000270A40F6C413FDEEC07A17EE904A9C428C
:10342000B8BF1C462246614226F0AEFAC5F8F00647
:10343000D6F8383FA342D4BFC6F8383FC6F8384F55
:10344000CDE700BF0AD7233C0000AA4235FA8E3CE4
:103450003CF6FFFFE02E65420000C84210B500F5C3
:1034600040530446D3F8080903681B68984704F5DD
:103470000053D3F8382F514226F086FA04F5A043C2
:10348000C3F8F0062046BDE81040FFF74DBF00002E
:1034900070470000012070470820704701207047E6
:1034A00070470000014B93F8A4047047104C0020B3
:1034B000034B93F9B80C003818BF0120704700BFC8
:1034C000104C0020014B93F9A6047047104C0020CB
:1034D00013B5054B986D4B690468009308310EC90C
:1034E000646CA04702B010BD107C00207047000043
:1034F000002070477047000038B5244DA86D036860
:103500005B6898470F2833D80F2838D8DFE800F0D9
:1035100008350808080808080837353535353535C1
:1035200010241B4B93F8D92612B193F8D8360BB957
:1035300044F01004174BAA6D9A42A3F1080303D07C
:103540009A4218BF44F01004134991F91915C1B1FA
:103550009A4218D0032902D1104B9A4201D144F06B
:1035600040040F487AF0F0FC68B144F080040AE0AF
:10357000182814BF01241824D3E71824D1E7012404
:10358000CFE79A42EDD144F0010038BD107C002015
:10359000105C0020707B0020104C0020347B002049
:1035A000FC8E002008B5044805F010FE00280CBF72
:1035B0000120022008BD00BF102C0020F0B52DED29
:1035C000028B8BB005460EF079FE4FF48071D0F877
:1035D000047290ED828AD0F80C6204461448FEF71B
:1035E000ABFF30B9134BDFED147A93ED007AA7EE01
:1035F000678A2D7C84F032FBD4F81823D4F81C336E
:10360000D4F814130892099327221C23CDE9003221
:103610000390079103AA1E21284604978DED058A81
:10362000069655F0A5FF0BB0BDEC028BF0BD00BFB8
:10363000102C00201C51002035FA8E3C2DE9F04161
:10364000404E2DED068BB26DA6F1A0039A428AB0D2
:1036500073D0A6F5005390F81080D3F80879D6F807
:10366000F0369FED399A07EE903AD6F8F436B8EE78
:10367000E7AA07EE903A3B6838469B68F8EEE79A6F
:10368000984707EE900AF8EEE77A384667EE897AAF
:103690002AEE09AAFDEEE77A69EE899A17EE903ACA
:1036A0001DB23B681B69984707EE900AF8EEE77A6F
:1036B000A6F5A04067EE897AFDEEE77A17EE903A1C
:1036C0001CB206F5CE63D3ED008ADFED207AF4EE6E
:1036D000E78AF1EE10FA58BFF0EE678A02F06CFE4E
:1036E0003B68D6ED23AADFED1A7A5B6908EE100A73
:1036F00038466AEEA7AA9847FCEEE88AB8EEC88A70
:1037000018EE903AB72228EE098AADF824301A2331
:10371000CDE900323E2103AA40468DED03AACDED4E
:10372000049A8DED058ACDED06AA8DED070AADF858
:103730002050ADF8224055F01BFF0AB0BDEC068BBF
:10374000BDE8F081107C00200AD7233C00FF7F47B2
:103750000000C84208B502480BF0FEF800B208BDF0
:10376000102C002037B50D46134840F2EF2203F02D
:103770006FFB2C7814F004040AD0696803220F4808
:1037800013F092FF0C4803B0BDE8304002F030BDAA
:1037900001AA2146284614F05BF80028F2D0DDED9E
:1037A000017A9FED077A67EE877A2246FDEEE77A87
:1037B00017EE901AE3E700BF102C0020FC8D0020CC
:1037C0000000C84210B5054C012384F8DB3657F0E1
:1037D000D1FB002384F8DB3610BD00BF105C002055
:1037E0005AF078BE2DE9F0412DED028B4FF0000824
:1037F00082B0CDE900281E4F9FED1E8A0C4615466B
:10380000B0EE480AB1F90220D7F8201F4FF47A73BE
:1038100006465BF047F90123CDE90053B4F90020D7
:10382000D7F8241FB0EE480A30464FF47A735BF0A5
:1038300039F9B4F90420D7F8281F9FED0F0A434641
:103840003046CDE900585BF02DF9CDE90058B4F9C8
:103850000620D7F82C1FB0EE480A4FF47A73304692
:103860005BF020F902B0BDEC028BBDE8F08100BF37
:10387000104C00200000FA4400007A4438B5C578A6
:103880000B46352D044628BF352535220021184624
:10389000AFF064FE2A4604F10C01BDE83840AFF0F9
:1038A00013BE000010B5074B93F9182840F24D34B1
:1038B00040F24D13002A08BF1C4657F0A3F92043DD
:1038C00010BD00BF107C002010B5044614F0F0FAC3
:1038D000204610BD10B50A4C002384F88B3658F0F2
:1038E00043F8A26DA4F1DC039A4208D194F804379E
:1038F0002BB904F5E060BDE810402BF0B7BD10BD5A
:10390000107C002013B5124C94F88E1204F5A070B0
:103910000CF000FA78B194F88E1204F5A0700CF057
:1039200067FC40B194F88E1204F5A07002B0BDE8B7
:1039300010400CF09FBC0EF0C1FC01A90EF0A2FAE1
:1039400018B19DED010A02B010BD9FED020AFAE721
:10395000104C00200000000008B5084BD3F8A82E3A
:10396000002A03DCBDE8084057F0C4B803F6C8508D
:1039700054F03AF990ED000A08BD00BF104C002049
:1039800008B51048826DA0F1A8039A4214D0B0F98E
:1039900070309BB990F8153683B990F86D306BB9DB
:1039A00090F8C53663B9A0F5A04005F00FFC0028DB
:1039B0000CBF0320042008BD0220FCE70520FAE725
:1039C0000620F8E7107C002010B5204BA3F1A002E0
:1039D0009B6D934290B0044636D000231C4802935E
:1039E00013F04CFE014618B9194802AA13F092FED2
:1039F000247C84F033F9174BDDED027A9FED167AC3
:103A0000D3E97D2305930023F8EEE77A0793089323
:103A100009930A930B930C930D930E934FF6F8535F
:103A2000ADF83C300023CDE9030267EE877A962299
:103A30008DF83E303323CDE90032572103AA2046CA
:103A4000CDED067A55F094FD10B010BD107C00202D
:103A5000FC8D0020108C00200AD7233C10B557F0B5
:103A6000CBFA044670B90848826D80F88B46A0F105
:103A7000DC039A4206D190F804371BB900F5E060E8
:103A80002BF0F4FC204610BD107C00200120704774
:103A900008B5034B986D03685B68984708BD00BF85
:103AA000107C002030B587B005460EF007FC0446B8
:103AB0002D7C84F0C7F8D4F88422D4F8883204929C
:103AC000059300211023CD22CDE90032029003910D
:103AD00002AA42F60C31284655F04AFD07B030BD27
:103AE00030B52DED028B89B005460EF0E7FB00F5F1
:103AF0005A7393E8070002AC84E80700DDED020A80
:103B00009DED030A2D7CF1EE600AB1EE400AADF0A6
:103B10002BFB2046B0EE408A28F07AFDDFED0B7AD1
:103B2000049B079328EE278A0C230122CDE900325B
:103B3000A82105AA28468DED058A8DED060A55F0C7
:103B400017FD09B0BDEC028B30BD00BFE02E654211
:103B5000282938B5054623D007D824292BD0272972
:103B600011D01B2908D1012413E0432937D008D8EC
:103B70004029F8D0422928D02846BDE838405BF0DB
:103B8000EDB85329EEE7122154F0F0FE044610B9C7
:103B90000024204638BD297C13484DF089FDF8E704
:103BA000162154F0E3FE04460028F1D0297C0E488B
:103BB0004DF058FEEDE70C2154F0D8FE04460028E5
:103BC000E6D02846FFF78CFFE3E7102154F0CEFE45
:103BD00004460028DCD02846FFF764FFD9E7017CC3
:103BE00002487FF0CFFEBEE728840020C48C00206E
:103BF000F0B52DED028B05468DB01646B0EE408A2D
:103C00000C46002930D0007C55F048FC0746287C43
:103C100056F048FB00F121039F4207D2287C0DB0EB
:103C2000BDEC028BBDE8F04054F08EBE6369089392
:103C3000636A2269CDF82530236AA069E16807929A
:103C4000CDF829306222212327680590CDE9003282
:103C50000691287C0397192303AAC2218DED048ABB
:103C60008DF8246055F084FC0DB0BDEC028BF0BDE6
:103C700070B52C4DAA6DA5F1A0039A42044650D010
:103C8000A5F54056B6F84A35DB0708D5A5F500532B
:103C900093EDE00A012203F55F71FFF7A9FFB6F883
:103CA0004A35980708D520490B4693ED000A043998
:103CB00002222046FFF79CFFB6F84A35590708D57F
:103CC0001A490B4693ED000A043903222046FFF7F8
:103CD0008FFFB6F84A351A0708D515490B4693EDFC
:103CE000000A043905222046FFF782FFB6F84A355C
:103CF000DB0616D5D5F8DC36042B12D10EF0DEFA31
:103D000005460C487FF06EFE95EDC70ADFED0A7A96
:103D1000014620EE270A20460622BDE87040FFF744
:103D200067BF70BD107C0020EC6000206062002046
:103D3000BC620020C48C0020E02E654270B50446B1
:103D40000E461DF099FB90F8F412B02303FB01011D
:103D5000DC31204603F0EAF9054690B13EB10EF0A1
:103D6000ADFA90F87C3243F0020380F87C3204F51F
:103D7000A04304F59E44986D3C34A04201D105F067
:103D800023FE284670BD000073B516460191044617
:103D90000EF094FA01990DF0BDFE054690B13EB1CA
:103DA0000EF08CFA90F87C3243F0020380F87C32FB
:103DB00004F5A043986D04F59E433C33984201D12D
:103DC00005F002FE284602B070BD000030B5054681
:103DD00085B00C46D1E9040125F0ECFF40B16846FE
:103DE00013F05CFC6A46214628465AF0CBFD08B920
:103DF000022066E0344840F24F32694603F028F86A
:103E0000D4ED037AF4EE677AF1EE10FA22D69FED44
:103E10002F7AF0EEE77AF4EEC77AF1EE10FA54BF9B
:103E2000012200229DF80030294962F341036846CF
:103E30008DF8003013F09CFD0028D9D12548694643
:103E400069F0C4FC40B951F015FA0522162150F072
:103E5000C9FFCDE70022E5E7D4ED017AFDEEE77A70
:103E600017EE903ADB0705D41B4BA3F1B4029B6D10
:103E7000934225D11949144802220AF083FB9DF888
:103E8000001011F0040102D1684613F0D1FC0E4875
:103E9000694603F099F894ED020AB4EE400AF1EE97
:103EA00010FA0BD6B5EEC00AF1EE10FA06DD9DF859
:103EB00000100A48C1F3400106F000FE002000E0B7
:103EC000042005B030BD00BF102C002000000034DD
:103ED000EC8D0020204F0020107C00205C7B002017
:103EE00010B52DED028BD1ED017A91ED008AFCEE3B
:103EF000E77A8AB0CDED037A9DF80C1005AA044646
:103F00005AF02AFDC8B1DFED0E7A059B009368EEEA
:103F1000277A0022FDEEE77A114617EE903A06A8BE
:103F200013F0DCFB23682046D3F8CC3006A9984771
:103F300000200AB0BDEC028B10BD0220F9E700BFE3
:103F40000000C84237B5114DA86D03681B6A0C46C6
:103F5000984738B9AA6DA5F1DC039A4202D0042033
:103F600003B030BDD4ED007AD4ED020A94ED010A1D
:103F70000748FCEEE77ACDED017A9DF8041003F0D6
:103F800089FE0028EBD00020EAE700BF107C00206B
:103F9000102C002008B5D1ED007A9FED087A084872
:103FA000F0EEE77AF4EEC77AF1EE10FA54BF012191
:103FB000002104F0D5FB002008BD00BF0000003444
:103FC000102C002010B5D1ED007AFCEEE77A17EE48
:103FD000903A9CB2012C02D0022C06D084B9114830
:103FE000214664F079FE002010BD0F4890F80C388F
:103FF0005B0707D55BF060F90C4A052154F084FAA1
:104000000420F1E790F9F8371BB95BF055F9084A3D
:10401000F3E7A0F5A04008F037FA002814BF00200D
:104020000420E1E708840020107C00201C830C0899
:1040300037830C0838B58B8BC02B05460C4631D81E
:10404000B12B0BD8112B00F09480142B00F094802E
:1040500021462846BDE838405BF074BFB23B0E2BCA
:10406000F6D801A151F823F0D740010851400108CA
:1040700051400108514001085140010851400108D8
:104080005140010851400108CD400108514001084C
:10409000F14001082941010851400108E1400108AF
:1040A000C3400108D42B08D0B3F5967F47D0D02B5E
:1040B000CED1BDE83840FFF785BFBDE83840FFF7F7
:1040C00069BF2146BDE83840FFF780BE2146BDE804
:1040D0003840FFF705BF2146BDE83840FFF732BF43
:1040E00094ED000A2748FEF723F8D8B100201AE023
:1040F000254C94F88130ABB1244904F5E0602BF0F5
:10410000B3FA78B1012384F839370222A4F1DC0133
:10411000A4F5A0400AF036FA0028E7D11A4B002295
:1041200083F83927042038BD174C94F88130002BD0
:10413000F8D0164904F5E0602BF01AFAE1E7D1ED6A
:10414000007A9FED137AF0EEE77AF4EEC77AF1EE9B
:1041500010FA14D5D1ED017AF0EEE77AF4EEC77AD1
:10416000F1EE10FA0BD50B49022206480AF00AFAC2
:10417000BCE709490222F8E708490222F5E70220D4
:10418000D1E700BF102C0020107C0020EC8D002017
:1041900000000034347B0020547B00204C7B002046
:1041A000F0B5414CA26DA4F1B4039A428FB00D4614
:1041B00077D1CE78272E28BF27262722002104A8D2
:1041C000AFF0CCF9324605F10C0104A8AFF07CF950
:1041D000059B9DF836500093069B0193ED43079B8A
:1041E0000293EDB2089B03938DF8365083F036FDB1
:1041F00015F0810F05F08707064601D1802F12D1F7
:10420000684627F06DF9DFED297AC4F8AC6620EE38
:10421000270ADFED277A20EE270ABDEEC00A10EE4E
:10422000103AC4F8A03615F0820F01D1802F12D1B8
:10423000684627F06FF9DFED1D7AC4F8B06620EE0E
:10424000270ADFED1B7A20EE270ABDEEC00A10EE2A
:10425000103AC4F8A43615F0840F01D1802F12D182
:10426000684627F067F9DFED117AC4F8B46620EEEE
:10427000270ADFED0F7A20EE270ABDEEC00A10EE06
:10428000103AC4F8A8366B060BD5DDED0C7A9FED1D
:10429000087AC4F8BC6667EE877A04F5D763C3ED85
:1042A000007A0FB0F0BD00BF107C0020E02E654208
:1042B0000000C84230B51E4C91B0084602A9FFF775
:1042C000DDFAA26DA4F1B4039A422FD19DF83C30DF
:1042D000072B2BD104F58054D4ED7C7ADDED056AF3
:1042E0009FED147AF8EEE77AE6EEC77AFDEEE77A0C
:1042F000C4ED7C7A5AF0E0FFD4F8C821D4F8F0314C
:1043000052689FED0D7A9B1A07EE903AF8EEE77A25
:10431000054667EE877A17EE900AFCF7F5F8074A2C
:10432000CDE900010621284654F0EEF811B030BD69
:10433000107C00200000C8420AD7233C50830C08A0
:1043400010B51D4BA3F1B4029B6D9342044696B089
:1043500008460FD108A9FFF791FA9DF8541003AA57
:1043600020465AF0F9FA38B95AF0A6FF134A042148
:1043700054F0CAF816B010BDBDF8503023F0040355
:104380009BB2002BF6D0DDED0B7A9FED0D7A039BEF
:10439000009367EE877A0022FDEEE77A114617EE6A
:1043A000903A04A813F09AF9236804A9D3F8CC3002
:1043B00020469847DEE700BF107C002064830C088D
:1043C0000000C84230B48D7A4B7A43EA0523CD7A97
:1043D00043EA0543562B04460A461BD008D8522B05
:1043E00012D0542B13D02046114630BC5AF084BF53
:1043F00003F18073863B23F07F43012BF3D8017CCC
:10440000064830BC4DF0F6BA30BCFFF7C9BE30BC30
:10441000FFF750BF30BCFFF793BF00BF28840020D8
:1044200000207047C8207047012070470020704767
:104430000020704790F89C308B4286BF283150F89E
:10444000210000207047000090F89C308B4286BF0E
:10445000283150F8210000207047000003207047E9
:10446000014B93F8A2047047104C002070B504462D
:104470004B4808F0CFFC18B1E36A43F40003E36251
:10448000474808F0C7FC88B146205DF09DFFDFED8E
:10449000457AB4EEE70AF1EE10FA07D8236B43F43D
:1044A00000032363636B43F400036363E36A43F431
:1044B000F843E3623C4B986D03685B6898470138AA
:1044C000172814D8DFE800F03A420C444242424236
:1044D000133A3A3A3A3A3A13131313131313133A9B
:1044E000324A92F8D8368BB392F8D9268AB3304B39
:1044F00093F8B030012B3DD0022B44D02D4B1D68DA
:10450000DDB12D4E284696F8121F47F06FFFA0B17F
:10451000E36A43F48073E36296F948351BB1236B79
:1045200043F48073236396F8121F284647F096FFE2
:1045300018B1636B43F48073636370BDD4E90C23DB
:1045400042F4E04243F4E04322636363012300E06A
:104550000023216B41F480622263626B42F480602D
:104560006063002BC3D041F4406142F44062216398
:104570006263BCE7E36A43F48003E362236B43F4C2
:1045800080032363BAE7E36A43F48003E362236BA7
:1045900043F480032363636B43F480036363ADE7F9
:1045A000102C0020000000B4107C0020105C0020C3
:1045B000108C002008910020104C002013B54FF4FF
:1045C0004470CDE9002113F06BFC044628B1DDE90D
:1045D00000215BF0B3F8024B2360204602B010BD0F
:1045E00064850C0800207047002070470020704749
:1045F0000020704700F514500430704700487047A1
:10460000ECAA0C0800F5A040806D03685B681847B1
:1046100000F5A04300F59E409B6D24301B1A5842C4
:10462000584170479B20704730B500F5A04303F216
:10463000F46353F8042CDFED296A07EE902AB8EEF4
:10464000E77AD3ED007AF8EEE77A85B027EE267A9E
:1046500067EEA67A0446002301A900F5A250039351
:104660008DED017ACDED027A04F58F550BF0D6FF72
:1046700004F54D523C32692128464FF0C7FC04F541
:10468000535218326A2128464FF0C0FC04F54053BB
:1046900093F91A2542B903F5A263D3ED007AF5EE3A
:1046A000C07AF1EE10FA06DD04F559520C326B2196
:1046B00028464FF0ABFC04F55954383420467BF0C3
:1046C00033FE28B104F130026D2128464FF09EFCE4
:1046D0000DF0F4FD0DF01AFB05B030BD0AD7233CF8
:1046E00010B54FF4801104460AF032F910B120469B
:1046F000FFF79AFF4FF4800120460AF029F928B10C
:1047000024F020FBBDE8104022F0AEB910BD00003F
:1047100070B590B0002300F5A256029302A90023C1
:1047200004460DF1070230468DF807300DF0B0FB5E
:1047300003A930460CF0DEFB08B92D4B0393302261
:10474000002104A8AEF00AFF04F5A045A3238DF8CC
:10475000103095238DF8113083F088FAD5F8F036B3
:10476000ADF81B3004F58053CDF81300D3F838268C
:10477000ADF81D20D3F83C36D5F8F426CDF8171047
:104780004620ADF81F20ADF821305DF01DFE10EE83
:10479000103A1520CDF823305DF016FE10EE103AD9
:1047A000CDF8273004F53F539FED127AD3ED2D7AE3
:1047B00067EE877A304617EE903ACDF82B30029BA1
:1047C000CDF82F309DF807308DF83330039B0D93D3
:1047D0000DF064FDD5F894308DED0E0A302204A959
:1047E00004F58F500F934FF04DFD10B070BD00BF1A
:1047F0002292CA7F0000C84270B58EB035220446AE
:1048000000216846AEF0AAFEA3238DF80030952360
:104810008DF80130012304F5A0468DF8023083F0B5
:1048200025FA04F5405506F5CE63CDF803001B6864
:10483000D5F80809CDF80710CDF80B3003681B69CF
:104840009847ADF80F00D5F8080903689B689847AA
:10485000ADF811001C4801F0AFFDADF81300D5F81C
:10486000080903685B69984710EE103AD5F8080903
:10487000CDF8153003689B69984710EE103ACDF8D3
:104880001930D6F88C30CDF81D3004F5C0433522F0
:10489000D3F8F411CDF82110D3F8F811CDF8251084
:1048A000D3F8F011D3F8A433CDF82910CDF82D307A
:1048B0006946D6F88430CDF8313004F58F504FF08A
:1048C000E1FC0EB070BD00BF102C002030B587B0E9
:1048D0001622044600216846AEF040FEA3238DF860
:1048E000003095238DF8013002238DF8023083F0DB
:1048F000BDF904F5A045CDF803002046CDF807101A
:1049000004F064FC05F5DC638DF80B001B68039371
:10491000124B1B68D86A90F89C308DF810300368F1
:10492000DB69984795F8C5368DF812308DF811007F
:1049300024F008FA23F0FCF9D5F8DC368DF81300E2
:104940008DF81430162295F8C6368DF81530694664
:1049500004F58F504FF096FC07B030BD0C2C0020B2
:1049600010B58AB02722044600216846AEF0F6FD55
:10497000A3238DF8003095238DF8013009238DF89D
:10498000023083F073F9CDF803000420CDF807104E
:104990005DF01AFD10EE103A1320CDF80B305DF0EB
:1049A00013FD10EE103A4620CDF80F305DF00CFDEF
:1049B00010EE103A1520CDF813305DF005FD10EE25
:1049C000103A0320CDF817305DF00EFD10EE103ACE
:1049D0001A20CDF81B305DF0F7FC10EE103ACDF840
:1049E0001F3004F5A0432722D3F8A030CDF82330A0
:1049F000694604F58F504FF045FC0AB010BD000029
:104A000013B5044600F58F5001904EF06DFF0198EC
:104A10004FF004F804F58053019893F910330BB16B
:104A20004FF0A4F8204602B0BDE81040FFF798BF51
:104A30007047000010B500F5A0430446986D036868
:104A40005B68984704F50053014693F8242404F565
:104A50008F504FF0D7FD04F5A2500DF07BFE04F50A
:104A60009070BDE810401BF071BD00009FED020A80
:104A7000002245F06FBE00BF0AD7233C1C4B70B527
:104A8000044640F8043B5BF08BFF1A4E1A4B636000
:104A9000542560195CF03AF966513035B5F5557F0B
:104AA000F7D104F555705EF083F8144A04F5EE6012
:104AB00002F66C317FF008FE04F67C15FF2384F8C3
:104AC0008C3984F894390E49284646F0D9F90D4BB3
:104AD0001A6812B10C4883F08FF81D60012320463C
:104AE0000A4984F8C13946F0CBF9204670BD00BFB1
:104AF000703A0020C8D50C08DCD50C087450002092
:104B000060120E08A89A002068C20C088CC50C0818
:104B10002DE9F04100F512519AB00D2220310446E2
:104B20004DF09CFF0022BE48BE4E272145F08AFD75
:104B3000042100205EF016F8132101205EF012F827
:104B4000462102205EF00EF8152103205EF00AF8DF
:104B50005DF074FD46F09AFBB34A138843F00403FA
:104B600013804FF000080AAF002110223846AEF043
:104B7000F5FC01238DF830303388ADF8283005A9D5
:104B800073680B93384645F065FCC8B19DF9143045
:104B9000002B15DD5CF084F89DF8141003680139D2
:104BA0001B68C9B2984758B1051D284645F0F0FB6F
:104BB00030B9B368ADF8183006A9284647F00CF8AC
:104BC00008F10608B8F12A0F06F10C06CCD1974877
:104BD00000220DF10B0145F0C3F906AD064620B3E6
:104BE00045F0D6FB08BB924B0FCB85E80F0004A91C
:104BF000284645F02FFC002840F03A814FF0040889
:104C00008C4B0FCB87E80F0005A9384645F022FCF6
:104C100028B105A845F0BCFB08B148F0010803A97C
:104C200030468DF80C8046F085FF834B0FCB85E82E
:104C30000F0003A9284645F00DFC002846D009982E
:104C4000002204A945F08CF9064600283ED045F024
:104C50009FFB0546002839D19DF80C30013BDBB2A3
:104C6000032B96BF754A0346D35C8DF82830304637
:104C7000394646F05FFF7248002205A945F070F9F9
:104C8000064668F0E5FF78B168F0E0FF90F8302064
:104C900090F8281090F84830114490F840200A44C9
:104CA000D34214BF0125002586B130469DF90C8002
:104CB00045F06EFB50B91DB1B8F1000518BF0125D4
:104CC000394630468DF8285046F034FF04F514502C
:104CD0000022B7EE000A01213C3045F03BFD04F50F
:104CE00013500022B7EE000A0221183045F032FDC1
:104CF00001230093534A002304F505518E2045F00B
:104D0000A5FC94F9DCC9BCF1000F1AD14E4E0FCEB0
:104D10003D460FC50FCE0FC50FCE0FC596E80F004D
:104D200085E80F0062460421384645F08BFC9FED74
:104D3000470A474846F04CFC4648B7EE000A46F0A2
:104D400047FC012504F50C51434A0095002310311E
:104D500040F2051045F07AFC04F5145002210C30A5
:104D6000FFF784FE04F5115003213430FFF77EFE77
:104D700004F5115003213C30FFF778FE04F5145080
:104D800003210830FFF772FE04F5145002211030A1
:104D9000FFF76CFE04F5125002210830FFF766FEA3
:104DA00004F5125002210C30FFF760FE04F512509A
:104DB00002210430FFF75AFE04F5C14034307EF082
:104DC00077FF264A1368D90709D42549156004F5E9
:104DD0000A5320330B6004F597531433CB6004F56A
:104DE00015501F4902221030012545F081FC1D4A53
:104DF0000095002304F58F51FD2045F027FC1A4B48
:104E00001A68D20705D4194A1D6004F59B5408346A
:104E100014601648012145F087FC1AB0BDE8F08106
:104E2000C8C20C0838C50C08EC9000208CC20C08D5
:104E3000E0770C08F0770C0800780C08C4C20C0866
:104E400097C20C0848EB0C0810780C080000000012
:104E5000A4C20C08B3C20C08A40D0E08042C002038
:104E600000220020CC840D08082C002018220020ED
:104E700004A845F08DFA00283FF4C0AE4FF00C08AE
:104E8000BEE600BF7047000000207047002070475A
:104E900000207047002070470020704770470000D6
:104EA000002070470020704784B001A880E80E0001
:104EB00004B00020704700000020704700207047B9
:104EC000704700001020704700487047D8D10C0888
:104ED00000487047E8D10C08002070477047000078
:104EE0000120704701207047002070470023436075
:104EF0008360C36003614361002303767047000051
:104F000010B50446FFF7F2FF0023637610BD0000E2
:104F1000027E531CDBB2042B037600EB820288BFB7
:104F2000002382ED010A88BF0376704710B504465E
:104F3000FFF7EEFFD4ED017A9FED107A94ED020AAF
:104F4000637E77EE877A042B77EE807A94ED030AFE
:104F500094BF0133052377EE807A94ED040A6376DB
:104F600077EE807A637E94ED050A77EE807A00EE24
:104F7000103AB8EEC00A87EE800A10BD00000000AB
:104F800010B5044612F094FF204610BD03F064BE35
:104F900003F07CB803F0D2BA03F084B801F0BCBCD3
:104FA00001F06AB801F0F2B901F032BAFDF7D2BBF4
:104FB000FDF766B870B5234B036000F54053044617
:104FC000D3F89C08204AC3F8E02608B112F074FF19
:104FD0001E4B236004F5005393F8DC2042B9D3F84C
:104FE000D8502DB1284620F0B7FD284612F060FFBA
:104FF00004F59A500C3078F003FA04F5985010300C
:105000005EF0DEFE04F6E46504F68466B54204D084
:10501000183D284620F0F6F9F8E70D4BC4F8C838DB
:1050200004F6282052F0BCFA04F6FC1052F0B8FA4C
:1050300004F65C1052F0B4FA04F5136052F0B0FAC2
:10504000204670BDE4B80C08C09F0D08CC7D0D084B
:10505000E03D0D0838B54C4B044640F8043B62F087
:1050600025F804F1100010F077FE04F168004BF011
:1050700057FC04F590701AF023FE04F58C600FF0D5
:1050800011FB04F2845012F019FF04F6C80021F05D
:105090001BFE04F5666061F0E7FD04F5736047F000
:1050A000CBF804F58F504FF021F804F597501430E9
:1050B00067F008FD04F5985010305EF069FE04F5C5
:1050C0009A500C3078F088F904F59B5008304BF07A
:1050D000E9FF04F59D501C3063F0C6F904F58053D8
:1050E00004F59F520025104683F8E053274B1030FB
:1050F0001A6041F0CBFE294604F5A2500BF0D2FB1A
:1051000004F5D550083072F077FA04F5FB500C30F6
:1051100075F086F904F50250043077F0B7FA04F51B
:105120000350283077F0ECFE04F505500AF01EFC21
:1051300004F50A50203072F041FF04F50B50144979
:10514000383045F09DFE04F50C50103068F056F8EC
:1051500004F50F500C3078F0DBFC04F5005304F537
:10516000105083F824540B4D3C3078F0F3FD2B683D
:1051700013B1094882F040FD2046084945F080FE01
:105180002C60204638BD00BFCC7D0D08149A00204D
:10519000D4130E0840910020F0D10C08D47C0D08E7
:1051A0002DE9F04F2DED028B04469FB0FFF752FF23
:1051B000E24B236004F515501030FFF75FFC04F557
:1051C0003C5018307AF03CF904F5005504F51353BF
:1051D0002A33C5F8403F04F53D50062385F8443F87
:1051E0002C305EF0E7F904F5115704F5A25304F5ED
:1051F000C14B04F54056C5F8E03F24370E930BF140
:10520000340B4FF40063C5F8EC3FC5F8E47FC5F8F4
:10521000E8BF5A2305F57D6586F86C304FF07E5364
:10522000C5F85C31C64BC5F86031C64BC5F8643172
:1052300004F54650C44BC5F86831C5F8CC312C3064
:1052400052F0CEFC04F5465004F53F59383052F088
:10525000C7FC4FF00008BD4BC6F8C83109F1100972
:1052600086F8E08109F5FC70FFF740FEB84BB949BC
:10527000C6F8C83186F8E181484645F001FEB64BD4
:10528000C6F8E8310E9BC6E97B390023C6F81C320C
:10529000C6F8243204F54755012386F82C32283508
:1052A00004F5495012F0FAF9AC4986F850822846C4
:1052B00045F0E6FD04F54950394614307AF076FCA5
:1052C00004F54E5039462C307AF0D4F804F5545099
:1052D000394604307BF034F82C22414606F5D5607F
:1052E000AEF03CF904F559509D49383004F55B584F
:1052F00045F0C6FD08F120089A4BC6F8E03608F1E3
:10530000140081F0D1FB04F55C5A04F55D530AF1F9
:10531000180A3C3350460F9357F004FB0F9B0AF1D9
:10532000140A5345F6D10723C6F8A0380023A6F87F
:10533000A4384FF4CB7012F0B9FDC6F89C0804F500
:105340006250283081F0B0FB04F563502C3081F0BE
:10535000ABFB854B1A680AB9C3F80080834BC6F8CB
:10536000E03604F564504FF48051C6F808590C300B
:1053700010F0F4FD04F566500C3043F04DF904F5DF
:1053800067500C3046F0DEFC04F5675020306AF0C0
:10539000F1FB04F59D4004F58045383004F0F6FA41
:1053A000734BC5F8B83E04F59D40403004F0EEFA6A
:1053B000704BC5F8C03E04F59D40483004F0E6FA55
:1053C0006D4BC5F8C83E04F59D40503004F0DEFA40
:1053D0006A4BC5F8D03E05F6E4630022B7EE008ABA
:1053E00004F59D40DA609A605A6083ED008A783057
:1053F00004F0CCFA624BC5F8F83E04F59E4004F088
:10540000C5FA604BC5F8003F04F59E40083004F033
:10541000BDFA5D4BC5F8083F04F59E401C3004F012
:10542000B5FA5A4BC5F81C3F04F59E40243004F0F1
:10543000ADFA574BC5F8243F04F59E403C3004F0CC
:10544000A5FA544BC5F83C3F04F59E40443004F0A7
:105450009DFA514BC5F8443F04F59E404C3004F58D
:105460009E4804F093FA08F158084C4BC5F84C3F9D
:10547000404604F08BFA4A4BC5F8583F04F59E406D
:10548000603004F083FA474BC5F8603F04F59E4056
:10549000683006F053F804F59F40103004F076FAB7
:1054A000414BC5F8903F414BC5F8983F04F59F40EC
:1054B0004FF4C053A5F8EC3F3D4904F5A045183022
:1054C00045F0DEFCFE2385F86430052385F8803046
:1054D000384B11934FF0FF3A374BC5F888A004F5CD
:1054E000A1404FF40071C5E9168885ED288A22464F
:1054F000009324302F4B10940FF00CFF05F5CB6375
:10550000104AC5F848A6DA600023C5F8A036C5F8E9
:10551000A436C5F8A836C5F8AC36C5F8B036C5F817
:10552000B4360323C5F8DC3605F5DF6383ED008A66
:10553000224BC5F8203704F5AE4841E0E4B80C082A
:10554000000080BF0000B4420000B4C25CD20C086E
:105550006CD20C08584E0E08CC4B0E08744B0E083B
:1055600010460E08C09F0D088494002040860C0849
:105570003CDC0C0840E00C0860E30C0884DA0C0802
:105580004CDD0C08D4DD0C08B4DC0C08BCDB0C08CA
:1055900038DB0C08C4DF0C08CCDE0C0854DE0C0829
:1055A000A4D20C084CDF0C08DCE20C0894D20C08E6
:1055B000E8580E088D4F010814830C08914F01081C
:1055C000834BC5F828374046824BC5F83037C5F8BD
:1055D0001C47C5F82447C5F82C47443012F05EF844
:1055E0004046603012F05AF840467C3012F056F8CF
:1055F000794BC5F8903708F19800A5F894A712F0F8
:105600004DF8764B7649C5F8F4A74046C3F80080BC
:1056100045F036FC4FF6FF73A5F83C3704F5AF4074
:10562000704B7149A5F858A77830186045F028FCF0
:1056300004F5B04018304CF005FE6C4BD6F8082944
:105640001294CDE913346A4BCDE91534694BCDE999
:105650001734694BCDE91934684BCDE91B34684BDD
:105660001D931EA911E903000CAB83E80300DDE9DB
:105670001A010AAB83E80300DDE9180108AB83E8EF
:105680000300DDE9160106AB83E80300DDE9140140
:1056900004AB83E80300DDE9120102AB83E80300F9
:1056A00004F5C0464146CDE900274B460E9A5846C0
:1056B00004F5C2487EF004F908F14008514BC6F8E1
:1056C000403108F13C0011F0E9FF4F49404645F0F8
:1056D000D7FB4E4B1F6817B14D4882F08DFAC3F8C7
:1056E00000804C4BC6F840310E9B86F8447103F5A0
:1056F0001B7304F5C340C6F8C83186F8497186F8B3
:105700006D714C3011F0CAFF04F5C3405C3011F0EC
:10571000C5FF04F5C3406C3011F0C0FF1C223946B0
:1057200006F5FE70ADF01AFF04F5C54804F5C44057
:1057300008F16C0868305EF079FC404678F0C4FBF4
:10574000354B3649C6F8EC32404645F099FB344AB1
:105750003449116004F5C64324334FF0140CB8B239
:105760000CFB00120137127C002AF8D12E4A10805F
:105770002E4A17680FB12E48AFE704F5C64028300F
:10578000136078F08BFB2B4BC6F828332A4BC6F8F6
:105790003833642386F83C33284BC6F8703304F55D
:1057A000C640274BC6F874332649383045F068FBAD
:1057B000254BC6F8383320460123C6F8987386F87F
:1057C000A07385F888361FB0BDEC028BBDE8F08F62
:1057D000954F0108994F01080000FFFF309000200D
:1057E0002C4C0D081C9A002078B30D089D4F010821
:1057F000A14F0108A54F0108A94F0108AD4F0108AD
:10580000B14F010844D20C08F0490E082CA2002028
:1058100004D20C0800D60C08747C0C084C7C0C08D4
:10582000FC9000204CC70C08FA900020B890002093
:1058300020D20C08B47C0C087CD20C089CE70C0825
:10584000F4E70C08F4A60D0874E90C0810B581F013
:105850000BFD064C064B18602046FFF7A1FC2046C6
:10586000044A0549BDE81040ABF036B9102C0020C1
:105870000C2C002088F20020B54F01080069C0F30D
:10588000401070470F299DBF302303FB01005030AB
:1058900000207047014B93F9E9047047104C002039
:1058A000014BD3F82C0F7047104C002008B503684B
:1058B0009B68984730B9044B93F87200B0FA80F0B7
:1058C000400908BD0020FCE7107C002008B5044812
:1058D00007F036F810B9034B93F86C0008BD00BF11
:1058E000102C0020107C0020022A10B50C4605D197
:1058F000BDE810400848352208F018BF074B986DE6
:1059000003685B689847A04205D15BF0C9F9BDE820
:1059100010405BF04FB910BD102C0020107C00200F
:10592000012910B50C4614D0022907D0D1B90E4B6D
:10593000C3F8981359F0C0FC0C4A05E00A4BC3F8B1
:10594000981359F0B9FC0A4ABDE81040062152F0FC
:10595000DBBD59F0B1FC074A062152F0D5FD024BE0
:10596000C3F8984310BD00BF108C0020BFD30C08B3
:1059700094D30C08A8D30C08012903D0022914BF22
:1059800000210221014BC3F8AC1E7047104C0020CF
:10599000012902D0022900D011B9024BC3F89C138F
:1059A000704700BF108C0020622910B400F388807B
:1059B00047291ADC402900F0978008DC162951DCC1
:1059C000032904DD504B01248C40234053B95DF87A
:1059D000044B5BF0DBBFA1F196040123A3404B4CC9
:1059E0002342F4D05DF8044B7047A1F148031A2B11
:1059F000EDD801A454F823F0E5590108CF59010866
:105A0000CF590108CF590108CF590108E5590108BC
:105A1000CF590108CF590108CF590108CF590108C2
:105A2000CF590108CF590108CF590108CF590108B2
:105A3000DF5A0108DF5A0108DF5A0108E559010859
:105A4000CF590108DF5A0108E5590108CF5901086B
:105A5000CF590108E5590108E5590108CF59010856
:105A6000E5590108A1F12703112BB0D8112BAED8AD
:105A700001A454F823F000BFE5590108CF590108EB
:105A8000CF590108CF590108E5590108CF5901083C
:105A9000CF590108CF590108CF590108CF59010842
:105AA000CF590108CF590108E5590108E559010806
:105AB000CF590108CF590108E5590108E5590108F6
:105AC000B02904DC952986DC6B2980D18AE7B529C9
:105AD00088D0A1F1D003022B3FF679AF82E75DF8C1
:105AE000044B00235BF024BF094B012283F894236D
:105AF000A3F58043D3F8280F00283FF473AF5DF877
:105B0000044B64215BF012B910004100A100800435
:105B1000108C002038B50B466B2B0446114600F361
:105B2000AA80472B14DC382B00F38E80262B5FDCF9
:105B3000102B00F0CD80162B00F02181042B00F0FB
:105B4000DE800A4620461946BDE838405BF080BC3E
:105B5000A3F14802232AF4D801A050F822F000BF94
:105B6000D95C0108435B0108435B0108435B010802
:105B7000435B0108035D0108435B0108435B0108C7
:105B8000435B0108435B0108435B0108435B010879
:105B9000435B0108435B0108175D0108555D01087F
:105BA0000F5D0108775D0108435B01085D5D010839
:105BB000095D0108435B0108435B0108BF5C010804
:105BC0008B5D0108435B0108E75C0108435B01084A
:105BD000435B0108435B0108435B0108435B010829
:105BE000435B0108435B0108435B0108B15D0108A9
:105BF000A3F12702112AA4D801A050F822F000BF77
:105C0000BF5C0108435B0108435B0108435B01087B
:105C1000C35C0108435B0108435B0108435B010867
:105C2000435B0108435B0108435B0108435B0108D8
:105C3000F95C0108E15C0108435B0108435B010872
:105C4000F35C0108ED5C0108402B7FF47AAF931EF2
:105C50005942674C594184F8931359F02DFB654A1A
:105C600094F89313644B002908BF1346634A062136
:105C700052F04AFC23E09D2B00F08E800BDC962B2B
:105C800000F088809B2B7FF45CAF022A17D15C4820
:105C900006F064FD13E0B52B00F099800ADCAD2B13
:105CA0007FF44FAF022A0AD19FED560A5448FCF701
:105CB0003FFA04E0A3F1D002022A3FF642AF0124EA
:105CC00053E08A1E504B5142514183F86510F6E76C
:105CD0000A21FFF709FEF2E70A4601212046F8E70C
:105CE0000A460421FAE70A460321F7E70A460C218F
:105CF000F4E70A460F21F1E70A460021EEE70B21FF
:105D0000E7E70A460D21E9E70A460521E6E72046CE
:105D1000FFF732FED3E7364CC9B102290CD101237B
:105D200084F89033A4F58053986D03685B6A9847B4
:105D300010B1334800F07EFD59F0BEFA334A94F8B2
:105D40009013334B002908BF1346324A8FE784F87B
:105D50009013E7E72046FFF7E3FDB0E7012431B1F8
:105D6000022902D12C4B83F88C42204638BD2A4BA5
:105D700083F88C12F9E72046FFF70AFE9FE7022A14
:105D80009DD11F4806F080FB99E75AF089FF5AF031
:105D900011FF94E707219CE701242AB1022AE4D1EC
:105DA000134B83F89243E0E7114B83F89223DCE72F
:105DB000022917D1144DA86D0368DB6B9847044680
:105DC00048B10121A5F5A04002F0CAFCCDE7134877
:105DD0007FF0FCFF73E759F06FFA114A042152F08B
:105DE00093FB6CE70648002102F0BAFC67E700BFAE
:105DF000108C0020D4D30C0877BB0C08DCD30C0823
:105E0000102C002000000000107C0020D3A60C08FD
:105E1000ACE00C08ECD30C08104C0020A87B002050
:105E2000FFD30C0810B5074CA06D03689B6B984717
:105E300028B9A06DA03C001B18BF012010BD022096
:105E4000FCE700BF107C002008B5022103205CF0B5
:105E5000D3FD022108465CF0CFFD012104205CF057
:105E6000CBFD022115205CF0C7FD132002215CF060
:105E7000C3FD124806F0CEFFA8B1002146205CF019
:105E8000BBFD002149205CF0B7FD00214A205CF0F9
:105E9000B3FD002101205CF0AFFD0021BDE808400A
:105EA00008465CF0A9BD012146205CF0A5FD01215A
:105EB00049205CF0A1FD0121E8E700BF102C002083
:105EC00002490348052208F05DBB00BF347B002077
:105ED000102C002038B5304B01241C7090F90A308A
:105EE0002B2B0CD12D487DF0E1FE2D4808F0D6F883
:105EF000BDE838402B4801220921FBF743BD284D5E
:105F00009FED290AD5ED460A642103205CF03EFB93
:105F1000D5ED460A9FED240A642102205CF036FB91
:105F20009FED220A03205CF03BFA9FED200A02203D
:105F30005CF036FA9FED1E0A04205CF031FA9FED0A
:105F40001C0A15205CF02CFA13209FED190A5CF056
:105F500027FA284606F05EFFA0B1002146205CF03B
:105F600079FD002149205CF075FD00214A205CF09C
:105F700071FD002101205CF06DFD002108465CF000
:105F800069FDB2E7214646205CF064FD21464920C8
:105F90005CF060FD2146E9E7E4940020C48C002019
:105FA000102C0020FC8E0020000000000000C842E1
:105FB00000A08C4500F5A040806D03681B6C18475D
:105FC00000F5145393ED027A00F5C040B5EEC07AA7
:105FD000F1EE10FA03F108035DBFD0F8C831DFED30
:105FE000086AD3ED017AD0F8E0015FBFF8EEE77AF6
:105FF000E7EE267AFDEEE77A17EE900A704700BFCB
:106000000000C84200F5005090F8480528B141F062
:106010000101084214BF01200020704713B5034658
:10602000FFF7F0FF58B103F5005191F8480FC00792
:1060300005D501F6647191ED000A02B010BD03F5BB
:10604000C04412B994ED860AF7E794F8B020022A0A
:10605000F8D103F5B040012201A918304CF078FACC
:106060000028EFD09DED010AE7E7000000F5C043EE
:1060700093F80422FFF7D2BF10B54B68516800F5C2
:10608000C0448B42D8BF0A46D4F8FC01CCBF1A46A4
:10609000194623F079FCC4F8FC0110BD10B5044684
:1060A0004E4867F007FA10F0080217BF4C4BDFEDBF
:1060B0004D7A93EDC77AD3EDC97A1FBF77EE877A11
:1060C0009FED497A012267EE877A10F0010317BF2E
:1060D000434B9FED447AD3EDC96A93EDC67A1CBF5A
:1060E00037EE667ADFED406A04F5145118BF27EEEB
:1060F000267AD1ED046AF5EEC06A18BF0123F1EEED
:1061000010FA34DD394A9FED386AD2ED006A66EE46
:10611000866A0122F4EE676AF1EE10FA58BFF0EEDB
:10612000667A04F5C04090F8041229B373B1D0ED3B
:10613000826AF8EEE66AF4EEC76AF1EE10FA58BF2A
:10614000F0EE476AFDEEE66AC0ED826A9AB190ED24
:10615000827AB8EEC77AB4EEE77AF1EE10FAD8BFD9
:10616000B0EE677ABDEEC77A80ED827A03E0002A4E
:10617000D7D1002BD5D110BDB3B1D0F8C831D3EDF4
:10618000016AF8EEE66A76EE876A90ED7F7AB8EEFD
:10619000C77AF4EEC76AF1EE10FAD8BFB0EE667AAD
:1061A000BDEEC77A80ED7F7A002AE4D0D0F8C831FE
:1061B00093ED017AB8EEC77A77EE277A90ED7F7A81
:1061C000B8EEC77AF4EEC77AF1EE10FA58BFB0EE27
:1061D000677ABDEEC77A80ED7F7ACCE7204F00204A
:1061E000104C0020000000000000C8422051002098
:1061F00000F5C0400023C0F80032704773B5164662
:10620000044600236A463046009311F035FB48B13E
:10621000DDED007A9FED277A67EE877AFDEEE77A6B
:1062200017EE900A04F5C045C5F8000233785B0705
:1062300018D595F80432ABB104F5B040012201A99C
:1062400018304CF085F968B1D5ED827ADDED016A40
:106250009FED187AF8EEE77AE6EEC77AFDEEE77A78
:10626000C5ED807A04F5A043D3F8DC36042B1FD0AB
:1062700004F50054B4F94225002A16DDD5F80032A1
:106280009FED0D7A83EAE371A1EBE37107EE901ABB
:10629000F8EEE77A67EE877A07EE102AB8EEC77A4B
:1062A000F4EEC77AF1EE10FA02D50023C5F80032F9
:1062B00002B070BD0000C8420AD7233C37B50B7846
:1062C0005A0704460D461DD500F5B040012201A92C
:1062D00018304CF03DF9A8B1D5ED017A2B78DFEDFF
:1062E0001B6AF8EEE77ADB0767EEA67A19D59DED13
:1062F000017AB4EEE77AF1EE10FACCBF012000206B
:1063000003B030BD2B78D5ED017A13F0010FF8EE14
:10631000E77A04F5C0440FD194ED787AB8EEC77AE5
:10632000E7E704F5C044D4F8C83193ED017AB8EE3C
:10633000C77AE7EE667ADAE7D4F8C83193ED017AE6
:10634000B8EEC77A77EE877AE6E700BF0AD7233C34
:1063500000F5005300F59E42B3F9F23400EE103A16
:1063600000F5A0432432996D9142B8EEC00A0CD1D9
:10637000D3F8DC26042A02D093F889362BB100F535
:10638000C040D0ED2D7A30EE270A704710B5044694
:1063900004F5C044FFF7DCFFD4ED787A9FED057A71
:1063A000F8EEE77AE0EE477AFDEEE77A17EE900A2C
:1063B00010BD00BF0000C84237B500F5C045044617
:1063C00095F80432DBB100F5B040012201A9183084
:1063D0004CF0BEF898B1D5ED827AD5ED836A9FED89
:1063E0000B7AF8EEE77AE6EE877ADDED016AE6EE03
:1063F000C77AFDEEE77A17EE900A03B030BD20466B
:10640000FFF7C4FFD5F8FC31181AF6E70000C842C0
:1064100010B5044604F5C044FFF79AFFD4ED867A20
:1064200037EEC00ADFED047A20EE270AFDEEC07ACF
:1064300017EE900A10BD00BF0000C8422DE9F041E0
:1064400000F5C34700F5C3455C376C350446294663
:10645000384611F085FC04F5A04804F5C34608F55C
:10646000CE634C362A46314683ED000A384611F099
:10647000ADFB08F27463DFED220A83ED000AB7EE8C
:10648000001A762023F0E0F904F53F5383ED750AF6
:106490002046FBF7F5FDD8F8580003685B6898477D
:1064A0000B280DD008D80A2811D004F5C0440023C9
:1064B000C4F80032BDE8F0810E38C0B20128F4D82B
:1064C00029462046FFF7FAFE0028EED011E02946C3
:1064D0002046FFF7F3FE30B90A484FF48041FCF73D
:1064E0002BF80028E1D12046FFF792FFB0F5FA6FB4
:1064F000E6DD2A4631462046BDE8F041FFF77EBE84
:1065000000000000102C002010B52DED028B00F5CE
:10651000C043D3ED7C7A93F8EC31DFED1D8AB8EE01
:10652000E78ADA0728EE288A82B0044609D400F503
:10653000805202F5D662D2ED007AF8EEE77AA7EE45
:10654000E88A5B070FD504F5B040012201A9183095
:106550004BF0FEFF38B19DED010A30EE480A02B063
:10656000BDEC028B10BD204604F58054FFF70EFFF2
:1065700004F5D66393ED000A07EE900AB8EEC00A60
:10658000F8EEE77A28EEC00AA7EEA80AE5E700BF12
:106590000AD7233C70B52DED028B00F5A04600F51F
:1065A0009E43B26D9A4204464DD100F58053D3F814
:1065B000405600F50053B3F94035002B66DD04F575
:1065C000C25292ED017AF7EE007AB4EEE77AF1EE7C
:1065D00010FA5BD404F53F52D2ED0E7AF6EE006A63
:1065E00067EEA67A87EE871AB5EEC01AF1EE10FABA
:1065F0004CD907EE905A9FED288AB8EEE70A07EECD
:10660000903A04F5B04004F5C044F8EEE70A20EEF5
:10661000080A18304CF0A8F8D4F800329FED1F1A81
:10662000DFED1F0A002BBCBF07EE903AF8EEE77AC9
:106630004FF42970B8BFA7EE880ABDEC028BBDE805
:10664000704023F001B905F0BBFDF8B904F54053E3
:1066500006F5CE66D3F8080903681B69984704F568
:106660000053DFED0F0AB3F9403596ED000A01EE55
:10667000103A0546B8EEC11A40F27F2023F0E4F844
:10668000BDEEC00A10EE103A1BB296E7BDEC028BCD
:106690009FED030A70BD00BF0AD7233C00007A4477
:1066A0000000000010B5044681F0D8FA04F500534C
:1066B000D3F85C2F801A41F2883290420FD8022121
:1066C0002046FFF79FFC50B104F5A044D4F8DC2627
:1066D000042A04D103F5756393ED000A10BD9FED04
:1066E000010AFBE70000000030B52DED028B00F53C
:1066F000C045DFED278A95F8043283B004465BB3CA
:10670000D5ED827A9FED230AF8EEE77A00F5B040E6
:1067100027EE800A012201A918304BF051FFD8B1B1
:106720002046FFF737FFDDED017A85ED830A37EE6E
:10673000800A20468DED010AFFF7B4FFDDED017AF6
:1067400030EE270A20EE280ABDEEC00A10EE100A2D
:1067500003B0BDEC028B30BDD5F8C821D5F8FC31B3
:1067600052689B1A08EE103A2046FFF7F1FDB8EE8A
:10677000C88A2046A0EE288AFFF794FFBDEEC88A9B
:10678000B8EEC88AA0EE288ABDEEC80ADEE700BFD0
:106790000000C8420AD7233C10B500F5A0430446C8
:1067A000986D03685B6A984718B104F5C04494F883
:1067B000900310BD38B500F5C0440D46D4F8FC3147
:1067C0000B44C4F8FC3194F804323BB1FFF7E4FF0A
:1067D00020B9D4F808122944C4F8081238BD0000C2
:1067E00030B500F50050D0F83C25D3070FD4094B45
:1067F00008201D785C688D4204D1224214BF01201C
:10680000002030BD013803F10803F2D1F9E701207F
:10681000F7E700BF50D60C0810B500F5A0430446BA
:10682000986D03685B68984701462046BDE81040B4
:10683000FFF7D6BF37B500F5C0440546D4F8E031C0
:10684000C4F8FC310023C4F80032FFF7E5FFD0B1F3
:1068500005F5B040012201A918304BF079FE90B146
:106860002846FFF799FF70B9DDED017A9FED087AB0
:1068700067EE877A0123FDEEE77A84F80432C4EDEF
:10688000827A03B030BD002384F80432F9E700BFF8
:106890000000C84238B504460D46FFF7BDFF30B1D1
:1068A0000321284610F0C4FF80F00103D8B204F59C
:1068B000C04484F8050238BD73B500F5C0444A6889
:1068C000C4F8FC210B780D46D90741BFD4F8C83174
:1068D0005B689B18C4F8FC3194F80532064623B176
:1068E00000F5C3416C31FFF7D5FF2B785B070FD55F
:1068F00006F5B040012201A918304BF029FE38B14D
:10690000012384F804326B68C4F8083202B070BD09
:10691000002384F80432F9E7F0B52DED028B04462C
:1069200083B004F5C0450E468DED010AFFF7C4FFA4
:10693000DFED350A9DED010A40F24310B7EE001A73
:1069400022F082FFD5F800325B4207EE903AF8EE73
:10695000E77A04F5155767EE807A2046FDEEE77A70
:10696000B0EE408A17EE901AFFF724FFD7ED017AB8
:10697000F5EEC07AF1EE10FA07F104073FDDD5F825
:106980000032002B3BDD2046FFF716FD07EE900A94
:10699000DFED1E6AB8EEE77AD7ED007A67EEA67AE9
:1069A000B4EEE77AF1EE10FA29D531462046FFF72A
:1069B00083FF04F5C34132465C312046FFF71EFCDD
:1069C000D5F800325B4207EE903AF8EEE77A2046BF
:1069D00067EE887AFDEEE77A17EE901AFFF7EAFE87
:1069E000B5EEC08AF1EE10FA09DDD5ED807AB8EE89
:1069F000E77AC7EE087AFDEEE77AC5ED807A03B054
:106A0000BDEC028BF0BD00BF000000000000C8C25A
:106A1000F0B500F5C04487B094F8EC3103F00503FD
:106A2000052B07460BD04CF013FE4FF4AE724FF41B
:106A300080114CF0C5FD0025284607B0F0BD1E486A
:106A40006A46032110F004FF0028F4D01B4801AA75
:106A5000032110F0FDFE05460028ECD0184BDFEDB9
:106A6000190A93ED000A40F26D10B7EE001A22F0F9
:106A7000EBFE04F5F6730FCBB0EE401A02AEDFED7D
:106A8000111ADDED010A9DED000AB7EE002A86E835
:106A90000F0022F00BFEDFED0C7A20EE270A3046C5
:106AA000FDEEC07A032217EE901A10F0FDFD31467C
:106AB0003846FFF701FFBFE7DC8D0020FC8D00208A
:106AC00084820020000000000000C842F7B50E4696
:106AD00002210446FFF796FA70B304F5A045D5F8F5
:106AE000DC36042B28D12046FFF796FE20B304F5B0
:106AF000B047183704F5C34101236A465C31384674
:106B00004BF010FCC0B104F5C341012301AA6C3164
:106B100038464BF007FC78B19DED017ADDED007A47
:106B200077EEC77A96ED007A37EE277A05F294650C
:106B300086ED007AC5ED007A03B0F0BDF0B52DED1D
:106B4000048B00F5005489B000F5736694F8121FA9
:106B500003910546304645F03FFC03990746304611
:106B600045F04CFC042F0399B0EE408A1FD100235E
:106B700005A88DED050A0693079325F035FA05A9BA
:106B800005F5BB5023F03CF9DFED9A7A8DED050A4F
:106B9000B4EEE71AF1EE10FACDED060A8DED071A04
:106BA00005DB05F5805393F8BC36DF070CD494F869
:106BB000483F002262F3000384F8602F84F8483FC6
:106BC00009B0BDEC048BF0BD94F8483F98075CBF5A
:106BD00043F0020384F8483F04F6647758BF04F694
:106BE0004C7305F53D5158BF83ED008A243187ED84
:106BF000001A2846FFF76AFF94F8603F092B00F25D
:106C0000898004F66873D3ED000A9FED7B9AB0EE9D
:106C1000480A22F007FD00BB04F64C7394F8121FDB
:106C2000D3ED008A304645F007FC07EE900A9FED51
:106C3000737AF8EEE77A78EEC88A67EE877AF0EE34
:106C4000E88A67EE897AF4EEE78AF1EE10FAC2BFBD
:106C500094F8603F013384F8603F04F6687394F859
:106C6000121FD3ED008A304645F0E6FB07EE900A8E
:106C7000F8EEE77A9FED627A67EE897A78EEC88A55
:106C800067EE877AF0EEE88AF4EEE78AF1EE10FA22
:106C900002DD002384F8603F04F6687383ED008A08
:106CA00094F8483FDA078BD5284605F5C046FFF72C
:106CB0002BFC04F6647393ED008A96F8043230EEF0
:106CC000488A002B4CD005F5B040012205A91830A8
:106CD0004BF03EFC002849D180F0C0FFD4F85C2F77
:106CE00041F28831821A8A42034604F5756204F63D
:106CF000547144D982ED008A284681ED008A022130
:106D0000FFF780F918B1D6F8C020C6F8BC20C4F847
:106D10005C3F55E794F8483F43F00103590784F876
:106D2000483FB9D405F5A042D2F8DC26042AB3D1F5
:106D300002212846FFF766F90028ADD043F004038E
:106D400084F8483F3868F9F7DFFB05F55B562036D5
:106D5000CDE900012B4A0621304651F0D5FB9BE7D7
:106D60002846FFF759FD0028ADD1B5E704F6647356
:106D700093ED000A9DED058A38EE408AACE79FED61
:106D8000200A92ED007ADFED207A28EE008AA7EE45
:106D9000278A82ED008AC4F85C0FD1ED007A38EEC4
:106DA000678AF3EE0E7AB0EEC88AB4EEE78AF1EEA7
:106DB00010FA7FF705AF94F8483F5B070ED504F64D
:106DC000647405F55B562068F9F79EFB2036CDE923
:106DD00000010E4A0621304651F096FB05F53D5064
:106DE00024220021083009B0BDEC048BBDE8F0403E
:106DF000ACF0B4BB000000340AD7233CCDCC4C3DF2
:106E0000CDCC4C3E10D60C08CDCC4C3F2DD60C082A
:106E100038B52DED028B0D460446FFF775FB0023B8
:106E200020462B70B0EE408AFFF73CFC0221204642
:106E300038EE400AFFF7E6F828B104F5005494F85C
:106E4000480F00F00100BDEC028B287038BD000037
:106E500070B50B7803F00503042B05460C46164667
:106E600015D105F5C0454CF0F3FBB2B24FF48011DB
:106E70004CF0A6FBD5F8C821636852689B1A13F53D
:106E8000FA7FC8BF6360237843F00103237070BDAD
:106E9000F8B500F5805300F5A047D3F8B066D7F8F1
:106EA0009856B542044619D00E4A1268D26A92F832
:106EB0009C209AB100F5C341751B25226C31FFF768
:106EC000C7FF07EE905AB8EEE70ADFED077A04F540
:106ED0003F5020EE270A10307CF07AFAC7F8986607
:106EE000F8BD00BF0C2C00200AD7233CF8B500F5F4
:106EF000A04C00F5C0449CF88BE605460F4604F50F
:106F0000E676BEF1000F53D004F5F6730FCB86E89A
:106F10000F0001238CF88C3697E80F0004F5F67605
:106F200086E80F00D4F8F43105F5C3466C3693B902
:106F3000D4F8F8317BB9D4F8E431D4F8F021C4F8AE
:106F4000F431D4F8E831C4F8F83122B9D4F8E011BA
:106F5000304610F0A9FB314628222846FFF778FF7B
:106F600094F8EC1111F0040102D1304610F060FCED
:106F700005F5C34105F5C34032464C315C3010F095
:106F80005BFE38B104F5E67604F5EE7494E80F0084
:106F900086E80F00284604F075FD2846FFF74EFAF4
:106FA000284605F0D3F82846BDE8F840FFF702B8B8
:106FB00004F5EE730FCB86E80F0001238CF88B36B7
:106FC0008CF88CE6A8E70000F8B500F500530446FD
:106FD000B3F99A34002B0D4635DB0B7813F0020F12
:106FE00014BF4FF0FF33012304F5C04606F5E677E2
:106FF00086F8A43106F5EE730FCB87E80F0095E80D
:107000000F0006F5F67787E80F0004F5C341572215
:107010006C312046FFF71CFF2046FFF70BFC204693
:10702000FFF70CFA204605F091F804F5A042002382
:1070300082F88C36C6F8A83182F891362046BDE831
:10704000F84004F01FBD4FF0FF33CDE72DE9F043CA
:10705000354B1B6885B00546D86AFAF765FA0028F3
:107060005FD105F5005393F9C03E5A1C52D0002B56
:1070700005F58C6611DD95F87124242107EE903A10
:1070800001FB026292ED0B7AF8EEE77AB0EEC77A76
:10709000B4EEE77AF1EE10FA3CDC05F5805305F525
:1070A000A25793F8BC3613F0010429D0C3F340086B
:1070B0009B0732D495F8141495F858444FF0B00952
:1070C00009FB015191F8F1314CBB022B18D96846EC
:1070D00010F0E4FA694638460AF02EFE044678B10C
:1070E00095F8143409FB03534246D3F8001268465E
:1070F00010F0DAFA0BF0E2F869460AF00BFD0446EC
:1071000030460DF0A3FB38460AF022FC2846FBF778
:10711000E7F9204605B0BDE8F0830024F0E74446D7
:10712000EEE70020F6E700BF0C2C002038B50C4B32
:107130001B680546D86A0C46FAF7F6F910B1002428
:10714000204638BD0BF0BAF821460AF0E3FC0446AD
:107150000028F4D005F5AE4025F034FDF0E700BF7F
:107160000C2C0020F0B500F5A04300F5C04600222D
:1071700083F88B2683F88C2606F5EE73044600EE22
:10718000101A0FCB87B006F5E67585E80F0002AD43
:1071900004F5C342B8EEC00A284617495C3244F0F1
:1071A000D9FE95E80F0006F5F67787E80F0004F59D
:1071B000C34140F257126C3120460191FFF748FE5F
:1071C00001992046FFF766FB01992046FFF774FB03
:1071D00004F500532046B3F99A34002BB4BF4FF0A6
:1071E000FF33012386F8A431FFF728F9204607B0C2
:1071F000BDE8F04004F0AABFDC65002010B50349EB
:10720000044644F0A7FE204610BD00BFDC65002008
:10721000F8B500F5C04505F5EE7304460E460FCBF4
:1072200005F5E67787E80F0006F108012046FFF72D
:107230005DFEB38803EB830303EB83039B001BB268
:1072400004F5A042002BD8BF4FF4C873A2F88636CD
:10725000D5F8C831D5F8F0115868091AC2F858168F
:1072600099680A31C5F8F411DB680A33C5F8F831BA
:107270000023C2F86C3682F8883682F89C36C2F851
:107280005C3602F5CA63002119604FF0FF33C2F883
:10729000483694F8711404F58C63242000FB013304
:1072A00004F5AD42DB6A1360F8BD000070B50E4610
:1072B00008310446FFF71AFEB38804F5A04543B32E
:1072C000642213FB02F3C5F85836B5F98636002B55
:1072D000D8BF4FF47A7304F53D50D8BFA5F8863671
:1072E000242200210830ACF039F904F5C04304F53C
:1072F000C14093ED860A314634307CF0D7FBD5F897
:10730000DC36072B0CD120460421BDE87040FAF78B
:1073100067BED5F85836002BD7DC40F6B833D2E735
:1073200070BD00000B7A00F5C04013F0020F14BFCF
:107330004FF0FF33012380F8A43170477FB501F18E
:10734000080305460E460FCB6C4684E80F0005F592
:10735000C3415C31204610F00BFB21462846FFF765
:10736000C5FD31462846FFF7DDFF04B070BD0000C3
:107370007FB501F1080304460E460FCB6D4685E844
:107380000F0004F5C3415C31284610F0F1FA29469C
:107390002046FFF7ABFD20463146FFF7C3FF3379A8
:1073A00007EE903A337E9B0748BF9FED0B7AF8EECD
:1073B000677A04F5C04448BF67EE877A9FED077A85
:1073C00067EE877A0123FCEEE77AC4F8BC31C4ED9E
:1073D000677A04B070BD00BF0000803B00A00C477E
:1073E0007FB501F1080304460E460FCB6D4685E8D4
:1073F0000F0004F5C3415C31284610F0B9FA294664
:107400002046FFF773FD20463146FFF78BFFB38818
:1074100004F5C0444FF47A725343C4F8B4310123E5
:10742000C4F8BC3104B070BD2DE9F34100F5C3458B
:1074300004466C3500F5C3400E464C30294610F02A
:1074400057FA04F5A047D0B94FF0FF33C7F84836D4
:1074500006F10807384610F051F9032802463CD1DE
:10746000F168284610F020F9B28804F5C0432046A0
:10747000C3F8BC2102B0BDE8F041FEF7B9BE19F077
:10748000FBFFFAF747FB012812D94FF0FF33C7F88B
:10749000483619F0F1FF90F8F432DFED150AB0220A
:1074A00002FB030090ED3C0A284610F0CFFCCFE72A
:1074B00004F58058D8F8400622F09AF904F5B25342
:1074C000C7F84806D3ED007A9FED0A0ADFED080AF7
:1074D000F8EEE77A27EE800AE6E701AA00213846AF
:1074E00010F018F90028BFD001990022B9E700BFB9
:1074F00000007A440AD7233C7FB501F10803044613
:107500000E460FCB6D4685E80F0004F5C3415C3194
:10751000284610F02DFA29462046FFF7E7FC2046C2
:107520003146FFF7FFFE04F5C0440023C4F8BC3128
:1075300004B070BD37B504460D4680F08FFBE060A7
:10754000D5ED027AF5EEC07AF1EE10FA15DD9FED79
:10755000127A67EE877AFCEEE77AC4ED027A57F08A
:10756000ABFEA2684FF47A73B2FBF3F30B4A062129
:1075700003B0BDE8304050F0C7BF65F0E9FD00231F
:10758000009395F90D2095F90E3095F90C1065F0E2
:107590007BFDA060E3E700BF00007A4490D60C08B2
:1075A0002DE9F0432DED028B85B004460AF086FEEE
:1075B00009F0B4FF04F5805304F5A04693F8383978
:1075C0000BB9002877D0D6F84836013373D1D6F8F6
:1075D0006C36002B4BD080F041FBD6F86C36C01ACD
:1075E000B0F5FA6F67D394F81424DFED607A9FED5D
:1075F000608A4FF0B00808FB024292ED840A20EE48
:10760000270A22F00DF906F5CA69D9ED007A30EEA5
:10761000670A22F005F9DFED577A20EE080A04F533
:107620005B5720EE270A22F0A3F8FDEEC07A203740
:1076300017EE905AC6F84856D9ED007A67EE887A68
:1076400017EE900AF8F760FFCDE9020194F81434C0
:1076500008FB0343D3F80C02F8F756FF464ACDE97E
:1076600000012B460621384650F04EFF23E004F57A
:107670009070FAF74FFA02281DD994F81434B0220A
:1076800002FB034393ED837AF1EE047AB4EEE77ADA
:10769000F1EE10FA0FDD394B1B68D86A0368DB691D
:1076A0009847012803D080F0D9FAC6F86C06D6F8BE
:1076B0006C36002B8FD104F54053D6F84816D3F81A
:1076C00008094A1C036847D01B6B98472C4807F0F1
:1076D0007BFD18B104F5AE4027F0F6FC2046FEF71E
:1076E00097FED6F858368342054638DA07EE905AA8
:1076F0009FED247AF8EEE77A04F55B5767EE877A18
:10770000203717EE900AF8F7FFFE1F4ACDE9000177
:107710003846062150F0F8FE04F5C0444FF0FF3320
:107720000125C6F8483686F8885604F5EE730FCB67
:1077300004F5E67704F5F67487E80F0084E80F0097
:10774000124865F081FE002386F88B36284605B086
:10775000BDEC028BBDE8F0835B6B9847B6E7084849
:1077600007F012FD0028C1D1F1E700BF35FA8E3CC9
:10777000E02E65420000C842A0D60C080C2C002068
:10778000102C00200AD7233CC4D60C08204F002020
:107790002DE9F04F00F5A0492DED028B4FF0FF339E
:1077A00000F5C04AC9F848360AF5F6730F46064692
:1077B0000FCBBC8897F8048089B004AD240A85E813
:1077C0000F001FD006F5C3474C372946384610F046
:1077D000C7FA29463846B0EE408A10F091F9DFED3D
:1077E000577AB4EEE78AF1EE10FA0BDBE3B200EE63
:1077F000903ADFED537AF8EE600A20EE270A284629
:1078000010F024FB06F5405B99F88C26DBF808099C
:107810009FED4C0A036806F5C3479B6A5C3732B399
:1078200006F5C3412A464C31984706F50051B1F997
:10783000CA34002B1EDD07EE903A09F5CE62F8EE51
:10784000E77A92ED007AB4EEE77AF1EE10FA11DD04
:1078500006F5C3412A464C31384610F0EDF900BB1D
:107860000024204609B0BDEC028BBDE8F08F2A460B
:107870003946D9E7B8F1000F1DD1002C3DD1B1F93F
:10788000C824DBF8080900EE102A026809F26463D4
:10789000126AD3ED000AB8EEC00A9047B0EE408AF3
:1078A0000DE0002CDCD10AF5EE730FCB0AF5E6757E
:1078B00085E80F00D5E707EE908AB8EE678A29467B
:1078C000384610F04DFAB4EEC08AF1EE10FA17DB2C
:1078D000B9F83C3703932946384610F041FABCEE1C
:1078E000C00A06F55B50039B174A8DED000A06217E
:1078F000203050F009FE0124B3E79FED128ADEE745
:1079000006F5C3412A464C31384610F095F9044635
:107910000028A5D0B9F83C3703932946384610F023
:107920001FFABCEEC00A06F55B50039B074A8DEDBB
:10793000000A0621203050F0E7FD92E700000034F5
:10794000E02E654200000000E0D60C08FED60C08D0
:1079500038B500F5005500F5C043B5F9CC14002941
:10796000ACBF01224FF0FF320029B8BF49420446A4
:1079700083F8A42189B204F007FD04F5AC4393ED2C
:107980001C7AB5F9C834002BCABF07EE903ADFED78
:107990000E7AF8EEE77AFCEEE77AF8EE677AB4EE64
:1079A000E77AF1EE10FA08D804F55B502030074A68
:1079B000062150F0A9FD012038BD204604F000FC4E
:1079C0000028F1D1F8E700BF000000001CD70C0828
:1079D000F8B500F5C34600F5C3454C366C35044692
:1079E000294630460FF084FF04F5405750B304F5A4
:1079F000A043D3F848164B1C24D0D7F808090368D5
:107A00001B6B984704F5C045D5F8BC31012B47D016
:107A1000D5F8BC31022B06D12046FEF7B7FCD5F8CD
:107A2000F031984243DD2046FEF7B0FCD5F8F03146
:107A3000C01A0028B8BF4042B0F5FA7FCCBF002082
:107A4000012035E004F5C34029465C3010F088F988
:107A5000DFED187AB4EEE70AF1EE10FA16D53046EB
:107A6000294610F04DF89FED147ADFED140AF6EE7A
:107A7000007AE0EE077A28469FED110AFDEEE77ADC
:107A8000F8EEE77A27EE800A10F0E0F9D7F8080957
:107A90009FED0C0A03682A469B6A31469847B1E776
:107AA0002046FEF773FCD5F8F0319842B0DB012098
:107AB000F8BD00BF00004843A00CB345000096434A
:107AC0000AD7233C0000000073B5374CD1ED026AA1
:107AD000D4ED787A9FED357AF8EEE77A0546D7EE61
:107AE000876A0E46F5EEC06AF1EE10FA08DD57F02F
:107AF000E3FB2F4A062150F007FD012002B070BDC4
:107B0000D1ED037AF5EEC07AA4F69814F1EE10FAEE
:107B100094ED006A12DDF4EEC67AF1EE10FA0DD59E
:107B200057F0CAFB05462068F8F7EEFC214ACDE97C
:107B300000010621284650F0E7FCDEE7DFED1E7A63
:107B4000337CB4EEE76AF1EE10FA54BFB0EE677A18
:107B5000B0EE467A0BB90020D0E7B5EEC06AF1EE80
:107B600010FA0CDC86EE876A03EB830307EE903A8B
:107B7000F8EEE77AF4EEC67AF1EE10FAEBD52C7C4B
:107B8000002CE8D180F06AF86B69C01A337C4FF49E
:107B90007A7253439842DED901232B7480F05EF849
:107BA00068612046AAE700BF108C00200AD7233C5A
:107BB00034D70C0845D70C080AD723BC38B505467E
:107BC00077F038FC76F0CAF9044640B980F046F800
:107BD000EB68C01AAB68984284BFAC6001242046B1
:107BE00038BD000038B504460D4680F037F804F57E
:107BF000C0439FED067AC3F8C001D5ED027A67EE67
:107C0000877AFDEEE77AC3ED6F7A38BD00007A44DB
:107C100010B5044680F022F804F5C043D3F8C02123
:107C2000801AD3F8BC2190424FF0000084BFC3F803
:107C3000BC01012010BD000000F5C04300F5AC41BF
:107C4000D3F8BC2191ED1C7A22EAE27207EE902A69
:107C5000F8EEE77A0020B4EEE77AF1EE10FA44BFCE
:107C6000C3F8BC010120704710B500F5005300F5C2
:107C7000C040B3F99A34002BB4BF4FF0FF33012357
:107C800080F8A43100F5F67400F5EE700FC884E8B2
:107C90000F0010BD38B504462DED028BF0EE408A82
:107CA000B0EE608A09B301295CD0B5EEC08AF1EE6E
:107CB00010FA67DDDFED347AB4EEE78AF1EE10FA00
:107CC00060D8FCEEC87A04F55B5017EE903A2F4A64
:107CD0000621203050F018FCFDEEC87A04F500545F
:107CE00017EE903A84F867343AE0F8EE000A21F093
:107CF00099FC40B104F5A0444FF0FF33C4F888303C
:107D0000BDEC028B38BD04F50053B3F9702407EEC7
:107D1000902AF8EEE77AF4EEE87AF1EE10FAC4D899
:107D2000B3F9723407EE903AF8EEE77AF4EEE87AB7
:107D3000F1EE10FAB9DBDFED147A154A68EEA77A96
:107D400004F5A043FDEEE77A04F55B50C3ED227A1B
:107D5000FCEEE87A062117EE903A203050F0D4FB82
:107D60000120CDE7FCEEC07A00F55B5017EE903AAB
:107D7000084A0621203004F5115450F0C5FBC4ED2B
:107D80000F8AEDE70020BBE70000C8428BD70C0844
:107D900064D70C0878D70C08D1F80D3000EE903A73
:107DA000D1F80930097A00EE103AFFF773BF0000EE
:107DB00070B58B88012B04460D4611D100F59076E5
:107DC0003046F9F7A7FE02280AD994F81414B02314
:107DD00003FB01612046DC31BDE87040FFF7A6B926
:107DE0000AF06CFA05F10801BDE8704009F092BE96
:107DF000F0B500F5A0460027A24B86F8917689B031
:107E0000044608460D4683F8057224F0EDFC48B39D
:107E1000012386F8883604F54053D3F8080903682F
:107E2000DB6B984704F5C04386F88F7603A8C3F848
:107E3000A8710FF033FCB6F83C174FF6FF73994268
:107E400008BF3946013101AA89B204F5AE4026F0D7
:107E5000BDFC28B1BDF80600A0F1150358425841F9
:107E600086F889066B885D2B00F0048133D81F2BC0
:107E70002AD80F2B01D800202BE0103B0F2BFAD86B
:107E800001A252F823F000BF7B7F0108917F010817
:107E90009B7F0108A57F0108B97F0108877F010842
:107EA000697F0108777E0108777E0108777E0108E7
:107EB000777E0108777E0108777E0108777E0108CA
:107EC000C97F0108AF7F0108532BD4D1012086F868
:107ED0008F0609B0F0BDBD2B18D8BB2B4BD8B22BE9
:107EE0007CD00CD8702B74D0722BC4D1D5ED027A13
:107EF000FDEEE77A04F5C044C4ED6F7A3BE0B32BA6
:107F0000B9D129462046FFF753FF34E0C33B9AB26C
:107F1000112AB0D8112BAED801A252F823F000BF1D
:107F200017800108777E010817800108777E010815
:107F3000777E0108777E010817800108777E0108A7
:107F4000777E0108777E010853800108777E01085B
:107F5000777E0108777E0108777E0108E77F0108B8
:107F6000777E010807800108002386F8C536294678
:107F70002046FFF74DF90120ABE705F10801204647
:107F8000FEF7B4FFF7E729462046FFF78FF9F2E73F
:107F900029462046FFF7D2F9EDE729462046FFF7AC
:107FA000E7F9E8E729462046FFF71AFAE3E729460A
:107FB0002046FFF7A1FADEE704F59E4129223C3175
:107FC000204606F0DFFAD6E729462046FFF72CFACE
:107FD000D1E729462046FFF705FECCE72946204693
:107FE000FFF7DAFEC7E7AB88012BC4D803F0010323
:107FF00086F88A3604F55B50AB88234A0621203088
:1080000050F082FAB7E7A988003918BF012120464D
:1080100000F0A6FBAFE704F5C446EB6804F5C044E6
:10802000683694F8E11273B92B6963B96B6953B977
:1080300030465CF029F804289DD194F8E1123046CE
:108040005CF02CF897E705F1080230465CF064F923
:1080500091E704F5C04304F5C44095ED041AD5ED4D
:10806000020A95ED030A93F8E112002268305CF0F1
:1080700037F880E704F59E4029462430FFF75AFA86
:1080800079E700BF108C00209CD70C0800F5A042B7
:1080900000F59E43926D24339A4201D1FFF7A8BEAA
:1080A0000120704710B500F5A04200F59E43926D87
:1080B00024339A4204460ED100F59E4108223C31F9
:1080C00006F060FA04F55B50034ABDE81040062153
:1080D000203050F019BA10BDACD70C0870B58EB076
:1080E00009AD044628460E460FF0D8FA04F5A04321
:1080F0004FF6FF72B3F83C37934208BF00230133B9
:1081000007AA99B204F5AE4026F060FBB0B104F5C1
:10811000C04416B10023C4F8A03195E80F0001AEA9
:1081200086E80F00D4F8F831009304F5F67494E86B
:108130000E00034802F098FD0EB070BD0120FBE771
:10814000547B002070B5054605F5C046002104F0BB
:108150001BF9D6F8A8417CB9284604F031F810B9CB
:108160000024204670BDD6F8A031012BF8DD7FF049
:1081700075FDC6F8A801F4E7D6F8BC1161B17FF02F
:108180006DFDD6F8A831C01AD6F8B4319842E7D9B7
:108190000023C6F8BC3101212846FFF79FFF0446A3
:1081A0000028DDD005F55B50054A0621203005F595
:1081B000A04550F0A9F9002385F89136D1E700BF1A
:1081C000D4D70C0838B50A468B88190A137EDB070A
:1081D00048BF01EB8101044648BF490004F0D4F8D0
:1081E00004F5A043002583F89156204603F0E8FFEC
:1081F00010B90025284638BD04F5C043D3F8BC119A
:1082000041B1D3E967128A42F3DD012AF1DDC3F8F7
:10821000BC5101212046FFF761FF05460028E8D048
:1082200004F55B50024A0621203050F06DF9E1E779
:10823000ECD70C0838B5054605F5C044898804F02C
:10824000A3F8D4F8BC3183BBD4F8A031002BB8BF5D
:108250005B42012B02DC0024204638BD94F8A521A6
:1082600094F8A63172B9002BF5D005F55B50D4F81F
:10827000E0216423062192FBF3F320300C4A50F0F6
:1082800043F901E0002BF0D10121C4F8BC112846CC
:10829000FFF724FF04460028DDD005F55B50054AB2
:1082A0000621203050F030F9D6E70021EFE700BF7B
:1082B00004D80C0822D80C082DE9F0474B881F2B56
:1082C0008AB004460A4631D80F2B07D804F55B5014
:1082D000984A0421203050F017F988E0A3F11001EA
:1082E0000F29F3D801A050F821F000BFFF83010847
:1082F000CD840108D9840108E784010801850108BB
:108300000D840108F3830108CD820108CD820108A4
:10831000CD820108CD820108CD820108CD820108FD
:10832000CD8201080D850108F3840108702B00F04F
:10833000FB800CD8532B00F0EF805D2BC6D100F5ED
:108340009E4024300AB0BDE8F047FFF737BCB32B9E
:1083500008D8B12B4BD8722BB8D10AB0BDE8F04782
:10836000FFF76ABCD42B3BD8BB2BAFD9A3F1BC021F
:10837000182AABD801A151F822F000BFEF83010801
:10838000EF830108CD820108CD820108CD8201086A
:10839000CD820108CD820108EF830108CD8201085A
:1083A000EF830108CD820108CD820108CD8201084A
:1083B000EF830108CD820108CD820108CD8201083A
:1083C000EF830108EF830108EF830108CD820108E4
:1083D000CD820108EF830108CD820108EF830108F7
:1083E000DF2B04D040F6B83293427FF46FAF012008
:1083F0002FE020460AB0BDE8F047FFF7D1B811469C
:1084000020460AB0BDE8F047FFF7C2B904F5A04521
:1084100004F5C146D5F8DC3604F5C34704F5C34876
:1084200004F5C349072B06F1340607F14C0708F1A0
:108430006C0809F15C090FD104F5AD445434019482
:10844000D5F85836009342464B46394630467BF0C5
:10845000F1FB0AB0BDE8F0870DF127010023364893
:108460008DF82730FEF7D4FC05F29463D3ED007A43
:10847000D5F878A605F5CD63D3ED000A05F274634F
:1084800030EE670A93ED001A8DED070A04F5C5403A
:108490006C30CDED060A8DED051A75F055FD0546DB
:1084A000204600F093FE9DF827309DED051ADDED86
:1084B000060A9DED070ACDE90203CDE900A54B466A
:1084C0004246394630467BF00BFBC2E72046918896
:1084D00003F05AFF0020BCE7114620460AB0BDE871
:1084E000F047FFF76FBE20460AB0BDE8F047FFF740
:1084F00029BE114620460AB0BDE8F047FFF79ABEF4
:1085000020460AB0BDE8F047FFF722BA20460AB07D
:10851000BDE8F047FFF75CBA00F59E4024300AB092
:10852000BDE8F047FFF7D0BA0AB0BDE8F047FFF763
:108530006FBB00BF3CD80C08102C002070B500F5B4
:10854000A04200F59E43926D24339A4205460E46A2
:1085500002D00024204670BDFFF7AEFE044600287E
:10856000F7D005F55B503188203054F0BDF9F1E7C4
:1085700021F04003152B04D0A1F15E03584258416D
:10858000704701207047000018294DD8DFE801F03E
:108590000D1115191D2125282C4C303438443C3C34
:1085A000404C4C4C4C4C4C4C480000F59E406030CC
:1085B000704700F59D403830704700F59D404030D1
:1085C000704700F59D404830704700F59D405030A1
:1085D000704700F59D407830704700F59E40704729
:1085E00000F59E400830704700F59E401C307047F3
:1085F00000F59E402430704700F59E403C307047A7
:1086000000F59E404430704700F59E404C30704766
:1086100000F59E405830704700F59E406830704726
:1086200000F59F40103070470020704700290DDB97
:10863000074890F8442FCBB29A4207D3D0F8403F76
:108640000122595CA0F5005006F070B8704700BFD9
:10865000104C00202DE9F34100F5005300F55B5567
:1086600093F8103F03F0010603F0020803F004073B
:108670005B07044605F1200535D01F4A0621284630
:108680004FF042FF26B104F54950143077F0E0FC7A
:10869000B8F1000F04D004F54E502C3077F054FAA6
:1086A00027B104F55450043078F0FCF804F5C044C8
:1086B000012384F89133114A114B1249B8F1000F8C
:1086C00008BF1A46002F08BF1946CDE900210E4AFF
:1086D0000621002E18BF134628460C4A4FF014FFFF
:1086E00002B0BDE8F0810A4A0621284602B0BDE882
:1086F000F0414FF009BF00BF69D80C085ED80C08E4
:1087000098B90D0865D80C0858D80C087AD80C0808
:108710008CD80C0810B5044600F54950143077F099
:10872000C3FC04F54E502C3077F03AFA04F554505F
:10873000043078F0F1F804F5C04393F891235AB16E
:10874000002283F8912304F55B50044ABDE81040F1
:10875000062120304FF0D8BE10BD00BFACD80C08A9
:1087600009B1FFF777BFFFF7D5BF000000F5A042C2
:108770000346916D074881420AD092F8650040B9DE
:1087800003F59E432433994203D192F88A06704739
:1087900000207047707B002010B504467FF05EFA21
:1087A000054B9B6FC01A642804D82046BDE81040D2
:1087B00058F0F0B910BD00BF107C002010B500F5D6
:1087C0003C54D4ED007AF5EEC07AF1EE10FA8AB09E
:1087D0004FF0000344D907930893099306AB019324
:1087E00007AB009303AA05AB04A900F5A25009F05A
:1087F00017FA30B3DDED080A9DED070AA8F018FB63
:10880000DDED090AA8F014FBD4ED007A9DED047AA1
:1088100077EEA76AB4EEE70AF1EE10FAF4EEC76A53
:10882000ACBF01200020F1EE10FA0CD802309DED13
:10883000037AF4EEC77AF1EE10FA0CD8003818BFBC
:1088400001200AB010BDF4EEC77AF1EE10FA9CBF19
:108850000130C0B2EBE7012894BF00200120F0E70F
:108860000020EEE710B5074B1A7A4AB901241C72B2
:108870004CF000FD22461121BDE810404CF0B2BA88
:1088800010BD00BFB88F002010B5074B1A7A4AB14F
:1088900000241C724CF0EEFC22461121BDE8104071
:1088A0004CF0A0BA10BD00BFB88F0020F0B505464F
:1088B00085B0684605F5A2560EF0F0FE69463046D2
:1088C00009F002FBA0B13348334C344F75F03CFB48
:1088D00040B105F53C53D3ED007AF5EEC07AF1EEE8
:1088E00010FA07D8002328462380FB73FFF7CCFF3C
:1088F00005B0F0BD2846FFF761FFA0B363787BBBEE
:1089000023780133DBB2082B237002D1304609F003
:10891000F3F92378092B02D1304609F0E5F92378E1
:10892000092B1DD94FF4857323804CF0A3FC022240
:1089300010214CF057FA7FF091F96368C01A47F2A2
:108940003053984209D905F55B50154A0221203071
:108950004FF0DAFD7FF082F960602846FFF782FF72
:108960006378FB73C4E72678002EF9D0013E637864
:10897000F6B22670002BF3D0002EF1D166704CF0C9
:1089800079FC324610214CF02DFA2846FFF77CFF87
:10899000E6E700BFFC8E0020B88F00205D9000202D
:1089A000C0D80C0800F5A040D0F8DC36042B14BF6A
:1089B00090F808070120704773B500F5A0450192B3
:1089C000A5F8701004467FF049F96867A86D036840
:1089D0005B68984785F86E00A86D03685B689847E8
:1089E0000F28019A0BD80F2826D8DFE800F01B25A6
:1089F0001B1B1B1B1B1B1B254C250A250A0A1828A1
:108A00001AD104F50056019296F9DC34A3B1A86D91
:108A100003685B68984785F86E0096F9DC34019A24
:108A2000022B27E01F4B93F89233F3B104F59D41DD
:108A30007831204605F0A6FDA86D95F86E600368B4
:108A40005B68984704F55B54864204F1200420D00B
:108A5000A86D03689B689847134A03460421204683
:108A600002B0BDE870404FF04FBD04F5005393F9DC
:108A7000DC34022BDAD0042B16BF04F59D4104F53B
:108A80009E413831D5E72046FFF78CFF0028D3D12F
:108A9000B7E7064A0421204602B0BDE870404FF017
:108AA00033BD00BF108C0020D0D80C08F2D80C08C1
:108AB000F0B5044604F5A04685B00F46154657F0BC
:108AC000EFFFB06DA6F8707003685B6898471828D0
:108AD0001ED8DFE800F00D0D0D0D0D0D0D0D0D1D57
:108AE00052680D0D57571D1D1D1D1D1D1D1D0D000F
:108AF000304BD3F8DC26012A20D104F5005393F83B
:108B0000DD34023B012B19D904F5405383F8DC26F0
:108B1000B06D294A294B052D18BF134602680393EF
:108B20009268904704F55B5420340090039B244ADC
:108B3000042120464FF0E8FC05B0F0BD214B93F82E
:108B400092333BB104F59D412A467831204605F029
:108B500019FDDDE704F5005393F9DD34032B03D150
:108B6000204603F06BFCD3E7022BEBD0042B15D18E
:108B700004F59E412A462431E8E72046FFF712FF1C
:108B80000028C5D104F5005393F9DD34032BE7D059
:108B9000022BD7D0042BEBD0012BB9D104F59E4189
:108BA0002A463C31D2E704F5005393F9DD34042B17
:108BB000AED1DDE7107C002008D90C0801BD0C08FF
:108BC00010D90C08108C002070B500F55B550446D8
:108BD0002035114A0421284604F5A0464FF094FCA4
:108BE0000023A6F8703004F5005393F82434032BC7
:108BF00011D196F86E103022204605F097FDB06D29
:108C000003689B689847054A034606212846BDE845
:108C100070404FF079BC70BD24D90C083BD90C08CA
:108C200000F5405310B500220529044600F55B50BD
:108C300083F8DC2600F120000CBF054A054A042118
:108C400004F5A0444FF060FC0023A4F8703010BD80
:108C500054D90C0865D90C0830B50B4687B00446CA
:108C6000052A18D8DFE802F0172A0350175D00F52F
:108C7000A043D3F8DC36042B20D02C4D95F881305E
:108C8000E3B12B4905F5E06026F072F928B1274BD6
:108C9000012283F8082707B030BD254905F5E060BB
:108CA00026F066FC50B104F59E4104222431A5F55E
:108CB000A04007B0BDE8304005F064BC04F5A04317
:108CC000D3F8DC36042BE6D004F5005393F9A7342F
:108CD000022B0AD1154890F8813033B1144900F5C0
:108CE000E06026F045F90028D1D104F59E41042228
:108CF0003C31204605F046FC04F51150273007B002
:108D0000BDE8304042F092B90A4A112101A87EF034
:108D10005BF804F5C24001AA0121403077F0AEFEB5
:108D2000B9E707B0BDE8304003F088BB107C0020F5
:108D3000EC8D002080D90C0870B52DED048B044615
:108D40007EF080FF4F4BB4F8BE101A884E4E8A4218
:108D500005464E4A06D01980002330601370BDECE2
:108D6000048B70BD33684A49C31A8B4276D90123FC
:108D7000137057F095FF57F04DFE356057F090FF98
:108D800057F048FE04F5405393F8DB3623B104F561
:108D9000C240403077F0C6FD57F064FE0428DED9AB
:108DA00057F07EFE0021204603F070FE0021204691
:108DB000F0EE409A03F074FE01212046B0EE409A96
:108DC00004F02EF800212046B0EE408A03F072FE37
:108DD00004F5C5406C30F0EE408A75F0BFF8DFED69
:108DE0002D7A0028B0EE690A4FF0040008BFB0EEFB
:108DF000678A59F0D5FAB0EE490A132059F0D0FA33
:108E0000B0EE680A152059F0CBFA04F5C245B0EE71
:108E1000680A1A2059F0C4FA40354620B0EE480AD4
:108E200059F0BEFA284677F00BFE08BB0121084630
:108E300059F0B8FD9FED170A022059F0B1FA9FEDE5
:108E4000150A032059F0ACFA204604F0FDF9BDECF8
:108E5000048B2046BDE8704005F020B91278002A46
:108E60003FF47DAF44F6206293427FF678AF80E70F
:108E70002846FDF72FF804F5C04393F94A312B2B10
:108E8000D4D06CE7C48F0020C88F0020C68F00208C
:108E9000400D03000000000000F5A04300F59E40D7
:108EA0009A6D2430824202D193F80807E8B10F4B43
:108EB00093F8240403F58043A0F12702012A93F8D4
:108EC000A0330FD92C2809D00A2809D0A0F13102EB
:108ED000504250410A2B18BF002070470120F9E78B
:108EE000012070470A3B584258417047104C0020FF
:108EF00008B500F5005393F8102342B193F84C33B2
:108F00002BB1FFF7C9FF80F00100C0B208BD0120FE
:108F1000FCE700002DE9F04700F50055A54F95F856
:108F20004C83044600F5C5408AB06C3075F00CF8EF
:108F3000D7F8DC36042B06464DD000284BD0B7F8C6
:108F40003E17A7F5A040FFF713FB014620B197F8A5
:108F500004174B1E5942594104F50C57DFF868A21B
:108F60001037384664F0D6FD9AF8A0330A2B8146B4
:108F700003D196BB00238AF8A03395F81033002B59
:108F800037D195F916338C4D012B03D0063BDBB25C
:108F9000012B0FD895F824340A2B0BD104F5A046E9
:108FA000B06D03681B6A984720B1F16D2B222046F3
:108FB00005F0E8FA9AF8A0330A2B04BF37238AF8A1
:108FC000A03395F824340A2B02D1372385F82434B2
:108FD0000AB0BDE8F0870121BEE740EA0803DBB232
:108FE000002BCAD1AAF5C04000F0F0F80028C1D08B
:108FF000C3E7002EECD004F5C14034307AF0E6FC33
:109000000028E5D12046FFF747FF0028E0D1B9F15D
:10901000000F00F0BD8069494A46384664F052F9B5
:1090200095F91683B8F1010F06D040F38380A8F1BB
:109030000603DBB2012B7DD85FFA88F8B8F1010F87
:109040004BD104F5A04204F59E43916D243399421F
:1090500007D192F8083723B195F8A734013B012BCB
:10906000B6D904F59E410A223C31204606AE05F0F1
:1090700089FA30460EF012FB95F9292392BBB8F11C
:10908000010F2FD004F5C048B5F92A33D8F8C8111C
:10909000DFED4B5AD1ED017A002BF8EEE77A52DD85
:1090A00007EE103AF8EEC76AE6EEA57A3046FDEE16
:1090B000E77A17EE901A0EF0F7FA00233846CDE95A
:1090C000043364F0C3FD04A965F004FB002859D003
:1090D000049B0893059B099317E004F59E410A221F
:1090E0004C31C2E72046FCF76BFF07EE900A6F4653
:1090F00004F5C3425C3221463846B8EEE70AFEF773
:109100007DF897E80F0086E80F0095F91633012BDC
:1091100010D031462046FDF7BDFB31462046FDF715
:1091200053FF95F91633072B04D104F5405401235E
:1091300084F8DA364CF09EF84A4609210AB0BDE8B8
:10914000F0474BF04FBED5EDC66A95EDC95A95ED87
:10915000C77A35EE076A36EEC57AB4EEC67AF1EE16
:1091600010FA8DBF37EE067A05F5A16393ED007A0C
:1091700027EE257A8ABFF6EE006AE7EE257AE7EE5B
:10918000267A93E7D8F8C8319A680892DB68A2E794
:10919000B8F1000F3FF41CAF95F84C33002B7FF46F
:1091A00017AF04F55B50074A052120304FF0ACF9AA
:1091B000C0E700BF107C0020104C00208CD90C08A8
:1091C0000000C84295D90C08108C002010B5044648
:1091D00000F5C5406C3074F0C1FE04F5A04404F500
:1091E000DC6494ED007A48B1DFED067AB4EEE77AFC
:1091F000F1EE10FAACBF0120002010BDDFED027AC5
:10920000F4E700BFCDCCCC3D6666663F10B500F5F7
:10921000A04200F59E41946D68318C42034602D114
:1092200092F8D40688B903F59E4324339C420DD1AD
:1092300092F8D40648B1D2F8DC36032B06D1B2F846
:109240003E07A0F116035842584110BD0020FCE72C
:109250002DE9F84F00F5A04600F59E43B26D24338A
:109260009A42054604D100F5005898F9803433B984
:109270000023C6F8C83686F8C536BDE8F88F7EF0FC
:10928000EDFCD6F87C46814634B1041B40F6C3138E
:109290009C4294BF002401242846FFF797FF834691
:1092A00020B1002486F8C44600273FE005F5C540FC
:1092B0006C3074F049FE82460028F2D005F5C147B3
:1092C000343738467AF082FB002840D096F8C476CE
:1092D000C7BB44B305F5805141F27072D1F83836FE
:1092E000002BB8BF5B42934206DCD1F83C36002B22
:1092F000B8BF5B42934228DD05F5AE4105F5C3409A
:1093000044315C300EF02CFDDFED457AC6F8C8968E
:10931000B4EEE70AF1EE10FA4FF000034CBF01275C
:109320000027C6F8CC36012386F8C43605F59070C0
:10933000F8F7F0FB022835D9002C44D10023C6F8F9
:10934000C8369AE75C465F46EDE73C46EBE73846B1
:109350007AF024FB074638B1002CA5D04FF4FA73FD
:10936000C6F8CC3654469FE7D6F8DC36012B03D03E
:10937000032B0FD03C46D9E708F5A463D3ED007A60
:10938000F5EEC07AF1EE10FAF4DD96F8D436002B43
:10939000F0D1E3E72846FFF739FF0028EAD1002C97
:1093A000DCD1C3E705F5055A98F88E12504606F051
:1093B00027FE0028C2D098F88E12504606F018FFFB
:1093C0000028B9D1BAE7D6F8C83613B9C6F8C89696
:1093D00053E7D6F8CC26A9EB03039342FFF44DAF35
:1093E00096F8C536002B7FF448AF012286F8C526D3
:1093F00098F88034DB0705D505F5C5400C216C30A5
:10940000F8F7C0FA05F55B5020302FB1054A02216C
:10941000BDE8F84F4FF078B8034A3946F8E700BF87
:1094200000009642ACD90C08C2D90C082DE9F04FC7
:109430002DED028B054685B0002305F500580393FA
:109440007EF00CFC08F27C43D3ED007AF5EEC07A96
:10945000F1EE10FAC4BF9FEDC07A67EE877A05F58A
:10946000907BC8BFFCEEE77A07465846CCBF17EEA4
:10947000906A9626F8F74EFB022840F2FB8095F89A
:1094800014349FEDB67AB02202FB0353D3ED837AF6
:1094900067EE877AFCEEE77A17EE903A9E428CBF31
:1094A00000260126B8F97034022BB8BF022307EE5C
:1094B000903AB8EEE78A03A9F6EE087A05F5A250CD
:1094C00028EE278A08F0DEFC044640B1DDED037A81
:1094D000F4EEC87AF1EE10FAACBF0124002458462D
:1094E000F8F718FB05F5C549012809F16C0905F5E0
:1094F000A04A18D8484674F027FDA0B19CB90AF5D7
:10950000DC6292ED007ADFED967AB4EEE77AF1EE66
:1095100010FA08DDDDED037AF4EEC87AF1EE10FA08
:10952000ACBF01240024484674F00EFD00900028D2
:1095300000F0FE8095F8142405EB0212D2F8C02149
:1095400072B158460192F8F7E5FA012800F29480CA
:10955000019A41F28731BA1A8A428CBF0022012255
:10956000DAF8781601B11AB9002C40F08780344639
:10957000DAF8581005F59E42243291421AD198F932
:10958000A824002A40F0828000228AF8C626DAF851
:10959000DC26042A00F0AA80072A00F0BD80032AF6
:1095A00008D12846FFF732FE20B100248AF8C546CC
:1095B000CAF87C469AF8C62602B18CB907EE904AE2
:1095C0009FED687AF8EE677A0AF5DC6267EE877AD3
:1095D000D2ED006A9FED647AE6EE877AC2ED007AFA
:1095E0002846FFF7F3FD044698B19AF8E406CAF856
:1095F000787608B9CAF8E876DAF8581005F59E4288
:109600002432914205D1DAF87C2602B108B9CAF8B1
:109610007C769AF80C288AF8E44664F3C3028AF848
:109620000C286EF0CFFD21466EF0A8FD4F4A28466B
:109630005471FFF70DFE2846FBF748F934B198F84E
:1096400026241AB97EF00AFBC8F8280488F82644B4
:109650002846FFF7BBFD00287BD1484674F07EFC0E
:1096600080F00100C0B28AF8EC0605B0BDEC028BB8
:10967000BDE8F08F002615E7002271E71FF062FBBE
:109680001EF056FB00287FF472AF71E7524207EEDE
:10969000902A05F61862F8EEE77A92ED007AF4EE79
:1096A000C77AF1EE10FA13DD01228AF8C626CAF84D
:1096B000D0760AF5DC62DFED2E7A92ED007AB4EE18
:1096C000E77AF1EE10FA7FF762AFC2ED007A5EE75B
:1096D0009AF8C626002A3FF45AAFDAF8D02640F6A8
:1096E000B831BA1A8A423FF64FAF50E705F5C1408C
:1096F00034307AF053F900283FF45CAF0AF5CD62BC
:1097000092ED007ADFED1A7AB4EEE77AF1EE10FA14
:109710007FF750AF009C4DE70AF5CD6292ED007ADD
:10972000FEEE007AB4EEE77AF1EE10FAF2D441E7F9
:10973000DAF8DC26002C18BF3446012A07D005F5DC
:10974000C14034307AF020F900283FF433AF0024D0
:1097500030E7002087E700BF0000B4420000C842A5
:109760009A99993E9A99193E9A99593F5D9000208D
:10977000CDCC4C3E00207047002070470120704740
:109780000020704701207047034BD3F8DC06431ECE
:1097900058425841704700BF107C002030B587B058
:1097A00002A80DF07BFF3B487AF0EEF820B13A4971
:1097B0003A48FDF781F81FE036487AF0EFF8E8B153
:1097C000374C04F12405234604F11002A4F11001E2
:1097D000A4F5947000957AF007F9CDE90045A4F658
:1097E0006C3292ED000A2F4904F11003A4F110022B
:1097F000A4F594707AF0BAF807B030BD254802A9F4
:109800007AF00AF908B102A9D2E7274CD4F8A83EA9
:10981000002B0CDD94F8483E4BB1A4F500502049D4
:10982000FDF74AF8A4F50050FCF7E2FCE4E71B481A
:1098300002F0C6FC0028BAD11C4C94F8EC315B074E
:1098400020D4D4F80032002BB1D0134AA2F1200169
:10985000A2F110000EF0F0F90028A8D1144C0F4826
:10986000D4ED007AB7EE000A04F6783130EE670ADC
:10987000FDF752F8094804F6583204F67831FCF73F
:10988000FBFBB9E7A4F5C040FDF7C2F80028B3D14F
:10989000D7E700BFC48C0020FC8D0020102C0020D6
:1098A000EC8D0020585B0020104C0020108C002014
:1098B0008482002008B50A4890F81935013B012B35
:1098C00003D8A0F50050F9F771F90648F9F798F8B0
:1098D0000448F9F731F9BDE808400248F9F74EBCF1
:1098E000104C0020102C002010B5134CA0420FD0BB
:1098F00004F1080290420BD004F11002904207D00C
:1099000004F13802904203D004F15C02904206D187
:109910000A4B93F9D104B0FA80F0400910BD0368F6
:109920001B6A984730B1A4F5F65494F8DA0680F033
:109930000100F3E70120F1E7D07A0020104C00206D
:1099400010B5114CA0421AD004F10802904216D072
:1099500004F11002904212D004F1380290420ED06D
:1099600004F15C0290420AD003681B6A984740B138
:10997000A4F5F65494F8DA0680F0010010BD00203A
:10998000FCE70120FAE700BFD07A0020024A02601B
:10999000024A4260704700BF14DA0C0850400020B1
:1099A00008B503681B6E98470648826DA0F1E40372
:1099B0009A4205D0BDE80840A0F5A040FEF7AABE37
:1099C00008BD00BF107C00202DE9F041474C04F594
:1099D000CA6300221A60A4F1DC03C11A4B42A4F549
:1099E00000584B4188F87C3904F5CC63002584F895
:1099F0003456A4F88A5684F88E5684F84C5684F867
:109A0000C55684F8C656C4F8B456C4F8B056C4F85F
:109A1000AC56C4F8BC561A60436804F58057D3F8B6
:109A2000FC31A4F8843607F5EE7306460FCB07F534
:109A3000E67C8CE80F0084F88D5684F89C56C7F8B5
:109A4000A8517EF00BF92066336830465B69984771
:109A50004FF0FF3384F8900684F8915688F8DC566E
:109A600087F8055284F88F56C4F88830336830463A
:109A7000DB6D98470546002835D0336830469B6B30
:109A8000984784F8D406D8F808090368DB6B984730
:109A900008F5CF6076F044FCA4F5A04002F064FF26
:109AA000A8F54F6064F09CF894F80837C3B1A4F5AA
:109AB000A040FFF78BFB98B907F53B7074F04EFAA6
:109AC00070B9A06D03685B6B984748B955F0F4FB1B
:109AD000074A06214EF018FD04F5E06025F0F4FA7F
:109AE0000448F8F7CDFA2846BDE8F081107C002044
:109AF000D4D90C08102C002070B503685B6E0E469C
:109B000015469847044650B995F900303BB90548C9
:109B1000054B00683246C06A29461BF0B7FF204655
:109B200070BD00BF0C2C0020F8D90C0810B50E4CED
:109B3000204676F0F1F904F5AC7075F069FF04F594
:109B40002C7076F097FE094B03F5A042002182F8B5
:109B50004C1602F5CA62002103F540531160012240
:109B600083F8A02110BD00BF645E0020102C0020EF
:109B700008B52DED028B1520B0EE408A58F010FC90
:109B8000B0EE480ABDEC028B1A20BDE8084058F040
:109B900007BC000008B5084890F9D1340121A0F5B0
:109BA000005033B103F03CF9BDE80840462058F0BE
:109BB000F7BB03F05DF9F7E7104C00200420704775
:109BC00000487047C61D0E0800487047C61D0E08A5
:109BD000037A73B1D0ED037AFDEEE77A17EE903A8F
:109BE000084AC2F8F036437A3BB10369C2F8F4364A
:109BF00070474368D3F8F831F2E74368D3F8FC3193
:109C0000F4E700BF107C002008B50023038100F1B9
:109C10001401406808F04CF9012008BDF8B56D4EFC
:109C20002DED048B04460121304606F5A04797ED43
:109C3000289ADFED699A02F029FF0121B0EE408AEF
:109C4000304602F02DFFC8EE297A06F5005560680F
:109C5000B5F9F43404F1140108EE903AF8EEE88A0C
:109C6000B5F9F63468EEA78AC0EE297A08EE103A04
:109C7000B8EEC88A28EE278A08F01AF995F9FA345E
:109C80005BB39FED567AF0EEE87AF4EEC77AF1EE28
:109C900010FA22D5227A6368002A54D10122227256
:109CA0000022E26094ED037ADFED4D7AD3F8F831CB
:109CB0004C4867EEC77A9FED4C7A67EE877A0122AF
:109CC000FDEEE77AB0EE490A17EE901A0B44C7F89A
:109CD000F036002376F0B0F808E000234148237204
:109CE000F0EE490AB0EE680A76F0A2F8042058F0C7
:109CF00057FB95F9FA3443B19FED387AF0EEC87A04
:109D0000F4EEC77AF1EE10FA28D4002337486372D4
:109D1000F0EE490AB0EE480A75F0E4FC132058F062
:109D20003FFBB5F9F834002B03DD314E96F91A35B7
:109D30005BBB28482021F8F7FFFB002842D12548CB
:109D400002F0E2FC41E0D3EDC56A96ED467AD4ED2F
:109D5000037AE6EE877AC4ED037AA3E7637A2BB938
:109D6000012363726368D3F8FC3123612169C7F86A
:109D7000F4166368D3F8FC010023091A1A461B483D
:109D8000B0EE490A75F094FDC8E70121A6F54050F0
:109D900002F090FE80EE297AB5F9F834002106F23F
:109DA000045007EE903AF8EEE77AF0EE490A27EE13
:109DB000870A76F05FFCBDEC048B2046BDE8F840D6
:109DC000FFF7D6BE0348F9F745F807EE900AB8EE5C
:109DD000E70AF0E7102C002000A08C4500000034BA
:109DE000E02E6542645E00200000C842BC5F002097
:109DF000105C00202DE9F04F2DED0C8BDFF8A0A3B7
:109E00009FEDDCDA9FEDDC9A97B000F114050AF5BE
:109E1000A04B0446012150469BED28BA02F036FEC5
:109E200001215046F0EE408A02F03AFE01215046F0
:109E3000B0EE408A02F03EFEDFEDD07A88EEA77ADF
:109E40000AF5005601A8B6F9F4340AEE903AF8EE95
:109E5000EAAAB6F9F634DFEDCA8A6AEE87AA88EE76
:109E6000277A0AEE103AB8EECAAAB6F9F8349FED8E
:109E7000C58A2AEE07AA80EE277A09EE903AF8EE14
:109E8000E99A6AEE8D7A69EE879AF0EEEACAF4EE04
:109E9000C8CACDED017AB0EECACA6AEE0D7AF1EE0B
:109EA00010FAF0EEE9BAB4EEC8CACDED027A58BFA6
:109EB0004FF0010969EE8D7A48BF4FF00009F1EECD
:109EC00010FAF4EEC8BA9AED460ACDED037A54BF03
:109ED0004FF001084FF00008F1EE10FA54BF0127CF
:109EE000002721F087FF01A9284621F08DFA284696
:109EF00021F07CFB284621F0F3FA20EE090A2846DF
:109F000020EE280ABDEEC00A10EE103ACBF8F0366B
:109F100021F000FB20EE090A20EE280ADFED9A8AE4
:109F2000BDEEC00ACDED0D8A10EE103ACBF8F43636
:109F30000DF1280B4FF07E53594660680A93CDED22
:109F40000C8ACDED0B8A07F0B3FF0021504602F0DA
:109F500067FFB0EEC00AB4EEC80AF1EE10FA16D5EB
:109F60005046FFF733F990B9F4EEC8CAF1EE10FA93
:109F70000DD5B4EEC8CAF1EE10FA08D5F4EEC8BAA1
:109F8000F1EE10FA44BF9BE80F0085E80F000AA825
:109F900021F090FB294612A88DED141A8DED120ABE
:109FA000CDED130ACDED151A21F096FB0DF1100A37
:109FB00051460EA88DED101ACDED048ACDED058A1F
:109FC000CDED068A8DED0E0ACDED0F0ACDED111AFD
:109FD00021F054F9B6F9F434DFED6C7A01EE103A61
:109FE000B6F9F63409EE103AB6F9F83408EE903ABC
:109FF000B8EEC11AB8EEC99AF8EEE88A21EE271A2F
:10A0000029EE279A68EEA78AF4EEC8CAF1EE10FA94
:10A0100021EE0D1A29EE0D9A68EE8D8A07D594F877
:10A020002430DFED597A002B18BFB0EE671AB4EE7A
:10A03000C8CAF1EE10FA07D594F82530DFED527A50
:10A04000002B18BFB0EE679AF4EEC8BAF1EE10FA22
:10A0500007D594F82630DFED4C7A002B18BFF0EED0
:10A06000678A9AE8070007AE86E80700F1EE410A22
:10A07000C2209DED070A1FF0E7FBC3208DED070A04
:10A08000B0EE491AF1EE490A9DED080A1FF0DCFB1B
:10A09000B0EE681AF1EE680A8DED080AC4209DED55
:10A0A000090A1FF0D1FB514630468DED090A21F017
:10A0B00037FE12A928468DED120ACDED130A8DED5B
:10A0C000141A21F0A1F9284621F090FA304BDDED69
:10A0D000076A93ED967A9FED280AC6EE877A304696
:10A0E000DDED086ACDED077AD3EDEC7A86EEA77A3E
:10A0F000DDED096A8DED087A86EEA77A8DED097A95
:10A1000021F078FEB9F1000F01D0CDED07AAB8F12A
:10A11000000F01D08DED08AA0FB1CDED099AF0EE38
:10A120004B0A9DED070A1B4875F082FE042058F08B
:10A1300037F9F0EE4B0A9DED080A174875F0D2FA90
:10A14000132058F02DF90021F0EE4B0A9DED090A7D
:10A15000124876F08FFA2046FFF70AFD84F8249023
:10A1600084F8258084F8267017B0BDEC0C8BBDE810
:10A17000F08F00BF35FA8E3CE02E654200A08C4582
:10A180000000C8420000003400000000CDCC4C3E6E
:10A19000105C0020645E0020BC5F00201461002081
:10A1A000102C002010B50446FFF7F4FC0B4B93F97C
:10A1B000FA24022A0DD1B3F9F824002A09DD03F5A7
:10A1C000805393F91A3523B12046BDE81040FFF7BC
:10A1D00011BE2046BDE81040FFF720BD104C002006
:10A1E0000A2070470048704735E60C080048704761
:10A1F00035E60C08012070470120704701207047A8
:10A200000120704701207047034BD3F8DC06031F81
:10A2100058425841704700BF107C0020F8B51C4ED2
:10A2200006F5805404F5EE730FCB04F5E67504F5DE
:10A23000F67485E80F0084E80F00002706F5E0605B
:10A2400086F8907625F080F9124B1C68E56A2B6839
:10A2500028465B689847A8B195F84D3093B1E36AFA
:10A260009B8F7BB155F028F8E36A0B4A9B8F062140
:10A270004EF04AF9E36A06F5E060998F24F050FF4A
:10A28000E36A9F8705487AF017FB0120F8BD00BFFD
:10A29000107C00200C2C0020ECDA0C08D058002098
:10A2A00010B50A4C94F80437012B0AD104F5E0608C
:10A2B00022F00EFAB4F83E37152B02D1044879F09B
:10A2C00043FC0023C4F87C3610BD00BF107C002086
:10A2D000C48C002008B507F0F1FF90F87C32DB0752
:10A2E00004D5BDE80840024824F0CABF08BD00BF3D
:10A2F0001083002010B52F4C94F80437012B0ED09A
:10A30000A4F1C4010822A4F5A04004F03BF954F0E4
:10A31000D3FFBDE81040284A06214EF0F5B8B4F846
:10A320003E37162B05D0152B34D1D4F8DC36072B4D
:10A330000AD1224804F0ACFC204804F0F9FDBDE845
:10A3400010401E4804F008BDA4F5A040F9F786F8B7
:10A35000A4F5A040F8F780FFA4F54053D4F8F01618
:10A3600093F93825164864235A4379F049FBC4F819
:10A37000F006134879F086FC30B1BDE810409FED3F
:10A38000110A462058F00CB8A4F5A040BDE81040D2
:10A39000F8F748BD1E2B18BF4FF0FF33074818BF12
:10A3A000C4F84836F9F75AF80448F8F755FF034857
:10A3B000ECE700BF107C002004DB0C08102C002010
:10A3C000C48C00200000000010B5144BB3F83E37D9
:10A3D000532B04461ED103F00DF99FED110A4620C0
:10A3E00057F0DEFF9FED0E0A492057F0D9FF9FED91
:10A3F0000C0A4A2057F0D4FF462058F0B1F8492003
:10A4000058F0AEF84A2058F0ABF82046BDE81040AE
:10A41000FFF78CBBBDE81040FFF74CBA107C002062
:10A42000000000000820704700487047A0DB0C08BF
:10A4300000487047ACDB0C080120704708B50248A3
:10A44000FEF708F9012008BD102C0020014800F09B
:10A4500061B900BF087B002010B50446FFF72AFA57
:10A460002046BDE81040FFF795BB00000120704773
:10A470000048704724DC0C08004870472CDC0C08AE
:10A48000012070470120704710B5054B03F5F674A5
:10A4900003F5EE730FCB84E80F00012010BD00BF61
:10A4A000108C002008B50B4800F5A04200F50053C1
:10A4B0000321D3F8383F93FBF1F3C2F8F036F8F7F5
:10A4C00033FF0448F8F7C8FEBDE808400148F8F734
:10A4D000A9BC00BF102C002007207047004870471F
:10A4E000BEBE0C0800487047A4DC0C080120704771
:10A4F00001207047012070477047000010B5064CDE
:10A5000000230372036120467AF0D6F9A4F5335094
:10A51000FCF790F9012010BDD058002010B5194C5F
:10A52000D4F8203FB3F9083023B9D4F82C3FB3F95D
:10A530000830F3B1002303720361D4F8200F56F002
:10A540009FFC04F63873D3ED007A0F48F8EEE77AF3
:10A5500027EE800ABDEEC00A10EE103AC0F8F036C1
:10A56000A0F5A040F8F7E0FEBDE81040074801F074
:10A5700025BD037A002BE0D0A4F50050F8F76EFF5C
:10A58000F2E700BF104C0020107C0020102C0020AF
:10A5900070B54E4DDFED4E7A95F814349FED4D7A3F
:10A5A0002DED048BB02606FB035393ED848A9FEDBB
:10A5B0004A9A28EE278A05F5B253BDEEC88A93ED74
:10A5C000030AF8EEC87A044667EE897A97EE870A9E
:10A5D0001FF026F9237AF0EE408A002B62D105F5B0
:10A5E0000053D3F8203FB3F90830002B5AD1284646
:10A5F00002F08AF8002855D195F8143495F85814CB
:10A6000006FB035393F8F12100294BD1012A49D9C4
:10A6100093ED837AF0EE087AB4EEE77AF1EE10FA71
:10A6200040DBDFED2E7AB0EEE80AB4EEE70AF1EE99
:10A6300010FA37D5236993B37DF010FB2369C01A54
:10A64000B0F5FA7F32D8237A002B3CD0244DA5F107
:10A65000200696E80F0085E80F0094ED038AA5F127
:10A6600010013046B8EEC88A0DF07AFB28EE098A50
:10A67000DFED1C0A284670EE200AB0EE480A0DF005
:10A68000E5FB194B9FED190AD3F80809BDEC048BC3
:10A6900003682A4631469B6ABDE8704018477DF042
:10A6A000DDFA20612369002BCDD0C5E7104D84ED84
:10A6B000038A012323720023236105F110030FCBCA
:10A6C00085E80F00BFE7BDEC048B70BD102C0020A7
:10A6D0000000C84235FA8E3C0AD7233CDB0FC93F45
:10A6E000FC8D002000007A44105C00200000000077
:10A6F000DC8D0020C3680B60007A7047052070472E
:10A70000004870471CDD0C08004870472CDD0C0821
:10A710000120704738B52DED028B4D4C9FED4D8AD1
:10A72000D4F8200F56F0ACFBD4F8383F07EE903A3F
:10A73000F8EEE77A04F5405527EE800AA4F50050BC
:10A74000BDEEC00A10EE103AC5F8F036F8F7ECFD91
:10A75000D4F8240F56F094FBB5EEC00AF1EE10FACF
:10A76000CBBF04F5916304F63C73D3ED007AD3EDCF
:10A77000007A3948CBBF20EE270A20EE270A20EEC8
:10A78000080A28EE400ABDEEC00A10EE103AC5F8DD
:10A79000F436F8F793FD04F5916393ED007AD5F85C
:10A7A000F40604F63C7327EE087AD3ED007A27EE20
:10A7B000888AFDEEC77A17EE902AFDEEC87A17EE6A
:10A7C000901A1FF0E1F8C5F8F4062348FDF7CEFF14
:10A7D00020B1D5F8F4365B42C5F8F43695F86C3004
:10A7E00063B194F9DC34022B08D100230121462007
:10A7F000C5F8F036C5F8F43658F02CF956F050FA92
:10A800005F2157F07FFAF8B157F04CFA02281BD1BC
:10A8100095F88D36C3B905F5CC6304F5A56493EDC1
:10A82000007AD4ED007AB4EEE77AF1EE10FA0BD5A7
:10A83000012385F88D36BDEC028B084A0848BDE837
:10A84000384004214DF060BEBDEC028B38BD00BF26
:10A85000104C00200000C842102C002034DD0C08F1
:10A86000F062002010B50446FFF724F82046BDE84A
:10A870001040FFF78FB9000006207047004870476E
:10A88000B4DD0C0800487047C4DD0C080120704797
:10A890000120704701207047012070477047000079
:10A8A00010B5054C20467AF007F8A4F53350FBF7B5
:10A8B000C1FF012010BD00BFD058002038B50F4C9B
:10A8C00004F50055D5F8200F56F0DAFA05F638727F
:10A8D000D2ED007AF8EEE77A04F5A04327EE800A7D
:10A8E0002046BDEEC00A10EE102AC3F8F026F8F795
:10A8F0001BFD2046BDE8384001F060BB102C002055
:10A900000F207047004870473CDE0C080048704735
:10A9100044DE0C0801207047012070470120704779
:10A920000120704701207047012070477FB50B4D13
:10A9300005F54053002283F8DA2605F5C3435C335E
:10A9400006460FCB6C4684E80F0000232846B36010
:10A950002146FCF739FB012004B070BD102C00200B
:10A9600010B53C4CD4F8AC36002B2CDD7DF076F9DC
:10A97000D4F8AC36C01A40F6B733984223D8A4F5C1
:10A980004053D4F8A006D3F8382F51421EF0FCFFF4
:10A99000C4F8F006A4F5A040F8F7C6FCD4F8B03629
:10A9A000002B14DC2C48F8F757FC2C4890F8DA36CA
:10A9B00093B30121A0F5405002F032FABDE81040F7
:10A9C000462057F0EDBC2448F8F748FDE6E77DF057
:10A9D00045F9D4F8B036C01A40F6B7339842E1D8FA
:10A9E0001F4BDFED206A93ED007AD4F8A40603F63E
:10A9F000B423D3ED007A27EE267A67EEA67ABDEE71
:10AA0000C77AFDEEE77A17EE102A17EE901A1EF0BD
:10AA1000BBFFC4F8F406C8E7A0F5805090F967348E
:10AA2000012B04DCBDE810400B48F8F7FBB9D4F863
:10AA3000BC36002BF6D07DF011F9D4F8BC36C01A24
:10AA400040F6B7339842EDD804F5D76494ED000A88
:10AA5000B4E700BF107C0020102C0020105C002008
:10AA6000985000200000C842D0ED027A0348FCEE66
:10AA7000E77A17EE903A99B201F086BC102C0020CC
:10AA800084B010B503AC84E80E000B4821466F2259
:10AA9000FCF7DEF99DF80C1011F0040102D12046FC
:10AAA0000CF0C6FE04482146FCF78EFABDE81040C3
:10AAB000012004B0704700BF102C0020B0EEC00A87
:10AAC000FDEEC07A38B54FF6FF7205460C4617EE1C
:10AAD000900A00211EF058FF07EE900A002CF8EEB5
:10AAE000E77A054BC5ED027A14BF4FF0FF32012221
:10AAF00083F8A42138BD00BF108C0020FEF74EBEA5
:10AB00000C20704700487047BCDE0C0800487047B6
:10AB1000B51D0E08012070470120704701207047C5
:10AB2000012070470120704708B50C48FDF79CF8DC
:10AB30000A480B49FBF7AEFE0848F7F7F1FE40B1B3
:10AB400006484FF48051F7F7F7FC10B10348FBF7C4
:10AB500071FE024800F096FF012008BD102C002075
:10AB6000FC8D002008B50D48F8F778FC0B48F7F786
:10AB7000D7FE50B109484FF48051F7F7DDFC20B102
:10AB8000BDE80840054801F019BA0448F8F764FB2D
:10AB9000BDE808400148F8F745B900BF102C002077
:10ABA00008B50A484FF48051F7F7C6FC38B1084899
:10ABB0000022D0F8FC1100F5F6700CF075FDBDE830
:10ABC00008400248002101F0DFBB00BF102C00202C
:10ABD000108C0020881A10B51EF0FEFD104BD3F823
:10ABE000A0210028B8BF4042002AB8BF524248F610
:10ABF000A041B2FBF1F24FF47A7102FB01118842DD
:10AC00000CDC93F8EC21D20606D503F5F67403F5B7
:10AC1000EE730FCB84E80F00012000E0002010BD90
:10AC2000108C002013B504464068019100F57F7038
:10AC300020F01AFFDFED0A7A20EE270A1EF06EFDE3
:10AC4000DFED087A019920EE270A2046FDEEC07A52
:10AC500017EE902A02B0BDE81040FFF7BBBF00BF5F
:10AC6000E02E65420000C84284B070B52DED048B23
:10AC700086B00FAD85E80E004D4CDFED4E8A0646DE
:10AC8000D4F8080904F5405494ED6E0A0368B0EE58
:10AC9000C00A5B6A9847B4EEE80AF1EE10FAB0EE2B
:10ACA000408A07DA012006B0BDEC048BBDE8704095
:10ACB00004B07047404928460CF05EFF02A8CDED75
:10ACC000030A8DED020A20F073FF04A88DED040A3B
:10ACD000B0EE480ACDED050A20F064FE13A928461F
:10ACE0008DED000ACDED010A0CF046FF02A88DEDB6
:10ACF000020ACDED030A20F001FFB4EEE80AF1EEFE
:10AD000010FACFDBB4EEC08AF1EE10FA9FED2B9A69
:10AD1000DFED2B8ADFED2B9A2BD802A8694620F0B5
:10AD200031FE04A88DED040ACDED050A20F09CFE4D
:10AD3000684620EE098A20F097FE94F9A43107EEC8
:10AD4000903AF8EEE77A28EE288AA7EEA90A1EF0D4
:10AD500067FD20EE090ABDEEC88A20EE280A18EE2B
:10AD6000101AFDEEC07A304617EE902AFFF732FF38
:10AD700099E738EE400A38EE088A80EE080AA6F015
:10AD8000BFF902A8B0EE408A20F06EFE94F9A4311B
:10AD9000F0EE007AB0EE697AA8EE677A07EE903AA4
:10ADA000F8EEE77AA7EE270A1EF03AFDC0E700BFEB
:10ADB000105C002000000034EC8D0020E02E654285
:10ADC0000000C842DB0FC93F10B504460848F7F73A
:10ADD000A7FD20B92046BDE81040FEF7DFBC0448BF
:10ADE0004FF48051F7F7A8FB0028F3D010BD00BF47
:10ADF000102C0020002070470048704734DF0C08FA
:10AE0000004870473CDF0C08002070470020704766
:10AE100038B5154C05460021204601F037FE0420C8
:10AE200057F0BEFA0021204601F03AFE132057F0F9
:10AE3000B7FA0021204601F03DFE2846FEF798FEB5
:10AE40002046012101F0ECFF462057F0A9FA6B687B
:10AE500004F5A044D3F8F831C4F8F0366B68D3F8A1
:10AE6000FC31C4F8F43638BD102C0020FEF75EBE6D
:10AE70000B2070470048704762E20C08004870479A
:10AE8000B4DF0C0801207047012070470120704793
:10AE90000020704770B50B4E06F5C04505F5EE7302
:10AEA0000FCB05F5E67484E80F003046FBF788F811
:10AEB00001463046FCF756F9002385F86032012040
:10AEC00070BD00BF102C002038B53148F8F7C6FA25
:10AED0002F48F8F7C1F92E48F7F7A4FF2C481021A6
:10AEE000F7F72AFBE0B12B4AD2F8E031D2F8F02193
:10AEF0009342D4BF00230123264C94F8602272B9F8
:10AF000073B304F5EE730FCB04F5E67585E80F0017
:10AF1000A4F5C040FBF792FA012384F8603238BDF3
:10AF20001D4AB2F9041F0029F9DD02F580429FEDA8
:10AF30001B7AD2F8E031D2F8D0219B1A07EE903A72
:10AF4000F8EEE77A67EE877A07EE101AB8EEC77A5E
:10AF5000F4EEC77AF1EE10FACCBF01230023CBE761
:10AF6000A4F58043642193F9382512FB01F2D3F84C
:10AF7000381FA4F580548A42A8BF0A46D4F8F006C8
:10AF8000C3F8382F51421EF0FFFCC4F8F006C6E7A4
:10AF9000102C0020108C0020104C00200AD7233CDD
:10AFA00038B52A4DB5F9CC3483EAE371A1EBE371EE
:10AFB00089B241B1002B05F58043B4BF4FF0FF3299
:10AFC000012283F8A421224C224801F0DDF994F8F3
:10AFD0008E36DBB995F9A734022B18D194F881305D
:10AFE0008BB11D49A1F6DC2024F0C2FA58B101232F
:10AFF0001A49184884F83937282203F0C3FA28B9C7
:10B00000002384F83937012384F88E3638BD012BAC
:10B010000ED1A4F5A04001F0D3F848B1A4F5A040AA
:10B02000FBF7CAF90028B8BF4042B0F57A7FD5DBFC
:10B0300095F9A734042BE9D194F88130002BE2D0A4
:10B040000549A1F6DC2024F00FFBCFE7104C0020CF
:10B05000107C0020102C0020EC8D0020347B002080
:10B0600002207047004870472CE00C0800487047E9
:10B07000AA1D0E08034B0022C3F8F026C3F8F426DD
:10B08000704700BF107C002038B5094D04462846A3
:10B09000F7F7B6FC2846F7F74FFD2046F7F764FDB3
:10B0A0002846F8F76BF82046BDE83840FEF772BD39
:10B0B000102C00200D20704700487047A8E00C08B5
:10B0C00000487047B0E00C0801207047012070472D
:10B0D000012070470023C37480F82430012070479A
:10B0E0000148002101F050B9102C00202DE9F04159
:10B0F000B44CD4E979322DED088B1343D4F8E02118
:10B10000134388B005460FD1AF48F8F7A7F9AE480A
:10B11000F8F7A2F89FEDAD0A462008B0BDEC088B09
:10B12000BDE8F04157F03CB907F0C8F890F87C3220
:10B13000DB07E9D5B5F90830E97C09EE103AB5F935
:10B14000103008EE903AB8EEC99AF8EEE88AA4F505
:10B150008056002940F0D7809FED9DAA29EE0ABABB
:10B160000122FDEECB7AA4F5C04017EE903AC6F866
:10B170005836FAF753FF686800F57F700790B0EE15
:10B18000408A20F071FCDFED937A20EE270A1EF052
:10B19000C5FA0798F0EE409A20F0B0FCA4F5C04044
:10B1A000F0EE40AAFEF712F8002878D104F5EE7709
:10B1B00097E80F0005F1140C8CE80F0097E80F00DA
:10B1C00004F5E67C8CE80F0004F5F67C8CE80F00B3
:10B1D000D4ED7C7A8048F8EEE77AF0EE680A77EEF4
:10B1E0008B7AB0EE690AFDEEE77AC4ED7C7A0CF05A
:10B1F0002DFE002386F8C53695F91230724803EB10
:10B20000830303EB83039B000121A6F88636F6F740
:10B21000E7FE96F8D486B8F1000F74D16F4B9FED1E
:10B22000707AB3F9703407EE903AF8EEE77A67EE89
:10B23000877AF4EEE7AAF1EE10FA64DD54F03CF8F8
:10B24000074619EE900AF5F75FF9CDE9040118EE0B
:10B25000900AF5F759F9CDE9020119EE100AF5F750
:10B2600053F9604ACDE90001062138464DF04CF90A
:10B270007CF0F4FCC6F84486C6F830067CF0EEFCA0
:10B280000123C6F8400629EE8A0AEB741EF070FA14
:10B29000BDEEC00A10EE103AC6F8483633E07CF036
:10B2A000DDFCD6F8E836C01A42F2107398427FF6F9
:10B2B0007DAFF0EE087AF4EEE7AAF1EE10FA7FF730
:10B2C00075AFBCEEC88A04F5F67718EE103A9BB25B
:10B2D00008EE103AB8EEC88AB4EEC89AF1EE10FA49
:10B2E00047D853F0E9FF404A06214DF00DF904F527
:10B2F000EE730FCB87E80F000123EB740321A4F555
:10B30000C040F6F76DFE304803F05EFF28B12E48CE
:10B310000321F6F765FE0023EB74D6F8DC36012B2B
:10B3200040F0B180D4F8E031AA699FED29AA9B1AB8
:10B3300007EE903AD6F848360133F8EEE79A5BD03C
:10B34000DFED2A7AE9EE0A7AF4EEE79AF1EE10FAE6
:10B350000ADA274905F114000CF002FDF4EEC08A68
:10B36000F1EE10FA00F28F8017480321F6F738FE4D
:10B3700089E053F0A1FF1F4A06214DF0C5F804F5FE
:10B38000EE7C9CE80F0005F1140E8EE80F009CE89F
:10B390000F0087E80F00D4ED7C7A39EE488AF8EE8A
:10B3A000E77AF0EE680AE8EE0A7A3846B0EE690A03
:10B3B000FDEEE77AC4ED7C7A0CF048FD0121E974DA
:10B3C0009DE700BF108C0020102C00200000000022
:10B3D0000000C842E02E6542FC8D0020104C002089
:10B3E0009A99993EF9E00C08B8E00C08000048C3AF
:10B3F000EC8D0020D4E00C08B5F90A3007EE903A45
:10B40000F8EEE77A05F1140767EE8A7AF4EEE79A28
:10B41000F1EE10FA51DB424938460CF071FBDFEDDA
:10B42000417AB6EE008AA0EE278A97E80F00BDEEBB
:10B43000C88A9FED3D0AB8EEC88A04F5F67C28EE6E
:10B44000008A8CE80F00F0EE680A3848B0EE480A2F
:10B450000CF0FCFCD4ED7C7AF8EEE77A28EE0A0AD0
:10B46000E9EE0A7AFDEEE77AC4ED7C7A1EF080F907
:10B47000BDEEC00A10EE103AC6F84836D6F8DC36F3
:10B48000012B3FF45DAF2A4803F07EFE18B1284837
:10B490000321F6F7A5FDD6F8DC36012B17D1244899
:10B4A00003F0F6FB224803F043FD214808B0BDEC51
:10B4B000088BBDE8F04103F04FBC194938460CF049
:10B4C0004FFCF4EEC08AF1EE10FAA4D9D6E795F855
:10B4D00024302BB9174861F0B7FF012385F82430D9
:10B4E0001348F7F7BBFF1248F7F7B6FE1048F7F717
:10B4F00099FC114890F8DC366BB1002380F8DC36FB
:10B5000033220221A0F5405008B0BDEC088BBDE805
:10B51000F041FDF7CDBA08B0BDEC088BBDE8F08175
:10B52000EC8D0020A00CB3450AD7233CFC8D0020F5
:10B53000102C0020204F0020105C002010B5044685
:10B54000FEF724FA2046054B40F8143B0CF0A6F811
:10B55000204603493FF094FC204610BDACE10C08A6
:10B5600044E10C08182070470048704714E20C08AA
:10B57000004870471CE20C0801207047012070470A
:10B580000120704708B50548F7F768FF0348F7F74B
:10B5900063FEBDE808400148F7F744BC102C0020CA
:10B5A00010B5074C204679F0F5FBBCEEC00AA4F5B7
:10B5B000335010EE103ABDE8104099B200F0E4BEEE
:10B5C000D058002010B50D4CD4F8A83E002B12DD49
:10B5D000A4F50050FCF748FBA4F5005000F052FA27
:10B5E00004F54C6079F020FD04F54C60044979F0D5
:10B5F000B9F8012010BD0020FCE700BF104C00206E
:10B60000FC8D002070B5234EF06D03688EB05B6832
:10B610009847072830D00A2809D0062805D106F017
:10B620004DFE90F87C32DB071DD4012019E006F2B4
:10B630003C750FCD07AC0FC495E8070084E8070000
:10B6400009AB0FCB06F5805501AC84E80F00D5F8A7
:10B65000F831009305F5F6730ECBA6F1BC00FFF7A9
:10B6600003FB0EB070BD06F029FE00F51B700FC87D
:10B6700006F5805501ACE8E707A9A6F1F800FFF749
:10B6800039F80028D1D00799A6F1BC00FFF7CAFA13
:10B69000E7E700BF107C0020F0B585B00D4E0391A8
:10B6A000144653F009FE06F5A0470546F86D0268FA
:10B6B00092689047039B0090074A284606214CF069
:10B6C00023FFF96D2246304605B0BDE8F04002F098
:10B6D00059BF00BF102C002024E20C082DE9F047D0
:10B6E0002DED028BDFF8C48196B00024074640465A
:10B6F00079F07AFB05940694079406F0DFFD05A91E
:10B7000006F026FB58B398ED797AB5EEC07AF1EEE3
:10B7100010FA08F50D5927DBDDED067ADDED056A37
:10B7200067EEA77A27EE077AE6EEA67AF4EEC77AF6
:10B73000F1EE10FA18DDD9F85C0003685B689847F1
:10B740000A2811D053F0B8FD544A06214CF0DCFE13
:10B750002622A9F1C401A8F5335002F013FF16B058
:10B76000BDEC028BBDE8F087D9F85CA04C4B01948E
:10B770009A4502940394049417D109F23C760FCEB3
:10B7800008AD0FC596E8070085E8070011A80BF083
:10B7900085FFB9F894170FAA0AF2DC7023F016F8A7
:10B7A00090BB02940194049403949FED3E0A3E4E94
:10B7B00001A820F003F903A88DED080A9FED390ACE
:10B7C000CDED090A20F0FAF838488DED0F0AB0EEF9
:10B7D000401AF0EE601ACDED100A9DED080ADDED7D
:10B7E000090A79F05BFA062804461AD10023C6F844
:10B7F000A0317CF033FA06F5F671C6F88C03A6F595
:10B800004D5078F0AFFFAAE701A911A80CF024F978
:10B810000028C6D003A90AA80CF01EF90028C0D041
:10B82000C3E77CF01BFADFED227A98ED508AD6F858
:10B830008C6328EE278ADFED1F7AB4EEE78AF1EEFB
:10B8400010FA0546384658BFB0EE678AFFF7DAFEB1
:10B8500048B9022C16D0BCEEC88AAD1B18EE103ABF
:10B860009D42FFF47CAF013C062C0ED8DFE804F0CB
:10B87000040A0D0D100D13000F4924223846FFF75E
:10B880000BFF6CE70D492522F8E70D491622F5E775
:10B890000C492622F2E70C490122EFE740E20C08AE
:10B8A000347B00200000C842108C0020D0580020BB
:10B8B00000007A4400409C4666E20C087BE20C08DB
:10B8C00090E20C08A8E20C08BFE20C0803207047C5
:10B8D0000048704744E30C080048704750E30C08E8
:10B8E000F8B52B4D06460027A5F54050A5F8D876AB
:10B8F000F7F71AFD7368A5F58052D3F8F811D2F85E
:10B90000383F994205F5005423DBC4F8F0367368DC
:10B910009FED206AD3ED7F6A02F5916393ED007A83
:10B92000F8EEE66A27EE067AF4EEC76AF1EE10FA50
:10B9300018DBBDEEC77A17EE103A1748C4F8F43694
:10B94000FCF714FF20B1D4F8F4365B42C4F8F436A7
:10B95000F8BD5B429942D8DD012385F8D836C4F89A
:10B96000F076D4E702F63C72D2ED007A67EE867A82
:10B97000F4EEE76AF1EE10FA93BFFDEEE77A0123E9
:10B9800085F8D93617EE903A88BF0023D5E700BF77
:10B99000105C00200000C842102C002070B500216F
:10B9A0002DED028B04463448344D01F06FF83248D7
:10B9B0000021F0EE408A01F073F895F8D836B0EE29
:10B9C000408AD3B1B0EE680A042056F0E9FC95F83D
:10B9D000D93693B3B0EE480A132056F0E1FC26485E
:10B9E000002101F067F82046FEF7C2F8BDEC028B9B
:10B9F0002046BDE87040FEF7CDB805F50056A5F528
:10BA00004050F6F7FDFFD6F8F036002B0CDCD6F8E8
:10BA1000F036002BDBDA042056F0D6FCB4EEE80A50
:10BA2000F1EE10FACED4D2E7042056F0CDFCB4EEFD
:10BA3000E80AF1EE10FAEADDC4E7114D0E48F7F717
:10BA40007BF8D5F8F436002B0CDCD5F8F436002B57
:10BA5000C5DA132056F0B8FCB4EEC80AF1EE10FABD
:10BA6000B8D4BCE7132056F0AFFCB4EEC80AF1EE30
:10BA700010FAEADDAEE700BF102C0020105C0020B9
:10BA8000107C002000F5C0400023C0E9673380F837
:10BA9000A53180F8A631704700F5A043D3F888306F
:10BAA000002BCBBF07EE903A00F51150B8EEE70A35
:10BAB000DFED037ADCBF90ED0D0A20EE270A704718
:10BAC0000000C8422DE9F0412DED028B00F5A25790
:10BAD00084B09FEDD58A054603A938468DED038ACB
:10BAE00006F0D0F905F5A044B0B19FEDD07ADDEDB8
:10BAF000037A04F2FC6367EE877AD3ED006A9FED68
:10BB0000CC7AE6EE877AF4EE487AF1EE10FA48BF86
:10BB1000F0EE487AC3ED007A2846F6F751FEF0EED3
:10BB2000000AB0EE408A9FEDC00A1DF065FFD4ED1B
:10BB3000287A94F86C3038EE678A05F50056E0EE06
:10BB4000087AC4ED287A002B40F01F81A26D05F51C
:10BB50009E439A4203D008339A4240F0168108214E
:10BB60002846F6F7E9FC804640B106F27443D3ED6F
:10BB7000007A9FEDB07A67EE877A01E102212846CC
:10BB8000F6F7DAFC0146002800F0E380D6F8283FFB
:10BB90001B8B2846414608EE103A01F041F9D6F8D1
:10BBA000280F4369B8EE488AB0EE401A002B00F027
:10BBB000B180012B00F0B380DFED9F7AF0EE671AC1
:10BBC00006F2744393ED000A9FED9A7AF4EEC17A7F
:10BBD000F1EE10FA20EE070A4FF06401C0F2AC80DB
:10BBE000B6F8702412FB01F2B0EE672A07EE902A35
:10BBF000F0EE400AB8EEE70A1DF058FDBDEEC00AAF
:10BC000084ED210AA06D03689B6B9847002851D0F2
:10BC100094F89830002B4DD0A36D05F59D4538352F
:10BC2000AB4247D0D4ED217A9FED847AF8EEE77AE3
:10BC3000384627EE878AD4ED257AF8EEE78A68EE53
:10BC4000878A06F02BFBC8EE807A9DED037A77EEAB
:10BC5000877AB6EE007AB4EEE78AF1EE10FA4CBFBE
:10BC600077EEC87ADFED747A77EE877A94ED277AEB
:10BC7000FDEEE77AF8EEE77AB4EEE77AF1EE10FA45
:10BC80000ADD37EE676ADFED6E6AB4EE666AF1EEE2
:10BC900010FA48BFF0EE477A94ED217ADFED656A3D
:10BCA000C4ED277AB8EEC77AA7EEA67ABDEEC77ABA
:10BCB00084ED217AA06D03681B6B984740B1B4F9FD
:10BCC0009020002AC2BFD4F884309B18C4F8843076
:10BCD000B6F97224B6F97014D4F8840064235A4378
:10BCE00059431DF051FEC4F8840006F57D63D6F873
:10BCF000E00F93ED4A8A06F0D1FAC8EE007A9DED86
:10BD0000037A77EEC77AC4ED237A04B0BDEC028BD8
:10BD1000BDE8F081DFED487AF1EE481A50E78DED8D
:10BD2000010A55F01FF807EE900ADFED431A9DED6A
:10BD3000011AF8EEE77A43E7B6F8723413FB01F321
:10BD400000EE903AB0EE482AF8EEE00AF0EE671AFC
:10BD500052E7B6F97024B6F972349B1A07EE903A9E
:10BD60002846B8EEE78A01F05BF8B6F87034642232
:10BD700013FB02F307EE903AF8EEE77AE8EE007A6A
:10BD8000FDEEE77AC4ED217A3CE7D6F8A83E002B19
:10BD900016DD96F8483E9BB1A26D05F59F43103322
:10BDA0009A4219D105F5335079F00EF9B5EEC00A73
:10BDB000F1EE10FADFED1F7A19DD20EE270A1DE7FC
:10BDC000D4F8DC36042B17D105F5C140343077F0B8
:10BDD00025FEC4F8840015E705F59E4324339A42F6
:10BDE0007FF410AF05F5335079F0F2F8DEE706F294
:10BDF000744393ED000AE0E7A26D05F59E434C33D2
:10BE00009A4206D1D4F88830002B02DDC4F8843081
:10BE1000F8E605F59E4324339A427FF4A6AE284601
:10BE2000FFF73AFEEAE600BFCDCCCC3DCDCC4C3E90
:10BE3000CDCC4C3F0000C842000000000AD7233C94
:10BE40009A99993F30B500F5A25587B00023044672
:10BE5000284603930493059305F0C2F8002846D0C2
:10BE600003A9284606F03CF8002840D004F5BB534F
:10BE700093ED007ADFED226A8DED017AB0EEC77A9C
:10BE8000D3ED037AB4EEE67AF1EE10FACDED027A54
:10BE900006D5F0EEE77AF4EEE67AF1EE10FA2DD45C
:10BEA00001A81FF07DFE03A901A81FF0C1FD04F544
:10BEB000115393ED0F7AB5EEC07AF1EE10FAC4BFCC
:10BEC000DFED107A27EEC00A04F5A044C8BFA7EE44
:10BED000270A03F13C03CABF01230023FDEEC07A09
:10BEE00084F89830CCBF17EE903A002304E004F5B4
:10BEF000A044002384F89830C4F8943007B030BDD3
:10BF0000000000340000C8422DE9F04100F5C047B0
:10BF10002DED028B07EE901AD7F8A83100F5C34536
:10BF2000B8EE678A04466C3500F54056B3BB00F5A1
:10BF3000A04200F59E43916D2433994204D000F550
:10BF40009E434C33994229D192F88C3633B304F591
:10BF5000C34029465C300BF003FFD6F8080903689C
:10BF6000F0EE408A5B6AB0EE480A9847F0EE087A35
:10BF700060EE277AF4EEE78AF1EE10FA0EDDBDEC02
:10BF8000028BD6F808099FED0C0A036804F5C3413B
:10BF90002A469B6ABDE8F0414C311847B0EE480A8A
:10BFA000BDEC028BD6F8080997F9A421036829464D
:10BFB000DB6ABDE8F04118470000000070B5044698
:10BFC0002DED048B04F5C0457BF03CFED5F8143212
:10BFD000544AC31A9342064676D907EE903AB8EE11
:10BFE000670ADFED517A9FED511ADFED510A20EE1D
:10BFF000270A40F295101DF027FCC5F8146204F5DD
:10C000000056DFED4C7AD6F8243FB3F9083008EE3D
:10C01000103A96F9CE34B8EEC88AF0EE408A28EE8F
:10C02000278A0BB1B1EE488A9FED437ADFED437A60
:10C03000B4EEC78AF1EE10FA6CDAD5ED846AF4EE4C
:10C04000C76AF1EE10FAB4EEE78AACBF0123002311
:10C05000F1EE10FA5BD995ED847AB4EEE77AF1EE61
:10C0600010FA54D82046FAF7E5FB96F9CF349FED45
:10C07000349A00EE103A04F54052D2ED000AB8EEC0
:10C08000C00A06F6F87393ED001A40F2A710F1EE1D
:10C09000600A20EE080A1DF0D7FB28EE800A204631
:10C0A00020EE090AFDEEC07A17EE901AFAF782FB2D
:10C0B000D6F8A83E002B05DD96F8483E8BB1204609
:10C0C000FAF7B8FB85ED848A2046F9F7E7FF2046AA
:10C0D000F6F7A8FEBDEC048B2046BDE87040F7F7EC
:10C0E000BBB8184BDFED187A93ED007AE7EE097ACA
:10C0F000F0EE678A06F0E2F8D0ED9C7AF8EEE77A87
:10C1000077EEA87AFDEEE77AC5ED7F7ADAE7002BC5
:10C11000A8D1AAE7B4EEE78AF1EE10FAA5D9002378
:10C1200099E700BF9F860100BD3786359A99193E71
:10C13000CDCCCC3D5304693900000034000000B47C
:10C140000000C8429C5A002000007A4470B54FF0AD
:10C15000FF31054600F5AE4022F08EFB431C06463B
:10C1600005F5A04404D104F26464124B236070BD51
:10C1700005F5C34105F5C3406C314C300BF0C0FCF4
:10C180009FED0D7AF6EE007AE0EE077A04F2646431
:10C19000FDEEE77A17EE900A301A1DF01DFB07EE50
:10C1A000900A9FED067AF8EEE77A67EE877AC4ED9B
:10C1B000007ADCE70000B442A00CB3450AD7233C68
:10C1C00000F54050D0F8080903689B6B1847000041
:10C1D000F7B500F540530546D3F8080903681B6915
:10C1E000984707462846FFF7EBFF05F5C04406468B
:10C1F000D4F8A001002860D13EB1D4F8E031C4F8F1
:10C20000AC313D4BC4F8B0310120C4F898711DF039
:10C21000E3FAD4F8A03194F9A42100FB0230C4F869
:10C22000A0012EB30023019394F80432002B48D0D0
:10C2300094F8B030022B44D105F5B040012201A999
:10C24000183046F085F900283BD0D4ED827ADFED36
:10C250002B6AB8EEE77ADDED017AE7EE667AB1EEA9
:10C26000047AF0EEE77AF4EEC77AF1EE10FA33D4FE
:10C2700094F8A531002B3DD1D4F8A031D4F8B021E9
:10C28000002BB8BF5B42934234DBD4F8E011D4F802
:10C29000AC31C4F8AC11CB1A03F2F31340F2E63020
:10C2A000834202F5D2328CBF0023012302F5F072E3
:10C2B00084F8A631C4F8B0211CE0D4F89831F81AFB
:10C2C000A3E7D4F8FC21D4F8E0319B1A03F2F3136E
:10C2D00040F2E6329342CBD8012384F8A531002303
:10C2E00084F8A631D4F8A03103F5D23303F5F07306
:10C2F000C4F8B03103B0F0BDE0A501000AD7233C7B
:10C300002DE9F04100F5A045044695F88130BBB316
:10C3100000F5C043D3F8F42112B9D3F8F8317BB358
:10C3200004F5C34604F5C34720465C366C37FAF77C
:10C33000AFFD394630460BF013FD05F5CE6304F52D
:10C34000C3413A464C31304683ED000A0BF03EFCC7
:10C3500005F27463DFED0B0A83ED000A7620B7EE79
:10C36000001A1DF071FA04F53F53204683ED750A5B
:10C37000FFF72EFFA86D0368BDE8F041DB6A1847A0
:10C38000BDE8F08100000000012970B5044600F509
:10C39000C04512D800F5005395F8EC21B3F99A3452
:10C3A00083EAE371A1EBE37189B2012998BF3C21D3
:10C3B000920730D5FF2385F8A43107EE901AF8EEE6
:10C3C000677A2046C5ED6E7AFFF79EFDD5F8A83155
:10C3D0003BBB2046FFF7F4FE04F5A04650B906F239
:10C3E000746393ED007AF7EE007AB4EEE77AF1EE3B
:10C3F00010FA16DD7BF032FCC5F8A801B06D0368B9
:10C400001B6A984768B104F55B500021BDE8704095
:10C41000203050F069BA002BB4BF4FF0FF33012336
:10C42000C9E770BD10B500F5AF44783420465CF024
:10C4300091FC2046BDE810405CF0FCBC10B500F556
:10C44000A043044693F80C389A0717D45B0700F50D
:10C450005B504FF002014CBF094A0A4A20304CF0B1
:10C4600053F804F5AF4078305CF048FC04F53B50DD
:10C470000121BDE810400C3062F0A8BF10BD00BF24
:10C48000C8E30C08E2E30C0870B500F5A0460546C9
:10C4900096F9F8479CB196F80C38C3F380045B0713
:10C4A00029D4B6F9FE37002B0BDC2846FFF7C6FF70
:10C4B00005F53B5001210C3062F088FF0124204635
:10C4C00070BD2146F9F7D2FDB6F9FE3707EE903A76
:10C4D000F8EEE77AB4EEE70AF1EE10FAE5D5D6F811
:10C4E0007836002BE1D005F55B50044A042120305A
:10C4F0004CF00AF8E3E70024E1E700BFF8E30C089A
:10C5000008B52DED028B08EE901A30B3F2B1B0F9F8
:10C51000083008EE103AB8EEC88AF8EEE88A9FEDC7
:10C52000100ADFED100A28EE800ADFED0F8A4FF4C3
:10C53000D470B7EE001A1DF087F9C8EE280A1DF076
:10C54000DFF820EE280ABDEC028B08BD54F08EFC0B
:10C5500007EE900AB8EEE78ADFE79FED020AF2E7FE
:10C560000AD7233C0000000000A08C4537B500F539
:10C570000054054694F9FB34002B52D054F090FB44
:10C5800054F084FBC4F8200F54F08AFB54F06AFB8B
:10C59000C4F8240F54F084FB54F06EFBC4F8280F49
:10C5A00054F07EFB54F072FB41F29411C4F82C0F4E
:10C5B000D4F8200F54F0BEFBD4F8240F41F29411AC
:10C5C00054F0B8FBD4F82C0F41F2941154F0B2FBA4
:10C5D000284600F01FFC48BBD4F8280F642154F013
:10C5E000A5FB54F05DFBD02155F08CFBC4F8300F57
:10C5F00054F056FBD22155F085FBC4F8340F05F5F5
:10C60000225024304921019056F00AF901984A211C
:10C6100056F006F90198462103B0BDE8304056F0C7
:10C62000FFB854F03DFB54F013FBABE705F5C043F6
:10C63000D4F8280F93F89433642173B154F076FB47
:10C640006421462055F0E4FF6421492055F0E0FFC5
:10C6500064214A2055F0DCFFC3E754F06BFBEFE7A1
:10C6600010B500F500541E21D4F8200F54F066FBDD
:10C67000D4F8240F1E2154F061FBD4F82C0F1E2196
:10C6800054F05CFBD4F8280F1E21BDE8104054F094
:10C6900055BB000007B500F0BDFB014658B901903D
:10C6A000462055F0D7FE0199492055F0D3FE019957
:10C6B0004A2055F0CFFE0021042056F09DF90021BC
:10C6C000132056F099F90021462056F095F90021E3
:10C6D000492056F091F900214A2056F08DF90021A9
:10C6E000152003B05DF804EB56F086B910B504468A
:10C6F00056F0C8FB56F018F8204601F0CFFCBDE814
:10C70000104056F0C7BA000038B500F50055044691
:10C7100095F9FB340BB1002038BD0121F5F70CFF72
:10C7200088B104F5A0439A6D04F59E4360339A42A4
:10C7300009D004F59D4340339A4204D004F59D434B
:10C7400050339A42E7D12046F6F7EAF80028E2D0C3
:10C75000D5F82C3FB3F90800DEE7000038B52DED21
:10C76000028B00F5A04393F86C30002B40F0B880AA
:10C770005D4A00F59E43926D603300F55B549A422A
:10C7800004F1200408D0594A0321BDEC028B204655
:10C79000BDE838404BF0B8BE00F500559FED546A37
:10C7A000D5F8202FB2F90830002BB8BF5B429BB2FE
:10C7B00007EE903A138B06EE903AF8EEE66AF8EE42
:10C7C000E77A66EE866AF4EEE67AF1EE10FA17DCA6
:10C7D000D5F8242FB2F90830002BB8BF5B429BB2CA
:10C7E00007EE903A138B07EE103AB8EEC77AF8EEE0
:10C7F000E77A27EE067AF4EEC77AF1EE10FA01DD59
:10C800003C4AC1E700F5BA5014301FF001FFDFEDDC
:10C810003A7A20EE270AF3EE0E7AB4EEE70AF1EE4A
:10C8200010FA01DD354AAFE7042056F09DF81320D9
:10C8300056F09AF8152056F097F84D2056F094F8D7
:10C840004E2056F091F84F2056F08EF8502056F0BA
:10C850008BF8152055F0B8FD9FED298AB0EEC00A7F
:10C86000B4EEC80AF1EE10FA0BD5102056F07CF8A1
:10C87000562056F079F8112056F076F8572056F0E9
:10C8800073F8032055F0B0FDB0EEC00AB4EEC80A4C
:10C89000F1EE10FA0FD5022055F0A6FDB0EEC00A59
:10C8A000B4EEC80AF1EE10FA05D5182056F05CF87F
:10C8B000192056F059F8D5F8200F811D0C303FF0A3
:10C8C000A5F9D5F8240F811D0C303FF09FF9D5F85C
:10C8D0002C0F811D0C303FF099F90A4A052154E7CD
:10C8E000BDEC028B38BD00BF107C00200CE40C08AE
:10C8F000CDCC4C3E2CE40C08E02E654254E40C08F0
:10C900000000003470E40C0810B500F5005494F9F0
:10C91000D2349BB1D4F8280F54F01EFAD4F8282F43
:10C92000B4F9D43430B1B2F906009842ACBF00205B
:10C93000012010BDB2F906008342F7E70120F8E7B5
:10C9400010B50446FFF7E0FF58B104F5A0447BF0B2
:10C9500085F9A36FC01AB0F57A7F94BF002001203B
:10C9600010BD0120FCE7000070B50546FFF7E8FFA9
:10C9700005F5005400B3D4F8203F9A89DA80D4F842
:10C98000243F9A89DA80D4F82C3F9A89DA80D4F847
:10C99000203F00261E81D4F8243F1E81D4F82C3F6E
:10C9A0001E8105F5A043986DC3F8906003685B682D
:10C9B0009847D4F8283F1E8105F5C5406C3071F0CA
:10C9C000C3FA80B3002654F06BF9437A13B954F0DC
:10C9D00067F9837A94F9D224012A23D106B10BB3E3
:10C9E0002846FFF7ADFF05F5A04494F8723038B340
:10C9F0000133DBB20A2B84F872300CD105F55B50A1
:10CA00001E4B1F4A042120304BF07EFD1D4A01239E
:10CA100084F86C30937294F872300A2B02D90A238E
:10CA200084F8723070BD2846FCF7D0FB0028C9D1CD
:10CA300054F036F954F0F8F8061E18BF0126C2E784
:10CA4000002BEFD0013BDBB2032B88BF032384F81C
:10CA5000723094F87230012B09D105F55B500A4B06
:10CA6000074ABDE87040042120304BF04DBD002B3B
:10CA7000D8D1044A84F86C309372D3E7BF410E08D2
:10CA800080E40C085D9000208BE60C0800F5005057
:10CA90000A4690F9061FD0F8200FFFF731BD0000BD
:10CAA00000F500500A4690F9071FD0F8240FFFF751
:10CAB00027BD000000F500500A4690F9081FD0F885
:10CAC0002C0FFFF71DBD000010B54FF48061044628
:10CAD000F5F732FD04F5005328B1BDE81040D3F856
:10CAE000280F54F0BFBABDE81040D3F8280F54F017
:10CAF000C3BA00002DE9F04100F500530546D3F814
:10CB00002C3FB3F9088000F5C044B8F1000F02D102
:10CB1000012384F8303305F5C5476C37384671F08A
:10CB200013FA0646F8B9B8F57A6F2EDD7BF096F861
:10CB3000D4F82C33804693B1C31A40F6B7329342EF
:10CB40000FD905F5A045012231463846F4F7F4FE29
:10CB5000C4F82C6384F83063C5F8208601E0C4F87B
:10CB60002C03BDE8F08118F57A6F0EDA7BF076F8C9
:10CB7000D4F82C336BB1C01A40F6B7339842F0D9D1
:10CB8000012200213846F4F7FDFE0023C4F82C33BF
:10CB9000E7E7C4F82C03E4E770B52DED028B0446FB
:10CBA00054F07EF853F036FF30B9BDEC028B2046CE
:10CBB000BDE87040FFF7D8BE04F5A04595F86C308D
:10CBC00013B97BF04BF8E8672046FFF79DFE10B1E4
:10CBD0007BF044F8A8672046FFF7C6FE2046FCF726
:10CBE00087F904F500560023C5F8903096F9D6343D
:10CBF0006BB3D6F8283FB3F90830322B27DD30B3BA
:10CC0000323B1BB207EE903AB8EEE78ADFED217AAD
:10CC100004F5A25028EE278A04F01CF940B3B6F9B7
:10CC2000723407EE903A06F2744696ED007AF8EE0A
:10CC3000E77A77EEC77A27EE888ADFED177A28EE53
:10CC4000278ABDEEC88A18EE103AA5F89030204623
:10CC5000FFF750FFA86D03685B689847BDEC028B37
:10CC6000014604F5C6403830BDE8704056F088BB38
:10CC700096F9653496F967249B1A07EE903AF8EE18
:10CC8000E77A27EE888ABDEEC88A18EE103AA5F832
:10CC90009230DCE70AD7A33C0000C84270B500F52B
:10CCA0000054D4F8D8340BB9002040E094F964342F
:10CCB000002BF9DA00F5A045A86D03685B6898477A
:10CCC0000138172832D801A353F820F0C5CD010848
:10CCD00001CE01082DCD0108F7CD0108EDCD0108E9
:10CCE000D9CD0108CFCD01082DCD01082DCD0108EA
:10CCF00031CD0108BBCD0108B1CD0108A9CC010897
:10CD0000E3CD0108E3CD01082DCD01082DCD0108AB
:10CD10002DCD01082DCD01082DCD01082DCD010807
:10CD20002DCD01082DCD01080BCE0108012070BDCD
:10CD3000B5F83E67162EB7D0D4F8D81411F0020318
:10CD400001F0010205D0A6F1150CDCF1000343EB64
:10CD50000C0311F0040043EA020303D0A6F11F0400
:10CD60006042604143EA000211F0080007D01F2E24
:10CD70001AD0A6F1110002288CBF0020012011F06A
:10CD8000100340EA020005D0102E0FD0A6F1520287
:10CD900053425341034311F4006014BF95F8081740
:10CDA000014643EA0100C2E70120E8E70123F1E779
:10CDB000D4F8D804C0F34010B9E7D4F8D804C0F3CD
:10CDC0008010B4E7D4F8D804C0F3C010AFE7D4F8AB
:10CDD000D804C0F30020AAE7D4F8D804C0F3402058
:10CDE000A5E7D4F8D804C0F38020A0E7D4F8D8048D
:10CDF000C0F300309BE7D4F8D804C0F3403096E786
:10CE0000D4F8D804C0F3803091E7D4F8D804C0F344
:10CE1000C0308CE700F5005090F86404C0097047FA
:10CE200038B504460D4653F03BFF0368DB6898476E
:10CE3000C8B104F50053D3F8280F6DB154F016F8BB
:10CE400007EE900AB8EEE70A04F5C04494F893336D
:10CE50000BB1B1EE400A38BDB0F9083000EE103A1F
:10CE6000B8EEC00AF0E79FED010AF4E70000000009
:10CE700038B52DED028B04460D4653F011FF0368C3
:10CE8000DB68984700283FD0214BD3F8283F5B69E7
:10CE9000012B07D0BDEC028B29462046BDE8384067
:10CEA000FFF7BEBF4FF480612046F5F745FB002831
:10CEB000F0D004F50053DFED177AD3F8280F93F97B
:10CEC0006734028B08EE903A00EE102AF8EEE88AFA
:10CED000B8EEC08A68EEA78A53F0D2FFB6EE001A09
:10CEE000A0EE011A04F5C044DFED0B0AB0EE680AAB
:10CEF0001CF0D8FC94F8933328EE000A0BB1B1EE85
:10CF0000400ABDEC028B38BD9FED030AF9E700BF74
:10CF1000104C00200AD7233C0000000073B500F538
:10CF2000C046044696F8B030022B00F5736512D166
:10CF300000F5B040012201A9183045F009FB50B1BD
:10CF4000019BC5F89C3228463FF0ECFA2046F9F7E1
:10CF5000F5FD02B070BD04F5A043D3F8DC36042B18
:10CF600005D12046F9F7D0FA8DED010AE8E7D6F8A9
:10CF700018320193E4E7000070B500F5A0450446BF
:10CF8000A86D03689B6B0E46984748B9D4ED460AD6
:10CF90009FED1A0A64213046BDE8704055F0F6BA9C
:10CFA000A86D04F59E4104F500522431884292F8A0
:10CFB000663492F930251DD195F8881641B93AB1F9
:10CFC000D3B2D5F8DC160139012998BFD3B209E0F4
:10CFD00004F5C04191F9301161B1D5F8DC0604289F
:10CFE00008D1CBB207EE903AD4ED460AB8EE670A04
:10CFF0006421D0E7002AF5D0E3E700BF000000007D
:10D000002DE9F04100F5A046044604F59E43B06DBD
:10D010006033984203D100252846BDE8F0810368BB
:10D020009B6B984740B196F80C5815F0010503D05A
:10D03000012386F8D436EFE704F5C140343076F0AA
:10D0400021FE054608B10125E6E796F8D436002B07
:10D05000E1D0B06D03689B6B984708B90023E8E7FF
:10D0600094F8143494F85874B02202FB034393F8F4
:10D07000F121B7BB012A0AD993ED837AF1EE047A44
:10D08000B4EEE77AF1EE10FAACBF01270027B26DDB
:10D0900004F59E4324339A4202D196F8883623B190
:10D0A00004F59E4368339A4241D104F5005320466B
:10D0B00093F92485FCF78AF8A8B9204601F06CFCA6
:10D0C0000028C0D0002386F8D43694F8711404F5F3
:10D0D0008C63242000FB013304F5AD42DB6A13604E
:10D0E0009AE72F46D3E77AF0B9FDD6F8E8364FF441
:10D0F000FA62C01A642313FB082341F28832934278
:10D1000038BF13469842D8D92046F9F781F9B0F5CF
:10D11000FA7FD2DD04F5805341F26E72D3F83C36CB
:10D1200003F6B7339342C8D8002FC6D096E704F56C
:10D13000C043D3ED867AB2EE047AF0EEE77AF4EEED
:10D14000C77AF1EE10FA89DA002F3FF47CAF04F5CC
:10D15000A25003F07FFE002880D004F5005304F5B0
:10D16000055093F88E1203F085F8F1EE047AB4EED0
:10D17000E70AF1EE10FAFFF666AF6FE7F8B52DEDAE
:10D18000048B0446084617461D46BDF9286055F035
:10D190001BF904F500543846B0EE408A55F014F9F6
:10D1A000B4F90025002AF0EE408A39DAC2F16403AE
:10D1B00007EE903A9FED217AF8EEE77A67EE877AEC
:10D1C00060EE278A04F2FC44D4ED007A9FED1C1A2D
:10D1D000DFED1C0A38EEC80ABC2020EE270A1CF03E
:10D1E00033FB38EE288AB0EE409A94ED000A9FEDAA
:10D1F000141ADFED140A28EE000ABD201CF024FBEF
:10D200002846B0EE408AB0EE490A55F0C9F8B0EEB3
:10D21000480ABDEC048B3046BDE8F84055F0C0B874
:10D22000D0D002F1640307EE903A9FED047AF8EE55
:10D23000E77A67EE877A28EE278AC3E70AD7233C86
:10D2400000A08C4500A08CC500B52DED048B0420FA
:10D2500083B055F0B9F80320B0EE408A55F0C4F819
:10D26000DFED189A9FED181ADFED180A8DED011AFF
:10D27000F0EE408AB0EE480AA8EEA90ACF20CDED24
:10D28000000A1CF0E1FAB0EE409AB0EE480A9DEDBB
:10D29000011ADDED000AA8EEE90AD0201CF0D4FA4C
:10D2A0001820B0EE408AB0EE490A55F079F8B0EE99
:10D2B000480A192003B0BDEC048B5DF804EB55F06F
:10D2C0006FB800BF0000344200A08C4500A08CC5A0
:10D2D000F8B52DED088B00F5005600F5C04596F920
:10D2E000EE3E13F0040F03F0010203F0020440F0DD
:10D2F000F580D5F898737B1E5F425F41002A00F0ED
:10D30000EF804D2055F060F84E20F0EE409A55F039
:10D310005BF8B0EE408AB6F90235DFED87AA0AEE77
:10D32000103A1520B8EECAAA55F04EF82AEE2AAAED
:10D3300020EE0AAA002C00F0DB80F0EE488AB0EE66
:10D34000699AB5EEC0AAF1EE10FA40F3D6809FEDCF
:10D350007B1ADFED7B0A38EE0A0A4FF480701CF06E
:10D3600073FA9FED761ADFED760AB0EE408A40F24E
:10D37000011038EECA0A1CF067FAF0EE408A96F9FE
:10D38000EF3E632B15DC07EE903A9FED6E7AF8EED8
:10D39000E77AB4EEC79A67EEAA7AF1EE10FAF4EEE5
:10D3A000C78A98BF29EE279AF1EE10FA98BF68EE67
:10D3B000A78AD5F8983396F9EC4E96F9ED6E022BC4
:10D3C00000F0B48024B2002C01DC002E6EDD0320BE
:10D3D00055F00AF8DFED5C7AB4EEE70AF1EE10FAE8
:10D3E000B0EE40AA62DB002F00F0A2809FED571A3A
:10D3F000DFED570A40F2271030EE000A1CF024FA45
:10D400009FED541ADFED520AB0EE40BA4FF494701B
:10D410003AEE410A1CF018FA70EE007AB0EE4BAA10
:10D4200007EE104AF8EEC7AA9FED4BBA9FED431ADC
:10D43000DFED430A6AEEA7AAB0EE690A40F22B10AC
:10D44000AAEE8B0A1CF000FA07EE906AF0EE409A02
:10D45000B8EEE70A9FED391ADFED390A2AEE40AA45
:10D46000B0EE490A4FF49670AAEE0B0A1CF0ECF9E4
:10D47000B0EE409AB0EE480A9FED301ADFED300A68
:10D4800040F22D10AAEE8B0A1CF0DEF9B0EE408AB5
:10D49000B0EE680AAAEE0B0A4FF497709FED271AB8
:10D4A000DFED270A1CF0D0F9F0EE408AB0EE690AF1
:10D4B000102054F075FFB0EE490A562054F070FF6A
:10D4C000B0EE480A112054F06BFFB0EE680ABDECD4
:10D4D000088B5720BDE8F84054F062BF01270DE7E4
:10D4E000042054F071FFB0EE408AF1EE409A12E74A
:10D4F000DFED178AB0EE689A23E79FED101ADFED93
:10D50000100A39EECA0A4FF482701CF09DF99FEDA3
:10D510000B1ADFED0B0AF0EE409A40F2051039EEDF
:10D520000A0A1CF091F9B0EE409A28E700244CE773
:10D53000F0EE407A74E700BF0AD7233C00A08C4588
:10D5400000A08CC5000000B4000000340000C842F8
:10D5500000000000000048426666E63E38B52DED4A
:10D56000028B00F500550446D5F8340FA0B304F53E
:10D57000A04393F86C207ABB93F8723063BB53F0EE
:10D580003BFD07EE900AB8EE678A462095F9645491
:10D5900054F01AFF002DF0EE408A20DA04F5C14065
:10D5A000343076F0F1F9E8B99FED101ADFED100A8A
:10D5B00040F25110B1EE680A1CF046F9B4EE408A10
:10D5C000F1EE10FAC8BFB0EE480ABDEC028B6E2037
:10D5D000BDE8384054F0E4BE9FED058AD5E79FEDE5
:10D5E000040AEBE79FED010AE8E700BF0000C8422C
:10D5F0000000000010B52DED028B4369002B4AD0CE
:10D60000037C0BB101330374037C002B41D0182B36
:10D610001FD803EB4303C3EB03139B001CB200238F
:10D6200007EE903AB8EEE78A0420B0EE480A54F0CC
:10D63000B7FE07EE904A1320B8EEE70A54F0B0FEAA
:10D64000B0EE480ABDEC028B1520BDE8104054F046
:10D65000A7BE4A2B02D8C3F13203DAE7632B01D805
:10D66000643BD6E77C2B08D8643B03EB4303C3EB56
:10D6700003139B001BB20024D2E7AE2B02D8C3F1E8
:10D680009603F2E7C72B01D8C83BEEE700230374EB
:10D69000F1E71C46C4E7BDEC028B10BD10B59FED51
:10D6A0001C7AD0ED017AF4EEC77A0023F1EE10FA7D
:10D6B000044643722BDB90ED007AB4EEE77AF1EE8C
:10D6C00010FA24D908F038FB217A07F089FFD4ED4D
:10D6D000010AF5EE007A60EEA77AB4EEE70AF1EE01
:10D6E00010FA14D494ED001A40F2A5101CF0ACF816
:10D6F000F7EE007AB4EEE70AF1EE10FA07D494EDF3
:10D70000007AC7EE007A01236372C4ED037A10BD7C
:10D7100000000034437A7BB391F9003090ED037A36
:10D7200007EE903AF8EEE77A67EE877A9FED137A84
:10D73000F4EEC77AF1EE10FAD8BFF0EE477AFDEEBC
:10D74000E77A17EE903A0B7092F9003090ED037A79
:10D7500007EE903AF8EEE77A67EE877A9FED087A5F
:10D76000F4EEC77AF1EE10FA58BFF0EE477AFDEE0C
:10D77000E77A17EE903A1370704700BF0000C8C2F6
:10D780000000C842437AF0EE407A5BB190ED030AA4
:10D790009FED051ADFED050A27EE800A4FF4E670CB
:10D7A0001CF052B8704700BF0000C8420000C8C259
:10D7B000F8B504460E4617467AF050FA054604F5C9
:10D7C000A140243008F096F804F5A044D8B34620D0
:10D7D00054F0FAFDDFED3D7AB4EEE70AF1EE10FA0F
:10D7E00010DB97F9002094F9D536193A934209DAFB
:10D7F000D4F8D826AA4205D0C4F8D856013384F804
:10D80000D53644E0462054F0DFFDDFED317AB4EE4A
:10D81000E70AF1EE10FA3AD896F90020002A36DA33
:10D82000C2F1FF2294F9D63602F57F02E732934225
:10D830002DDAD4F8D826AA4229D0C4F8D856013314
:10D8400084F8D63623E0D4F8D836EB1AB3F57A7FCD
:10D850001DD3462054F0B8FD94F9D53607EE903A22
:10D86000F8EEE77AB4EEE70AF1EE10FA01DD002BEC
:10D8700022DC462054F0A8FD94F9D63607EE903A03
:10D88000F8EEE77AB4EEE70AF1EE10FA18D497F959
:10D89000000094F9D5260021821A1CF085F8387012
:10D8A00096F90000002806DA94F9D6160022014401
:10D8B0001CF07AF83070F8BDC4F8D856013B9EE7EA
:10D8C000002BE4DDC4F8D856013BB9E70000003472
:10D8D000000000B410B52DED028B00F5005282B0AF
:10D8E00092F9643492F865248DF80630002B0446D2
:10D8F000B0EE408A8DF8072004DAFFF7CFF908B9B7
:10D900008DF8060004F5A043D3F8DC26012A4CD09C
:10D91000072A4AD004F5C140343076F035F80028A3
:10D9200058D104F53B500DF106010DF107023030DE
:10D93000FFF7F0FE2046FFF73BFF9DF906309DF90B
:10D940000720DFED258A9342A8BF134607EE903AE1
:10D9500004F53F54B8EEE70A103420EE280A2046BA
:10D960008DF8063075F008FA9DF9073000EE103A90
:10D97000B8EEC00A204620EE280A75F007FA9DF995
:10D98000073001EE103A9DF9063000EE903AB8EEFD
:10D99000C11AF8EEE00A40F24D20B0EE480A1BF042
:10D9A00053FF02B0BDEC028B10BD03F5C762D2ED90
:10D9B000007AFDEEE77A03F23C6317EE902AD3ED8E
:10D9C000007A8DF80720FDEEE77A17EE903A8DF891
:10D9D0000630A6E70023FAE70AD7233C70B50446D1
:10D9E00000F53B55303504F5A0462846FFF756FEB6
:10D9F000B06D03685B6D984740B1462054F0E4FC7D
:10DA00002846FFF7BFFE462054F0CAFCB06D0368FD
:10DA10001B6D984740B1462054F0D6FC2046FFF7D6
:10DA200059FF462054F0BCFC2046FFF7E9FA10B33A
:10DA300004F5005595F9D03443B101212046FFF794
:10DA4000EFF9BDE87040462054F0AABC04F5C1448B
:10DA50003434204675F098FF50B1204676F01CF91A
:10DA600030B195F9643400EE103AB8EEC00AE8E738
:10DA70009FED010AE5E770BD0000000010B5044607
:10DA80002DED028B462054F09FFC2046B0EE408ADC
:10DA9000FBF79CFB80BB04F5C5406C3070F054FA7A
:10DAA00050B304F5A253D3ED968A1BF04BF990F8CE
:10DAB000EC349FED137A0C2202FB0300D0ED807A48
:10DAC000E8EEC77AF4EEC77AF1EE10FA0CDC04F552
:10DAD000005494F9673407EE903AF8EEE77AF4EEE2
:10DAE000C87AF1EE10FA07D5BDEC028B0548BDE807
:10DAF0001040012104F056BEBDEC028B10BD00BFEA
:10DB00000AE81C41504000202DE9F34100F5005582
:10DB10000646D5F8303F002B41D1002706F5A04836
:10DB2000D8F8580003689B6B9847044600285FD0DC
:10DB300006F5A25003F08EF900283DD0D8ED217AE9
:10DB40009FED487AF8EEE77A67EE877AFDEEE77A9E
:10DB500017EE903A1BB295F917250AB19A422EDAC0
:10DB600095F9154574BBD8F8582006F59F43103336
:10DB70009A4209D105F56A63D3ED007AFDEEE77AA2
:10DB8000CDED017A9DF90440D8F8DC36013B062B37
:10DB90002ED8DFE803F01E2D24612D2D1E0053F03A
:10DBA0007FF80368DB6898470028B6D0D5F8300FB7
:10DBB00053F022FA47B2B1E795F96734CBE795F90C
:10DBC0001645D0E724B29C42ACBF95F91445002419
:10DBD000C9E795F91835002B18BF1C4608E095F9E0
:10DBE00018352BB13046FBF711FB08B195F91845F4
:10DBF00087EAE773A3EBE773DBB2A342C8BF3C46F7
:10DC000007EE904A0320B8EEE70A54F0C9FB07EE8E
:10DC1000907A0220B8EEE70A54F0C2FB95F9493534
:10DC2000D6ED460A00EE103A6421B8EEC00A032091
:10DC300054F0ACFC95F94935D6ED460A00EE103AA1
:10DC40006421B8EEC00A022054F0A0FC304602B0B5
:10DC5000BDE8F041FFF7F8BA06F5C04393F92F315C
:10DC6000B9E700BF0AD7233C38B504462DED048B35
:10DC7000462054F0A9FB584BDFED587A93F9B83E93
:10DC800008EE903AF8EEE88A152068EEA78AB0EE22
:10DC9000408A54F099FB9FED527A20EE280A04F551
:10DCA000C045C0EE077A04F5C2404030C5EDE27AC7
:10DCB00072F0C6FE10B10023C5F88833B5EEC08AF5
:10DCC000F1EE10FA43D52046FFF7A4F800287ED0E5
:10DCD0002046FEF7E3FF002879D0D5EDE27A9FEDEC
:10DCE000419A9FED411ADFED410AB0EE480AA7EED6
:10DCF000890A4FF43B701BF0A7FDD5EDE27A9FED4A
:10DD00003A1ADFED3A0AF0EE408A40F2ED20B0EE2A
:10DD1000480AA7EEC90A1BF097FDB0EE408A04F549
:10DD2000C5456C35284670F019F9D0BB284671F00E
:10DD3000DBF9022827D10321492054F08BFEBDECEA
:10DD4000048B0321BDE838404A2054F083BE3ED9FD
:10DD5000D5EDE27A9FED239A9FED251ADFED220A99
:10DD6000B0EE480AA7EE890A40F2F2201BF06CFDE3
:10DD7000D5EDE27A9FED1E1ADFED1B0AF0EE408A28
:10DD800040F2F320C3E79FED180A492054F008FB46
:10DD9000BDEC048B9FED140ABDE838404A2054F0D6
:10DDA000FFBAB0EE680A492054F0FAFAB0EE480A19
:10DDB0004A2054F0F5FA20464921FFF7DDF8BDEC82
:10DDC000048B20464A21BDE83840FFF7D5B89FEDC7
:10DDD000068AF0EE488AA2E7104C00200AD7233CBE
:10DDE00000A08C4500004842000000000000C8C2AE
:10DDF0000000C842F8B52DED028B00F5C046044680
:10DE000096F92D31002B31DD00F5A04200F59E433F
:10DE1000926D24339A4229D196F92C31002B25DDBD
:10DE200000F5C140343075F021FEF8B104F5C5406D
:10DE30006C3070F089F8C8B9124F9FED138A044610
:10DE40003D682D190ED0B5F9080054F0CFF848B14F
:10DE500096F92D31012B0CD1B5F90800B0EE480A26
:10DE600054F09EFA1434B4F5A07FE9D1BDEC028BD6
:10DE7000F8BD022BF6D1B5F90800032154F0EAFDF4
:10DE8000F0E700BFEC9400200000000037B500F57B
:10DE9000A043044693F834360BB39FED120A1520C5
:10DEA0004F2554F07DFA204600955023132215216A
:10DEB000FFF764F9152054F015FD80B9284654F099
:10DEC00011FD60B99FED070A4E2054F069FA9FEDED
:10DED000050A4D2003B0BDE8304054F061BA03B0EC
:10DEE00030BD00BF0000000070470000F8B52DED08
:10DEF000048B00F5A0440546A06D03689B6B984712
:10DF000030B9A26D05F59D4378339A4240F0C08048
:10DF100005F5C5406C3070F021F8002800F0B8809D
:10DF20002846FBF753F9002800F0B280D4F8F03609
:10DF3000002BB8BF5B42B3F52F7F00F3A980D4F864
:10DF4000F436002BB8BF5B42B3F52F7F00F3A080FF
:10DF500005F5C04779F082FED7F85832C31AB3F5F9
:10DF6000FA7F0646C0F0948005F5C25393ED017A1E
:10DF7000F2EE007AB4EEE77AF1EE10FA00F1888062
:10DF800004F2FC6494ED007AB4EEE77AF1EE10FA54
:10DF90007ED405F5405393EDE38A05F5225403F54D
:10DFA0009B63D3ED048A2434B0EE480A0421204652
:10DFB00054F06CFAB0EE680A1321204654F066FA69
:10DFC00078EEC89A4D21B0EE690A204654F05EFA08
:10DFD00038EE289A4E21B0EE490A204654F056FAFF
:10DFE000B0EE680A4F21204654F050FAB0EE680AAD
:10DFF0005021204654F04AFA05F50055B0EE480A83
:10E000001821204654F042FAB0EE480A1921204661
:10E0100054F03CFA95F9EE3E03F00202DB075CBFD8
:10E02000F1EE489AB0EE489A6AB3B0EE498AF0EE43
:10E03000698AB0EE690A1021204654F027FAB0EE42
:10E04000680A5621204654F021FAB0EE490A1121FF
:10E05000204654F01BFAB0EE480A5721204654F0EF
:10E0600015FAD7F85C32C7F85862F31A42F2107208
:10E0700093420DD9C7F85C62BDEC048B2046BDE825
:10E08000F84054F0E9BD9FED048AF0EE488AD0E7ED
:10E09000BDEC048BF8BD00BF0000000073B5044662
:10E0A00054F0F0FE054654F083FE2046FFF7DCFDF9
:10E0B0004E23009313224D2304212046FFF75EF8E0
:10E0C0004F2315211322009320465023FFF756F8C3
:10E0D0002046FFF7FDF82046FFF78CFE4FF4005175
:10E0E0002046F4F729FA10B12046FFF7CFFE04F5D9
:10E0F0000056D6F8BC0E48B104F5A04204F59E4384
:10E10000926D60339A4201D154F024F954F0E6FD47
:10E1100054F03AF8284654F053FE96F9903C2BB14F
:10E12000204602B0BDE87040FFF7E0BE02B070BD0F
:10E1300073B5044604F5C24554F0A4FE403554F0CE
:10E1400037FE284672F07CFC002865D104F5A04615
:10E15000D6F8DC36042B04D104F5C140343075F018
:10E160003FFC2046FFF73AFCB26D04F59E43603356
:10E1700004F5C5459A4205F16C0523D028466FF099
:10E18000EDFEF8B99FED320A462054F009F99FEDF3
:10E19000300A492054F004F99FED2D0A4A2054F02A
:10E1A000FFF8284670F0A0FF02280BD1032146207B
:10E1B00054F050FC0321492054F04CFC03214A2028
:10E1C00054F048FC2046FFF759FC2046FFF79CFC22
:10E1D0002046FFF7C3F920464621FEF7CDFE28462C
:10E1E0006FF0B2FE90B90190284670F07DFF68B1E3
:10E1F00002281CD10199462054F098FB019949202E
:10E2000054F094FB01994A2054F090FB204602B050
:10E21000BDE87040FFF742BF2846F7F75BFE04F504
:10E22000C04393F94A312B2B90D002B070BD9FEDC3
:10E23000080A462054F0B4F89FED050A492054F02E
:10E24000AFF89FED030A4A2054F0AAF8DEE700BFBA
:10E2500000000000F8B500F5A046044696F808173F
:10E26000204876F0EFFB04F50053D3F8A83E002BCE
:10E2700037DD04F53355284676F0D4FBB76D04F549
:10E280009F461036B74208D12846012176F018FC87
:10E290003846BDE8F840FDF721BA3B6838469B6A2E
:10E2A000984701462846C1B176F07CFAC8B12846A5
:10E2B00076F018FB284676F0B7FA90B104F55B507B
:10E2C000094B0A4A062120304AF01EF93146204601
:10E2D0001522BDE8F84000F055B9BDE8F84076F0E9
:10E2E000EFBBF8BDD058002014E20C0898E40C08ED
:10E2F000F6F7A0BB0148FAF71FBD00BF102C0020A5
:10E3000008B5044A0F2344F0EDFF80F00100C0B2CD
:10E3100008BD00BFB8E50C08F8B500F54057044645
:10E32000D7F8986879F09AFC04F5A042B2F97050D9
:10E33000AB1E9BB2012B04F5005377D9D2F8DC1643
:10E34000042973D0012D92F86C50916F08BF516F62
:10E35000C5B1411A07EE901A03F2E44191ED007A3B
:10E36000DFED466AF8EE677A27EE267AF4EEC77A92
:10E37000F1EE10FA06DD032202212046BDE8F84046
:10E38000FAF796BB93F9E81403291CD1926D04F5B2
:10E390009E4124318A4270D1002E6ED0801B07EE40
:10E3A000900A03F2E443B8EE677ADFED346AD3ED06
:10E3B000007A67EEA67AB4EEE77AF1EE10FA5CDD49
:10E3C00005220321D9E7012955D0022955D19EB153
